:020000040800F2
:1000000050CB002061020008892D0008EB25000874
:10001000852D00086F040008F32F00080000000081
:10002000000000000000000000000000A101000826
:100030007304000800000000FD0100088D2D000879
:100040007B0200087B0200087B0200087B0200089C
:100050007B0200087B0200087B0200087B0200088C
:100060007B0200087B0200087B0200087B0200087C
:100070007B0200087B0200087B0200087B0200086C
:100080007B0200087B0200087B0200087B0200085C
:100090007B0200087B0200087B0200087B0200084C
:1000A0007B020008852E00087B0200087B02000806
:1000B0007B020008952E00087B0200087B020008E6
:1000C0007B0200087B0200087B0200087B0200081C
:1000D0007B0200087B0200087B0200087B0200080C
:1000E0007B0200087B0200087B0200087B020008FC
:1000F0007B0200087B0200087B0200087B020008EC
:100100007B0200087B0200087B0200087B020008DB
:100110007B0200087B0200087B0200087B020008CB
:100120007B0200087B0200087B0200087B020008BB
:100130007B020008810500087B0200087B020008A2
:100140007B0200087B0200087B0200087B0200089B
:100150007B0200087B0200087B0200087B0200088B
:100160007B0200087B0200087B0200087B0200087B
:100170007B0200087B0200087B02000800000000F0
:100180007B0200087B020008DFF810D000F032F993
:100190000048004775620008AFF3008050CB002094
:1001A0002C4B19680868B0E8F04F80F30988BFF35A
:1001B0006F8F4FF0000080F311887047000000003F
:1001C00008480068006880F308884FF0000080F35A
:1001D000148862B661B6BFF34F8FBFF36F8F00DF35
:1001E00000BF00BF08ED00E0DFF80C00016841F43B
:1001F00070010160704700BF88ED00E0EFF30980F7
:10020000BFF36F8F134B1A681EF0100F08BF20ED5D
:10021000108A20E9F04F106009B44FF0500080F3CD
:100220001188BFF34F8FBFF36F8F11F0FFF94FF0BD
:10023000000080F3118809BC19680868B0E8F04F25
:100240001EF0100F08BFB0EC108A80F30988BFF3CE
:100250006F8F70475C000020EFF30580704700004F
:100260000648804706480047FEE7FEE7FEE7FEE750
:10027000FEE7FEE7FEE7FEE7FEE7FEE7712E000879
:10028000890100082DE9F05F0546002092469B4653
:1002900088460646814640241BE02846414647469C
:1002A000224600F097F853465A46C01A914110D39F
:1002B00011461846224600F07EF82D1A67EB010819
:1002C0004F4622460120002100F075F817EB000987
:1002D0004E41201EA4F10104DFDC484631462A4687
:1002E0004346BDE8F09F00000649074A08685043AE
:1002F00043F2390210440860400870470149086021
:1003000070470000980100206D4EC64110B5431A99
:10031000934209D28318881803E010F8011D03F8EE
:10032000011D521EF9D210BD40EA01039B0703D004
:1003300009E008C9121F08C0042AFAD203E011F824
:10034000013B00F8013B521EF9D210BDD2B201E0D0
:1003500000F8012B491EFBD270470022F6E710B5CA
:1003600013460A4604461946FFF7F0FF204610BD23
:1003700030B504460020034600E05B1C934203D2E4
:10038000E05CCD5C401BF8D030BD30B50B4601467B
:1003900000202022012409E021FA02F59D4205D324
:1003A00003FA02F5491B04FA02F52844151EA2F1CE
:1003B0000102F1DC30BD202A04DB203A00FA02F110
:1003C000002070479140C2F1200320FA03F3194343
:1003D00090407047202A04DB203A21FA02F00021E5
:1003E000704721FA02F3D040C2F120029140084345
:1003F00019467047064C074D06E0E06840F00103DF
:1004000094E8070098471034AC42F6D3FFF7C0FEDB
:10041000B42B0108D42B010870B58C1810F8015BBF
:1004200015F0070301D110F8013B2A1106D110F88D
:10043000012B03E010F8016B01F8016B5B1EF9D191
:100440002B0705D40023521E0DD401F8013BFAE717
:1004500010F8013BCB1A921C03E013F8015B01F882
:10046000015B521EF9D5A142D8D3002070BD00BF58
:10047000FEE7704710B50146002226E002EB820439
:100480000B6903EBC4000023036043608360C36017
:10049000036243624FF0004303604FF48C434360B8
:1004A000436823F00043436001F1480343F822000E
:1004B000032A07D202EB82040B6903EBC40328333F
:1004C000C36001E00B69C360521C042AD6D3002428
:1004D000CC650C668C66CC668C650B6803F5805326
:1004E0000C69DC6010BD10B50146002222E002EB71
:1004F0008204CB6803EBC400002303604360836085
:10050000C36001F1180343F82200036843F4801329
:100510000360032A07D202EB8204CB6803EBC40317
:100520002833C36001E0CB68C360036843F4400331
:100530000360521C042ADAD300248C620B6803F592
:100540008053CC681C6110BD38B504460020009073
:10055000206800F58050806940F48011206800F523
:1005600080508161206800F58050806900900120F2
:1005700000F0BEFA0099206800F58050816138BD16
:1005800010B5024800F050FB10BD0000B84F00202D
:1005900030B503461479557944EA0520084C0C44DB
:1005A0002064D4782406957844EA0544557844EAD2
:1005B0000524157844EA0500014C0C44606430BD04
:1005C0000080024010B5A4B0044601208DF83C0024
:1005D0008DF83D0000200D908DF84B0001208DF826
:1005E0004A0000208DF8480001208DF830000020DE
:1005F0008DF84C008DF83B0014908DF854001D9040
:100600008DF878001F908DF882008DF880004FF4EF
:1006100080401090C010119000208DF881000BA92F
:10062000204600F095F901208DF80C008DF80D00A2
:100630008DF81D008DF80E00002005908DF81C002F
:100640008DF81E00089001208DF824008DF804001C
:1006500000040290800106904012049001208DF861
:10066000250000200A9000906946204600F010F90D
:1006700024B010BD0020704710B501F07BF810BD0C
:1006800010B5024800F0D2FD002010BDB84F002088
:1006900070B504460D46164633462A4621460448A0
:1006A00000F0F6FC10B14FF0FF3070BD0020FCE709
:1006B000B84F002070B504460D46164633462A460C
:1006C0002146044800F00FFF10B14FF0FF3070BD1D
:1006D0000020FCE7B84F00202DE9F04F80460C4683
:1006E000164608F118031A69D3F810904FF0000C61
:1006F00053F82210A568E246086800F00040B0F107
:10070000004F04D003F1140050F8220010B1022071
:10071000BDE8F08F0CF1010C2868886048686FF321
:100720000C00D5F804B040EA0B004860207800F0D7
:10073000010038B1086820F44000D4F814B040EA51
:100740000B000860207800F0200038B1086820F025
:100750004060D4F810B040EA0B000860207800F048
:10076000040018B1086840F080000860086840F094
:100770008050086000BF00BF00BFBFF35F8F00BFA5
:1007800000BF00BF086840F0004008605DE00868F6
:1007900020F00050086026B1086840F080400860F2
:1007A00003E0086820F08040086000BF521C042A63
:1007B00000D3121F00BF53F82210086820F08050A9
:1007C0000860086800F00040B0F1004F04D003F169
:1007D000140050F82200E8B14A4653F822100027CE
:1007E00014E000BF00BF00BFBFF35F8F00BF00BFBA
:1007F00000BF086820F00040086000BF521C042AB7
:1008000000D3121F00BF53F822107F1C6745E8D3A6
:1008100002207DE70CF1010CAD682868886048680B
:100820006FF30C00D5F804B040EA0B0048600AF101
:10083000010A00BF00BF00BFBFF35F8F00BF00BF52
:1008400000BF086840F000400860A86800289ED1FA
:1008500026B1086840F08040086003E0086820F096
:1008600080400860086840F00050086003F1140000
:10087000D3F824B040F822B01A6172B60AF1010030
:10088000D3F828B05844986262B6002040E70000D0
:1008900070B505460C46286800F5805086692B48DF
:1008A0000640207B08B9012000E000208006617B23
:1008B00040EA4160617F09B9012100E0002140EA7E
:1008C0000150A17B40EA415061690843217F40EA21
:1008D000C110A17F40EA8110216A084394F82410D6
:1008E00040EA81000643286800F580508661286848
:1008F00000F580508669012000F0FAF8286800F5BC
:10090000805086612179A06840EA4160A16908436E
:100910002169084394F8251040EAC110A16A40EA11
:1009200081002168084340F40001286800F58050E8
:100930000160286800F580500668012000F0D8F8B2
:10094000286800F58050066070BD0000233FDEF887
:1009500070B505460C46286806683A480640207C73
:1009600008B9012000E00020C005617C09B901211F
:1009700000E0002140EA8150A1680843E17F40EA9D
:10098000014061690843A17F09B9012100E000210C
:1009900040EA4130217F40EA0130A16908432179D2
:1009A00040EA812094F8201009B9012100E00021DB
:1009B00040EA4120E17B40EAC110616A084394F8B3
:1009C000281040EA01100643286806602868066877
:1009D000012000F08DF828680660286886694FF6C7
:1009E00041700640A06C000494F84C1009B9012134
:1009F00000E0002140EAC110216D084394F8551031
:100A0000012900D100E0002140EAC10094F856100D
:100A1000012900D100E0002140EA810094F854103F
:100A2000012900D100E0002140EA41000643286886
:100A3000866128688669012000F05AF82868866176
:100A400070BD00000F8120FF2DE9F843044600200F
:100A500000904FF00108A66E04F1480050F82650AF
:100A6000E76E2FE0286A58B9684600F083FB0098CB
:100A700010B94FF0000803E0009828620098A860C1
:100A8000B8F1000F1ED0A06D10B91648686002E0E2
:100A90004FF48C40686000BF00BF00BFBFF35F8FA2
:100AA00000BF00BF00BF286840F00040286000BFC2
:100AB000761C042E00D3361F00BF04F1480050F806
:100AC00026507F1E17B1B8F1000FCBD1E06EB842AF
:100AD00006D00021206800F580508160A666E76698
:100AE000BDE8F8830046008072B600BFFEE7000054
:100AF00070B5044600F03EFE06462546681C10B15F
:100B000004480078054400BF00F034FE801BA84272
:100B1000FAD370BD5400002010B50446204600F002
:100B20000BF800F08000802803D10248006806F02E
:100B3000D7FF10BD180000200146D1F88C00704787
:100B4000024609B90120704710680068C0F3001020
:100B500081F828001068006800F0600048621068A2
:100B60000068C0F3402080F0010081F82000106888
:100B70000068C0F30040C87710680068C0F34030D8
:100B800080F00100887710680068C0F300300877B3
:100B90001068006800F4006088611068006800F464
:100BA0008040486110680068C0F3805080F0010008
:100BB000487410680068C0F3C05080F001000874E9
:100BC00010680068C0F3C010C8731068006800F4B3
:100BD0006020886010680068C0F380200871106889
:100BE0008069C0F3400081F8540010688069C0F348
:100BF000C01080F0010081F84C001068806900F09E
:100C00003000086510688069000C8864106880698D
:100C1000C0F3800081F8560010688069C0F3C000FE
:100C200081F8550000208EE710B50446206800F5D5
:100C30008050406900F0400040280FD1206800F546
:100C40008050C06900F04000402807D14249206828
:100C500000F580504161204600F0B0FA206800F5B0
:100C60008050406900F0010078B1206800F58050A4
:100C7000C06900F0010040B14FF00111206800F59B
:100C800080504161204600F01DFC206800F5805036
:100C9000406900F40040B0F5004F3DD1206800F5F8
:100CA0008050C06900F40040B0F5004F34D1D4F852
:100CB000880040F00800C4F88800206800F58050E3
:100CC000406900F40050B0F5005F15D1206800F5D0
:100CD0008050406921490840C4F88C00206800F524
:100CE0008050C06920F4C031206800F58050C16197
:100CF000E020C4F884000CE0206800F580504069D2
:100D000048F280610840C4F88C00206800F58050EB
:100D100041612046FFF700FF2068806B00F008006B
:100D200008280BD12068C06A00F06000C4F8940065
:100D3000204600F02BF90020C4F894000848006811
:100D400000F4002030B14FF400200549086020462F
:100D500000F0C8FB10BD00004000010000207E0034
:100D6000143C014038B504460CB9012038BDD4F814
:100D7000840028B92320C4F88400204600F05CF8E1
:100D800000BF002000902A48006840F480402849B5
:100D900008600846006800F48040009000BF00BF73
:100DA0002448006820F400002249086008460068D2
:100DB000A16808431F49086008460068206800F5DC
:100DC0008050006840F00101206800F5805001600B
:100DD00000F0D0FC05460DE000F0CCFC401BB0F567
:100DE000FA7F07D90420C4F88800E020C4F8840002
:100DF0000120BBE7206800F58050006800F001008A
:100E00000028E9D12046FFF7DDFB2046FFF76BFB0A
:100E10002046FFF72FFB002120466268FFF7B8FB52
:100E20000020C4F888001020C4F8840000209DE74A
:100E3000443802400438014010B586B004461421FD
:100E400001A8FFF78AFA4C49206888427ED100BF8A
:100E500000BF002000904948006840F000704749FA
:100E600008600846006800F00070009000BF00BFF6
:100E700000BF002000900846006840F080600860D5
:100E80000846006800F08060009000BF00BF00BF0F
:100E9000002000900846006840F0006008600846A6
:100EA000006800F00060009000BF00BF00BF00BFFE
:100EB000002000900846006840F0040008600846E2
:100EC000006800F00400009000BF00BF00BF0020D9
:100ED00000900846006840F001000860084600687D
:100EE00000F00100009000BF00BF00BF0020009094
:100EF0000846006840F0020008600846006800F0FC
:100F00000200009000BF00BF32200190022002903A
:100F100000200390032004900B20059001A918489D
:100F200000F016FB86200190022002900020039022
:100F3000032004900B20059001A9124800F008FB43
:100F40004FF4605001900220029000E011E0002078
:100F50000390032004900B20059001A90A4800F09B
:100F6000F7FA002205213D2000F0D0FC3D2000F0E2
:100F7000BDFC06B010BD00000080024030380240C9
:100F800000080240000002400004024070472DE9C2
:100F9000F05F04460F464FF00008C34647B9D4F847
:100FA000880040F00100C4F888000120BDE8F09FEF
:100FB000D4F88400232801D00120F7E7E66D04F17E
:100FC000480050F82650E06EC0F1040942E028685D
:100FD00000F4807018B1A969A167E96961672868A0
:100FE00000F4007008B9E06F40B3286800F40070A6
:100FF00010B1002121666166D4F814A0286800F4BD
:10100000807040B12868C0F30D40A0F1040A29683F
:1010100021674FF0010BA86828621FFA8AF304F1D8
:101020008001081F2A6A00F0D3F8206E401C206659
:10103000606E00EB0A0161660020286200BF761C2A
:10104000042E00D3361F00BF04F1480050F826508C
:1010500008F10108286800F0004020B9C84502D214
:10106000BBF1000FB3D0E06E00EB0801E166E06E6B
:1010700010B12046FFF7E8FCE665BBF1010F05D192
:10108000E06F38600021E16700208FE701208DE7E5
:101090002DE9F04705460E4617469846286804692C
:1010A00004F01C044FF4784000EAC62004434FF4D7
:1010B000F86000EA8710044324F0020444F00104BD
:1010C0002868046100F056FB81460BE000F052FBFB
:1010D000A0EB0900B0F5803F02D30120BDE8F08706
:1010E0002868046904F001000028EFD128684069ED
:1010F00080B2C8F800000020F0E72DE9F04706466E
:1011000006F11804A76AE56A4FF001082AE04FF0DB
:1011100001097F1E04F1140050F8250020B9681C55
:1011200000F003054FF00009B9F1000F1AD005EBEC
:101130008501F06850F8310000F0004080B904F1FA
:10114000140151F8250000F0C7F9002104F1140042
:1011500040F82510681C00F00305A762E56201E075
:101160004FF0000817B1B8F1000FD0D10020BDE852
:10117000F08700007CB504460D4805F0F5FD0546F6
:1011800085B105F1200020600A4828614FF4C06154
:1011900020682B464122CDE900010021084606F0D7
:1011A00055FF04E0012004490870002020607CBD48
:1011B00070280108C58700081400002010B50446F7
:1011C0000248006806F08CFC10BD000018000020EA
:1011D000F0B504460D4621462E460020A2F120001F
:1011E00000270760078143810F680FB9086001E09D
:1011F000376838603060086803E007891F4407815A
:1012000000680028F9D1F0BD70B504460D460DB94F
:10121000012070BDD4F88400102805D1294620464D
:10122000FFF796FB0020F4E70120F2E770B50646D1
:101230003068056925F01C0500F09EFC0446134843
:10124000844205D31248844202D245F008051AE0D0
:101250000F48844205D30F48844202D245F00C0562
:1012600011E00C48844203D30B48844200D20AE0C8
:101270000948844205D30948844202D245F0040556
:1012800001E045F010053068056170BD002D3101A9
:10129000C00E16020087930300E1F50580D1F00827
:1012A00070B50446D4F8840010285FD12320C4F818
:1012B00084000121A1652068C06B40F402702168A0
:1012C000C8632068D0F80C01294908432168C1F897
:1012D0000C012068D0F8100140F403102168C1F817
:1012E00010010421E1662046FFF7AEFB206800688C
:1012F00040F0080021680860206805680120FFF7B9
:10130000F7FB206805602068006840F00400216851
:101310000860206805680120FFF7EAFB2068056087
:101320002046FFF711F9206800F58050806940F4ED
:101330000051206800F580508161206800F58050E0
:10134000806940F00201206800F5805081612068CA
:1013500000F58050C06907490843216801F58051B4
:10136000C8612320C4F88400002070BD0120FCE780
:1013700060000200C1A001002DE9F0410446D4F84C
:101380008400232851D1C4F88400206800F58050DF
:10139000C06927490840216801F58051C86120686B
:1013A00000F58050806920F40051206800F58050DD
:1013B0008161206800F58050806920F0020120687A
:1013C00000F5805081612068006820F004002168E9
:1013D0000860206807680120FFF78AFB2068076023
:1013E0002046FFF7B1F82068006820F00800216867
:1013F0000860206807680120FFF77AFB2068076013
:10140000002508E004F1480050F82560706840F0BD
:10141000004070606D1C042DF4D30021A1651020E4
:10142000C4F884000020BDE8F0810120FBE7000043
:101430003E5FFEFF70B504460D463DB9D4F8880006
:1014400040F00100C4F88800012070BDD4F8840089
:10145000232835D1696BE163012229462046FFF735
:101460003BF938B1D4F8880040F00200C4F8880095
:101470000120EAE700BF00BF00BFBFF34F8F00BFEE
:1014800000BF00BF00BFA06A401CA062A06A042881
:1014900002D3A06A001FA06200BF206800F5805040
:1014A000406900F0040048B10421206800F5805034
:1014B00041610021206800F5805041600020C4E7B0
:1014C0000120C2E710B504460248006806F008FB98
:1014D00010BD00001C00002010B50446204607F097
:1014E0009DF810BD70472DE9F04705460E4617469A
:1014F00098462868046904F01C044FF4784000EA18
:10150000C62004434FF4F86000EA8710044344F017
:10151000020444F001041FFA88F029684861286831
:10152000046100F027F981460BE000F023F9A0EBFD
:101530000900B0F5803F02D30120BDE8F08728689C
:10154000046904F001000028EFD100BFF5E70000B6
:10155000F8B502460B460025002400200021D6E005
:10156000012606FA01F51E6806EA0504AC4274D1AC
:101570001E7906F00306012E04D01E7906F003063C
:10158000022E13D190684F000326BE40B0434F0097
:10159000DE68BE4030439060506801268E40B04304
:1015A0001E79C6F300168E40304350601E7906F057
:1015B0000306032E09D0D0684F000326BE40B04377
:1015C0004F009E68BE403043D0601E7906F003068F
:1015D000022E13D1CF0802F1200656F827004E073D
:1015E000F70E0F26BE40B0434F07FF0E1E69BE40E8
:1015F0003043CF0802F1200646F8270010684F005C
:101600000326BE40B0431E7906F003064F00BE40DD
:10161000304310605E6806F44036002E76D000BF7E
:10162000002600963C4E366846F480463A4F3E60AF
:101630003E46366806F48046009600BF00BF374E2F
:101640008F0856F827008E07370F0F26BE40B0438D
:10165000334EB24202D1002624E057E0314EB2426E
:1016600001D101261EE0304EB24201D1022619E01E
:101670002E4EB24201D1032614E02D4EB24201D1CA
:1016800004260FE02B4EB24201D105260AE02A4E75
:10169000B24201D1062605E0284EB24201D107260A
:1016A00000E008268F073F0FBE4030431B4E8F08D7
:1016B00046F82700224E3068A0435E6806F4801684
:1016C00006B120431E4E3060361D3068A0435E6870
:1016D00006F4001606B12043194E361D3060184E30
:1016E000361F3068A0435E6806F4003606B120431A
:1016F000134E361F3060361F3068A0435E6806F414
:10170000803606B120430E4E083E3060491C102939
:10171000FFF426AFF8BD000044380240083801400D
:10172000000002400004024000080240000C024099
:10173000001002400014024000180240001C024049
:10174000083C0140024613690B400BB1012000E048
:101750000020704710B5426921EA020302EA010441
:1017600043EA0443836110BD0AB1816101E00B04C7
:101770008361704701480068704700004C000020FA
:101780000148006870470000107AFF1F0148006898
:1017900070470000147AFF1F01480068704700007E
:1017A000187AFF1F03480068034909780844014973
:1017B000086070474C0000205400002010B50D4810
:1017C000006840F400700B4908600846006840F467
:1017D000806008600846006840F48070086003205C
:1017E00000F0D2F80F2000F007F800F055F80020C4
:1017F00010BD0000003C0240F0B587B00446002652
:10180000002700BF002000901E48006840F0010043
:101810001C4908600846006800F00100009000BF05
:1018200000BF01A902A800F085F900F0ABF946005D
:101830001548B6FBF0F0471E14481549086040F201
:10184000E7311348C1604760002101618160816117
:1018500000F0AAFC054695B90D4800F011FD0546BB
:101860006DB9192000F042F8102C07D20022214651
:10187000192000F04BF80748046000E001252846D5
:1018800007B0F0BD4438024040420F000000014064
:10189000AC0400205000002008B500BF00200090DC
:1018A0001148006840F480400F490860084600680D
:1018B00000F48040009000BF00BF00BF00200090F7
:1018C000081F006840F08050091F08600846006843
:1018D00000F08050009000BF00BF00220F21901E3A
:1018E00000F014F808BD00004438024001460846E4
:1018F000002809DB00F01F0301229A4043099B00E6
:1019000003F1E023C3F8002100BF70472DE9F05F29
:1019100080460D461646002701F07EFB07463946F5
:101920002A46334601F00700C0F1070ABAF1040F56
:1019300002D94FF0040A01E0C0F1070AD14600F1D4
:10194000040ABAF1070F02D24FF0000A01E0A0F139
:10195000030AD4464FF0010A0AFA09FAAAF1010A69
:101960000AEA020A0AFA0CFA4FF0010B0BFA0CFB16
:10197000ABF1010B0BEA030B4AEA0B04214640468C
:1019800001F052FBBDE8F09F00BF00F00702064BDC
:1019900019684FF6FF031940044B0B4343EA022139
:1019A000014B196000BF70470CED00E00000FA0524
:1019B00070B504460D460CB9012070BD584800684A
:1019C00000F00700A84209D255490D70084600688A
:1019D00000F00700A84201D00120EEE7207800F0D7
:1019E000020002281DD1207800F00400042805D14F
:1019F0004C48006840F4E0504A490860207800F004
:101A00000800082805D14748006840F4604045496F
:101A100008604448006820F0F000A168084341498C
:101A20000860207800F00100A8B36068012807D1A1
:101A30003C4808380068C0F34040B8B90120BCE712
:101A40006068022802D06068032807D1354808384A
:101A50000068C0F3406048B90120AEE7314808385B
:101A60000068C0F3400008B90120A6E72D480068CF
:101A700020F00300616808432A490860FFF77AFEF6
:101A8000064609E0FFF776FE801B41F28831884266
:101A900002D9032091E707E02248006800F00C001B
:101AA0006168B0EB810FEDD11D48006800F00700C0
:101AB000A84209D91A490D700846006800F00700CD
:101AC000A84201D0012078E7207800F00400042823
:101AD00007D11448006820F4E050E1680843114938
:101AE0000860207800F00800082808D10D48006838
:101AF00020F46040216940EAC1000A49086000F012
:101B000051F808490968C1F30311074A515CC840FC
:101B10000649086006480068FFF76EFE00204CE7A3
:101B2000003C024008380240B42801085800002058
:101B3000500000200F2202600D4A126802F00302DA
:101B400042600B4A126802F0F0028260084A126892
:101B500002F4E052C260064A126802F46042D208FF
:101B60000261044A126802F007020A60704700002E
:101B700008380240003C02400148006870470000FD
:101B80005800002000B5FFF7F7FF04490968C1F3CA
:101B90004231034A515CC84000BD00000838024091
:101BA000C42801082DE9F047002400250026A1469D
:101BB0002548006800F00C0020B1042805D0082852
:101BC0003AD105E0DFF8849039E0DFF8849036E020
:101BD0001D48001F006800F03F041B48001F0068FC
:101BE00000F4800078B11A481749091F0968C1F349
:101BF0008811A0FB01700146224600233846FEF7FB
:101C000041FB05460EE011480F49091F0968C1F361
:101C10008811A0FB01700146224600233846FEF7DA
:101C200031FB05460848001F0068C0F30140401C16
:101C30004600B5FBF6F902E0DFF8109000BF00BFE8
:101C40004846BDE8F0870000083802400024F40050
:101C500000C0A800F8B504460CB90120F8BD2078F2
:101C600000F00100002874D0F948006800F00C0072
:101C700004280DD0F648006800F00C00082813D1A5
:101C8000F348001F006800F48000B0F5800F0BD10E
:101C9000EF4808380068C0F34040002859D0606819
:101CA000002856D10120D9E700BF6068B0F5803F19
:101CB00008D1E7480838006840F48030E449083922
:101CC00008601EE06068B0F5A02F0DD1E04808382C
:101CD000006840F48020DE49083908600846006842
:101CE00040F4803008600CE0D9480838006820F4DF
:101CF0008030D749083908600846006820F4802001
:101D0000086000BF606890B1FFF734FD054606E04B
:101D1000FFF730FD401B642801D903209EE7CC4823
:101D200008380068C0F340400028F1D011E0FFF708
:101D300021FD054606E0FFF71DFD401B642801D983
:101D400003208BE7C24808380068C0F340400028F1
:101D5000F1D1207800F0020002285FD1BC48006871
:101D600000F00C0058B1BA48006800F00C000828D8
:101D70001CD1B748001F006800F48000B0B9B44817
:101D800008380068C0F3400020B1E068012801D0A5
:101D9000012063E7AE480838006820F0F8002169A8
:101DA00040EAC100AA490839086037E0E06800B39A
:101DB0000120A8490860FFF7DDFC054606E0FFF7B3
:101DC000D9FC401B022801D9032047E7A048083866
:101DD0000068C0F340000028F1D09D480838006832
:101DE00020F0F800216940EAC100994908390860EB
:101DF00014E0002097490860FFF7BCFC054606E0A8
:101E0000FFF7B8FC401B022801D9032026E79048C1
:101E100008380068C0F340000028F1D1207800F0B5
:101E2000080008282CD16069A8B101208A490860FF
:101E3000FFF7A0FC054606E0FFF79CFC401B0228CC
:101E400001D903200AE782486C300068C0F34000E3
:101E50000028F1D014E000207F490860FFF78AFCD9
:101E6000054606E0FFF786FC401B022801D9032047
:101E7000F4E677486C300068C0F340000028F1D1E8
:101E8000207800F00400042870D100277048383012
:101E9000006800F0805090B900BF002000906C48AE
:101EA0003830006840F08050694938310860084691
:101EB000006800F08050009000BF00BF0127674815
:101EC000006800F48070B0B96448006840F4807025
:101ED00062490860FFF74EFC054606E0FFF74AFC42
:101EE000401B022801D90320B8E65C48006800F4D2
:101EF00080700028F2D000BFA068012808D15448A3
:101F00006830006840F001005149683108601DE008
:101F1000A06805280DD14E486830006840F00400E4
:101F20004B49683108600846006840F001000860CD
:101F30000CE047486830006820F0010044496831EF
:101F400008600846006820F00400086000BFA06830
:101F5000A8B1FFF70FFC054609E0FFF70BFC401B9B
:101F600041F28831884202D9032077E626E03848DA
:101F700068300068C0F340000028EED013E0FFF79F
:101F8000F9FB054608E0FFF7F5FB401B41F28831FD
:101F9000884201D9032061E62D4868300068C0F30B
:101FA00040000028EFD1012F07D1294838300068C0
:101FB00020F0805026493831086000BFA069002811
:101FC00045D02348006800F00C0008285DD0A069C7
:101FD000022845D100201F490866FFF7CBFB0546C4
:101FE00006E0FFF7C7FB401B022801D9032035E6B6
:101FF000174808380068C0F340600028F1D1D4E9E0
:1020000007010843616A40EA81110122A06AC2EB1C
:10201000500041EA00412C20005D41EA00600C497B
:10202000091F086001200B490866FFF7A3FB05465E
:1020300006E0FFF79FFB401B022801D903200DE6B5
:10204000034808380068C0F340600028F1D049E038
:102050000838024000004742800E474200700040AE
:10206000002021490866FFF785FB054606E0FFF7DB
:1020700081FB401B022801D90320EFE51B480068C3
:10208000C0F340600028F2D12CE0A069012800D103
:10209000E4E51648001D0668A069012820D006F472
:1020A0008001E06981421BD106F03F01206A814234
:1020B00016D147F6C0703040616AB0EB811F0FD176
:1020C00006F440310122A06AC2EB5000B1EB004F90
:1020D00006D106F070612C20005DB1EB006F01D0DD
:1020E0000120BBE50020B9E500004742003802406E
:1020F0007047704730B502460B4600BF92F83C006F
:10210000012801D1022030BD012082F83C0000BF2F
:10211000022082F83D00106844681068816824F04D
:1021200070041868044310684460184D1068A84291
:102130001BD01068B0F1804F17D0154D1068A84221
:1021400013D0144D1068A8420FD0134D1068A84248
:102150000BD0124D1068A84207D0114D1068A8424C
:1021600003D0104D1068A84205D121F080015868B5
:10217000014310688160012082F83D0000BF00200B
:1021800082F83C0000BF00BFBDE700000000014036
:102190000004004000080040000C00400004014022
:1021A000004001400018004010B504460CB9012061
:1021B00010BD94F83D0028B9002084F83C0020466A
:1021C00000F026F8022084F83D00211D206800F070
:1021D00069FE012084F8460000BF84F83E0001211A
:1021E0003F200155402001554120015500BF00BF4F
:1021F000012084F842004320015544200155452028
:10220000015500BF012084F83D000020D0E7000008
:1022100038B504462068B0F1804F0FD100BF0020D0
:1022200000901548006840F0010013490860084616
:10223000006800F00100009000BF1BE00F4920681B
:10224000884217D100BF002000900B48006840F082
:102250000200094908600846006800F0020000908A
:1022600000BF00BF002205211D20FFF74FFB1D20EE
:10227000FFF73CFB38BD000040380240000400403E
:10228000014691F83D00012801D00120704702204D
:1022900081F83D000868C06840F001000B68D86014
:1022A0001A4B086898421BD00868B0F1804F17D0CD
:1022B000174B0868984213D0164B086898420FD005
:1022C000154B086898420BD0144B0868984207D009
:1022D000134B0868984203D0124B086898420CD1FF
:1022E0000868806800F00702062A0CD008680068B9
:1022F00040F001000B68186005E00868006840F0D5
:1023000001000B6818600020C0E7000000000140D9
:102310000004004000080040000C004000040140A0
:1023200000400140001800402DE9F04104460D46F0
:10233000002700BF94F83C00012802D10220BDE82C
:10234000F081012084F83C0000BF022084F83D00A9
:102350002068866826F0770626F47F462068866027
:102360002868502833D00CDC202850D004DC00280A
:102370004BD0102851D149E0302849D040284CD1C9
:1023800039E060282DD0702807D0B0F5805F03D0E9
:10239000B0F5005F41D10DE041E0D5E902136A6874
:1023A000206800F0EBFD2068866846F0770620681C
:1023B000866034E0D5E902136A68206800F0DEFD2B
:1023C0002068806840F480402168886027E0EA68DF
:1023D0006968206800F0E6FD5021206800F0D9FD12
:1023E0001DE0EA686968206800F0EFFD6021206860
:1023F00000F0CFFD13E0EA686968206800F0D2FDC4
:102400004021206800F0C5FD09E000BF00BF00BF0B
:102410002968206800F0BDFD01E0012700BF00BF72
:10242000012084F83D0000BF002084F83C0000BF7C
:10243000384684E7704710B5044620680069C0F349
:102440004000D8B12068C068C0F34000B0B16FF060
:10245000020021680861012020772068806900F06F
:10246000030018B12046FFF7E5FF05E0204600F025
:10247000ADF8204600F0ABF8002020772068006916
:10248000C0F38000D8B12068C068C0F38000B0B14C
:102490006FF00400216808610220207720688069BD
:1024A00000F4407018B12046FFF7C4FF05E0204655
:1024B00000F08CF8204600F08AF800202077206891
:1024C0000069C0F3C000D8B12068C068C0F3C00084
:1024D000B0B16FF0080021680861042020772068FF
:1024E000C06900F0030018B12046FFF7A3FF05E024
:1024F000204600F06BF8204600F069F800202077B5
:1025000020680069C0F30010D8B12068C068C0F32B
:102510000010B0B16FF0100021680861082020772A
:102520002068C06900F4407018B12046FFF782FFB0
:1025300005E0204600F04AF8204600F048F8002068
:1025400020772068006900F0010058B12068C06859
:1025500000F0010030B16FF00100216808612046F1
:1025600000F036F820680069C0F3C01058B1206848
:10257000C068C0F3C01030B16FF0800021680861FE
:102580002046FFF7B5FD20680069C0F3801058B100
:102590002068C068C0F3801030B16FF0400021683F
:1025A0000861204600F020F820680069C0F3401060
:1025B00058B12068C068C0F3401030B16FF02000FF
:1025C000216808612046FFF794FD10BD70477047F1
:1025D00010B5044603492068884201D1FFF7E2F8AC
:1025E00010BD000000000140704700BFFEE738B595
:1025F0000446002000906A460121636920689847DC
:10260000002802DA6FF0040038BD6A4601216369D0
:1026100020689847002802DA6FF00400F4E7009879
:1026200000F0040008B90120EEE76A460021636962
:1026300020689847002802DA6FF00400E4E7009869
:1026400000F48050B0F5805F1FD0009800F4005077
:10265000B0F5005F07D1009800F48070B0F5807F7E
:1026600001D10220D0E7009800F40050B0F5005FDF
:1026700001D10320C8E7009800F48070B0F5807F96
:1026800001D10420C0E70520BEE76A461F21636927
:1026900020689847002802DA6FF00400B4E7009839
:1026A00000F4805008B90620AEE7009800F01C0046
:1026B000182801D10220A7E7009800F01C00082884
:1026C00001D10320A0E7009800F01C00142801D1DC
:1026D000042099E7052097E7F8B504460027002075
:1026E0000090002500266068002855D1A06808B138
:1026F000A068804720202060002513E06A46122150
:10270000284663699847002802DA6FF0040608E05B
:10271000009800F01F00A84202D12560002603E0C7
:1027200000BF6D1C1F2DE9D900BF20681F2801D9EB
:102730006FF0020656BB4FF4004200212369206867
:102740009847002826DB6A4600216369206898477D
:1027500000281CDBA0698047074612E0A06980477B
:10276000C01BB0F5FA7F09D86A460021636920686A
:102770009847002805DA6FF0040607E06FF00106BD
:1027800004E0009800F400400028E7D104E06FF076
:10279000040601E06FF003065EB9A06980470746B2
:1027A00000BFA0698047C01BB0F5FA6FF9D90120BE
:1027B00060603046F8BD02462AB1C86818B1886822
:1027C00008B1086910B94FF0FF3070470868906091
:1027D0004B68D360CB6853618B6813610B6993615D
:1027E0000020F2E700B595B01C2212490EA8FDF7B3
:1027F0008DFD00210EA805F0CFF90F4908601C22BD
:102800000C491C3107A8FDF781FD002107A805F040
:10281000C3F90A4908601C22064938316846FDF7A9
:1028200075FD0021684605F0B7F90549086015B047
:1028300000BD00001C280108040000200800002042
:102840000C00002000B587B0142102A8FDF785FD1B
:1028500000BF002001907548006840F010007349E7
:1028600008600846006800F01000019000BF00BF3B
:1028700000BF002001900846006840F0800008601A
:102880000846006800F08000019000BF00BF00BF54
:10289000002001900846006840F0040008600846E7
:1028A000006800F00400019000BF00BF00BF0020DE
:1028B00001900846006840F0010008600846006882
:1028C00000F00100019000BF00BF00BF0020019098
:1028D0000846006840F0020008600846006800F002
:1028E0000200019000BF00BF00BF00200190084619
:1028F000006840F0080008600846006800F0080022
:10290000019000BF00BF012211464948FEF72CFF8D
:10291000012240F206414748FEF726FF01228021AE
:102920004548FEF721FF00224FF440414148FEF7A1
:102930001BFF00224FF60F714048FEF715FF0022E3
:102940004FF490513A48FEF70FFF00224FF419411F
:102950003B48FEF709FF7F200290002003900120F2
:10296000049002A93448FEF7F3FD01200290039081
:10297000002004900120059002A92D48FEF7E8FDF3
:102980004CF20640029001200390002004900320A6
:10299000059002A92748FEF7DBFD80200290012068
:1029A0000390002004900320059002A92248FEF71E
:1029B000CFFD4FF60F70029001200390002004908D
:1029C0000320059002A91D48FEF7C2FD4FF4905068
:1029D000029001200390002004900320059002A99A
:1029E0001348FEF7B5FD4FF4194002900120039003
:1029F000002004900320059002A91148FEF7A8FDCD
:102A0000F0200290002003900120049002A90B48BE
:102A1000FEF79EFDF8200290002003900120049014
:102A200002A90448FEF794FD07B000BD303802400B
:102A3000000802400004024000100240000C024066
:102A40000000024000B58BB0C0208B490870A82060
:102A50004870012088706520C870FF208749087081
:102A6000487088700020C870C02085490870A82070
:102A70004870012088701B20C870002108460EF0A5
:102A800075F87D48007800067B49497840EA0140A6
:102A90007949897840EA01207749C97808430206D4
:102AA0007548007800067449497840EA0140724947
:102AB000897840EA01207049C978084300F47F40D2
:102AC00042EA00226C48007800066B49497840EAE7
:102AD00001416948807841EA00206749C978084384
:102AE00000F47F0042EA1022634800780106624841
:102AF000407841EA00416048807841EA00205E4920
:102B0000C978084342EA10605E4908605B48007873
:102B100000065A49497840EA01405849897840EA14
:102B200001205649C9780843020654480078000637
:102B30005249497840EA01405049897840EA0120E9
:102B40004E49C978084300F47F4042EA00224B48CE
:102B5000007800064949497840EA014147488078B1
:102B600041EA00204549C978084300F47F0042EA61
:102B700010224248007801064048407841EA00416E
:102B80003E48807841EA00203C49C978084342EA3F
:102B900010603D4908603A48007800063849497895
:102BA00040EA01403649897840EA01203449C97831
:102BB000084302063248007800063149497840EA65
:102BC00001402F49897840EA01202D49C9780843FE
:102BD00000F47F4042EA0022294800780006284994
:102BE000497840EA01412648807841EA002024499A
:102BF000C978084300F47F0042EA10222048007898
:102C000001061F48407841EA00411D48807841EAAA
:102C100000201B49C978084342EA10601B4908603C
:102C20001B481C490022194BCDE900210290164A8D
:102C30001449194804F0E4F8174804F069FC1648F0
:102C400090F83100C0F3800018B1134804F0C2FDC1
:102C500002E0114804F062FC10490F4804F0D2FC75
:102C60001C220F4904A8FDF751FB0B4904A804F0EE
:102C700093FF0BB000BD0000400000204400002086
:102C80004800002034000020380000203C000020D4
:102C9000650D01086D450008C050002091430008F3
:102CA0009828010800B587B0002003900490059093
:102CB0000690019002904FF0804013490860002078
:102CC00048600021104881607721C16000210161C6
:102CD0008161FFF769FA08B1FDF706FF4FF48050F4
:102CE000039003A90848FFF71FFB08B1FDF7FCFE9E
:102CF00000200190029001A90348FFF7FBF908B1F9
:102D0000FDF7F2FE07B000BD1C04002000B587B03F
:102D100000200390049005900690019002901748BF
:102D2000174908604DF2FF70486000211448816027
:102D300040F2E731C1600021016180218161FFF72C
:102D400033FA08B1FDF7D0FE4FF48050039003A989
:102D50000B48FFF7E9FA08B1FDF7C6FE0020019025
:102D6000029001A90648FFF7C5F908B1FDF7BCFEBE
:102D70000348FFF785FA07B000BD000000040040DB
:102D80006404002000BFFEE700BFFEE710B500BFEF
:102D9000502080F31188BFF34F8FBFF36F8F00BFB8
:102DA0000FF0FCFA18B14FF080500449086000BFE2
:102DB000002080F3118800BF10BD000004ED00E08A
:102DC00000B593B0302107A8FDF7C7FA142102A877
:102DD000FDF7C3FA00BF002001902348006840F0CF
:102DE0008050214908600846006800F0805001903A
:102DF00000BF00BF00BF002001901C48006840F4E5
:102E000080401A4908600846006800F4804001903C
:102E100000BF00BF012007900004089002200D9021
:102E200041050E910A210F91C821109102211191A3
:102E30000421129107A8FEF70DFF08B1FDF754FE1B
:102E40000F20029002200390002004904FF4A05025
:102E500005900690032102A8FEF7AAFD08B1FDF730
:102E600043FE13B000BD0000403802400070004037
:102E70000348006840F47000014908607047000092
:102E800088ED00E010B50248FFF7D5FA10BD00004C
:102E9000AC04002010B50248FFF7CDFA10BD0000C9
:102EA0006404002010B50268294B98420ED0B0F19E
:102EB000804F0BD0274B984208D0274B984205D023
:102EC000264B984202D0264B984203D122F0700242
:102ED0004B681A431E4B984220D0B0F1804F1DD052
:102EE0001C4B98421AD01C4B984217D01B4B98424F
:102EF00014D01B4B984211D01A4B98420ED01A4B4B
:102F000098420BD0194B984208D0194B984205D0E3
:102F1000184B984202D0184B984203D122F44072C9
:102F2000CB681A4322F080034C6943EA0402026032
:102F30008B68C3620B688362054B984202D0084BD2
:102F4000984201D10B6903630123436110BD000066
:102F5000000001400004004000080040000C004058
:102F6000000401400040014000440140004801408D
:102F700000180040001C00400020004030B50C4606
:102F8000816821F47F4142EA03252543294381607A
:102F900030BD0A46816821F0700142F007031943F1
:102FA0008160704730B50B461446026A056A25F009
:102FB00001050562816921F0F00141EA041122F066
:102FC0000A021A438161026230BD30B50B461446D5
:102FD000056A25F0100505628169026A21F47041D5
:102FE00041EA043122F0A00242EA03128161026246
:102FF00030BD00BFFEE700000FB4054B10B503A9BC
:10300000044A029800F034F810BC5DF814FB00008C
:10301000454600089C01002002480068C0F30220D9
:10302000704700000CED00E010B5002804DB0A0733
:10303000130E054A135406E00A07140E034A00F063
:103040000F031B1FD45410BD00E400E018ED00E096
:1030500002E008C8121F08C1002AFAD17047704761
:10306000002001E001C1121F002AFBD170470000BF
:103070002DE9FF4F8BB09A460F460546002606E025
:1030800025280BD052460D9990476D1C761C287848
:103090000028F5D10FB03046BDE8F08F0024A046DF
:1030A0000122604900E0044315F8013F203B02FA89
:1030B00003F00842F7D128782E2817D115F8010F10
:1030C00044F004042A280ED06FF02F022878A0F1D3
:1030D000300109290AD808EB880102EB410100EB15
:1030E00001086D1CF2E757F8048B6D1C28786928DD
:1030F0003ED006DC0028CDD063280BD0642804D154
:1031000036E0732810D075284BD052460D99904761
:10311000761C85E017F8040B8DF8000000208DF870
:103120000100E946012003E057F8049B4FF0FF300F
:1031300061074FF0000401D40AE0641C44450DDA35
:103140008442FADB19F804100029F6D106E0641C69
:103150008442FCDB19F804100029F8D1264404E06D
:1031600019F8010B52460D999047641EF8D257E0AA
:1031700001CF4FF00A0B002802DA40422D2102E075
:10318000210504D52B218DF82410012103E0E1074E
:1031900005D02021F7E70DF1200908910CE000216E
:1031A000F9E701CF4FF00A0BF9E75946FDF7EDF8C3
:1031B00001F1300209F8012D0028F6D1ADEB09002C
:1031C00000F1200B600701D44FF00108D84502DD63
:1031D000A8EB0B0000E000208046002406E009A8D0
:1031E0005246005D0D999047641C761C08988442F5
:1031F000F5DB04E0302052460D999047761CB8F17B
:103200000001A8F10108F5DC05E019F8010B5246B0
:103210000D999047761CBBF10001ABF1010BF4DC7A
:103220006D1C34E7092801002DE9F04104460D46E4
:1032300016460727AA2020706670A878A070E87844
:10324000E07000202071F81E81B2601C0FF0D8FAE7
:1032500060713C20A071BDE8F08100002DE9F041D3
:1032600004460D4600BF05F00300002808D000BF4B
:103270000BA34FF4B67216A11DA0FFF7BDFE00BF51
:1032800000BF2E4606F056FA0746A0680068306078
:10329000A0680660384606F059FABDE8F0810000E3
:1032A0002E2E2F4D6964646C6577617265732F549F
:1032B000686972645F50617274792F4C7749502F3E
:1032C0007372632F636F72652F6D656D702E63006F
:1032D0006D656D705F667265653A206D656D207015
:1032E000726F7065726C7920616C69676E656400DD
:1032F000417373657274696F6E2022257322206694
:1033000061696C6564206174206C696E6520256458
:1033100020696E2025730A0070B5054606F00AFA8A
:103320000646A8680468002C16D02068A9680860C2
:1033300000BF04F00300002808D000BF09A34FF429
:103340008C7214A11CA0FFF757FE00BF00BF3046CF
:1033500006F0FCF9204670BD304606F0F7F9002073
:10336000F9E700002E2E2F4D6964646C6577617259
:1033700065732F54686972645F50617274792F4C61
:103380007749502F7372632F636F72652F6D656D70
:10339000702E63006D656D705F6D616C6C6F633A6C
:1033A000206D656D702070726F7065726C79206130
:1033B0006C69676E65640000417373657274696F50
:1033C0006E2022257322206661696C656420617419
:1033D000206C696E6520256420696E2025730A00C3
:1033E00070B50546002411E004EB4400094901EBE7
:1033F000C000067D4EB104EB440001EBC0008068C4
:10340000A84202D1204600F087F9641C0A2CEBDBAD
:1034100070BD000060C600202DE9FF5F06468946AA
:1034200017464FF00A0AD346D04600240A200390DC
:10343000002002900190009000BF73E004EB440074
:10344000764901EBC000057DB8F10A0F02D10DB934
:10345000A04665E0002D63D000BF012D0AD0022DEB
:1034600008DA00BF6EA340F223127BA18AA0FFF707
:10347000C3FD00BF00BFAEB104EB4401674A02EBDD
:10348000C1013068496888420CD13FB104EB440067
:10349000114601EBC0008068B84203D1204604B059
:1034A000BDE8F09F012D28D104EB44005B4951F8A1
:1034B000300080B104EB440001EBC000418A029867
:1034C00081422DDB039404EB4400544901EBC0001E
:1034D000408A029024E004EB4400504901EBC00014
:1034E000418A019881421BDBA24604EB44004B4910
:1034F00001EBC000408A019012E0022D10DB04EBCA
:103500004400464901EBC000418A0098814207DB34
:10351000A34604EB4400414901EBC000408A0090FF
:10352000601C04B20A2C89DB09F0020028B9B8F14A
:103530000A0F05D109F0010010B94FF0FF30AEE7D6
:10354000B8F10A0F01DA444631E0BBF10A0F11DA93
:103550005C4600BF04EB4400304951F8300040B1F4
:1035600000BF2FA340F26D1255A14BA0FFF744FD01
:1035700000BF0CE0BAF10A0F01DA544607E00398E5
:103580000A2801DA039C02E04FF0FF3087E700BF12
:103590000A2C08DB00BF22A340F27F124EA13EA0FE
:1035A000FFF72AFD00BF00BF204600F0B5F800BFBE
:1035B0000A2C08DB00BF1AA340F2831246A136A0F2
:1035C000FFF71AFD00BF00BF00BF04EB4400134922
:1035D00001EBC000007D40B100BF11A34FF4C272E7
:1035E00042A12DA0FFF708FD00BF00BF36B104EBDC
:1035F00044010A4A02EBC10130684860002004EB34
:103600004401064A02EBC101488204EB4400114622
:1036100001EBC0008760204641E7000060C6002043
:103620002E2E2F4D6964646C6577617265732F541B
:10363000686972645F50617274792F4C7749502FBA
:103640007372632F636F72652F697076342F6574A0
:10365000686172702E6300007374617465203D3D73
:10366000204554484152505F53544154455F5045A2
:103670004E44494E47207C7C207374617465203E23
:103680003D204554484152505F53544154455F5387
:103690005441424C45000000417373657274696F78
:1036A0006E2022257322206661696C656420617436
:1036B000206C696E6520256420696E2025730A00E0
:1036C0006172705F7461626C655B695D2E71203D33
:1036D0003D204E554C4C000069203C204152505F2B
:1036E0005441424C455F53495A4500006172705F36
:1036F0007461626C655B695D2E7374617465203DF5
:103700003D204554484152505F53544154455F4514
:103710004D5054590000000010B5044604EB44001D
:103720000C4951F8300060B104EB4401094A52F8E9
:10373000310004F073FF002004EB4401054A42F815
:103740003100002004EB4401024A02EBC10108757C
:1037500010BD000060C60020F0B587B007460D46DA
:1037600000BF002D0AD100BF2EA340F28A223BA148
:103770003EA0FFF741FC00BF07B0F0BD00BF7C6872
:103780002088B0F5807F08D12079062805D160799E
:10379000042802D16088082803D0384604F03EFF90
:1037A000EAE7D4F80E000690A0690590686808B9A9
:1037B000002607E005986968884201D1012000E0F1
:1037C000002006460EB1012000E00220034604F16D
:1037D000080206A9284600F0CBFCE088B0F5807FFF
:1037E00003D0B0F5007F15D113E086B1022206ABFD
:1037F00004F10800291DCDE90232CDE9001005F1E0
:103800002A0302462631284600F05CFB00E000BF98
:1038100001E000E000BF00BF384604F0FFFE00BF3B
:10382000AAE700002E2E2F4D6964646C65776172E3
:1038300065732F54686972645F50617274792F4C9C
:103840007749502F7372632F636F72652F6970769B
:10385000342F6574686172702E6300006E65746940
:103860006620213D204E554C4C000000417373658D
:103870007274696F6E2022257322206661696C65FF
:1038800064206174206C696E6520256420696E2057
:1038900025730A002DE9FE4304460F461546A94646
:1038A00000BF002C08D100BF5DA340F21E326AA108
:1038B0006DA0FFF7A1FB00BF00BF00BF47B900BF6D
:1038C00057A340F21F3272A167A0FFF795FB00BF1C
:1038D00000BF00BF002D08D100BF51A34FF44872B4
:1038E0006EA161A0FFF788FB00BF00BF21462868DA
:1038F00001F09BF910B1DFF8B48186E0287800F080
:10390000F000E02816D101208DF8040000208DF889
:1039100005005E208DF80600687800F07F008DF8C5
:103920000700A8788DF80800E8788DF809000DF1F7
:10393000040869E02868A1680840D4E90112114030
:1039400088420ED0288880B24FF6A961884208D0FC
:10395000E06810B104F10C0903E06FF00300BDE86A
:10396000FE835348007800EB4000524901EBC00051
:10397000007D02281BDB4E48007800EB400001EB85
:10398000C0008068A04212D14949097801EB410189
:10399000484A02EBC101D9F800004968884206D1C3
:1039A000434802783946204600F086F8D7E70026DB
:1039B00022E006EB46003F4901EBC000007D0228F3
:1039C00018DB06EB460001EBC0008068A04211D175
:1039D00006EB4601374A02EBC101D9F800004968FD
:1039E000884207D13248067032463946204600F0F8
:1039F00063F8B4E7701CC6B20A2EDADB3A464946D1
:103A0000204600F00DF9AAE700BF4FF400604346DE
:103A100004F12A0239460090204600F025FD9EE779
:103A20002E2E2F4D6964646C6577617265732F5417
:103A3000686972645F50617274792F4C7749502FB6
:103A40007372632F636F72652F697076342F65749C
:103A5000686172702E6300006E6574696620213D96
:103A6000204E554C4C000000417373657274696FB1
:103A70006E2022257322206661696C656420617462
:103A8000206C696E6520256420696E2025730A000C
:103A90007120213D204E554C4C000000697061643E
:103AA000647220213D204E554C4C0000CC2801086A
:103AB0007801002060C60020F8B505460E46144681
:103AC00000BF04EB4400314901EBC000007D022837
:103AD00008DA00BF2EA340F2EE223BA146A0FFF77A
:103AE0008BFA00BF00BF04EB4400284901EBC00083
:103AF000007D022839D104EB440001EBC000408A6C
:103B0000B0F58E7F11DD04EB44000A4602EBC000E5
:103B1000011D284600F09CFA38BB032004EB440149
:103B20001A4A02EBC10108751FE004EB4400174973
:103B300001EBC000408AB0F5877F16DB04EB440040
:103B40000B4603EBC00000F10C0204EB440003EB56
:103B5000C000011D284600F087FA30B9032004EBAD
:103B600044010A4A02EBC10108754FF4006000905D
:103B700004EB4400054901EBC00000F10C0305F122
:103B80002A023146284600F06FFCF8BD60C60020CE
:103B90002E2E2F4D6964646C6577617265732F54A6
:103BA000686972645F50617274792F4C7749502F45
:103BB0007372632F636F72652F697076342F65742B
:103BC000686172702E6300006172705F7461626C74
:103BD000655B6172705F6964785D2E737461746592
:103BE000203E3D204554484152505F535441544576
:103BF0005F535441424C4500417373657274696F61
:103C00006E2022257322206661696C6564206174D0
:103C1000206C696E6520256420696E2025730A007A
:103C20002DE9FE4F81460F46164609F12A0A4FF04C
:103C3000FF300290002001904946386800F0F5FFFF
:103C400038B9387800F0F000E02802D00FB13868B9
:103C500018B96FF00F00BDE8FE8F4A4601213846C3
:103C6000FFF7DAFB8046B8F1000F02DA4FFA88F06E
:103C7000F1E700BFB8F17F0F08D300BF5FA340F2A8
:103C8000C1326CA16FA0FFF7B7F900BF00BF08F009
:103C9000FF0404EB4400754901EBC000007D70B9DE
:103CA0000120019004EB4401704A02EBC101087548
:103CB00004EB4400114601EBC000C0F8089000BFBF
:103CC00004EB4400694901EBC000007D01280FD0DE
:103CD00004EB440001EBC000007D022808DA00BFBD
:103CE00046A340F2CD3262A156A0FFF785F900BF8E
:103CF00000BF019800B93EB93946484600F0A8F91E
:103D000002900EB90298A6E700BF46B900BF3BA3D8
:103D100040F2E13260A14BA0FFF76EF900BF00BF97
:103D200004EB4400514901EBC000007D022811DB87
:103D30005C4804704FF40060009004EB440001EB19
:103D4000C00000F10C0352463146484600F08CFB9F
:103D5000029050E004EB4400444901EBC000007DB8
:103D6000012848D14FF0000B354618E000BF6889A4
:103D7000298988420AD1286840B100BF1FA340F2B8
:103D8000F13249A12FA0FFF737F900BF00BF287B10
:103D900000F0400010B14FF0010B02E02D68002D43
:103DA000E4D100BFBBF1000F07D032464FF42071C1
:103DB0000E2004F027FA054603E03546284604F0B5
:103DC0003DFEA5B104EB4400284951F8300030B164
:103DD00004EB4401254A52F8310004F01FFC04EBC7
:103DE0004400224941F830500020029002E04FF098
:103DF000FF30029000BF02982DE700002E2E2F4DBD
:103E00006964646C6577617265732F546869726464
:103E10005F50617274792F4C7749502F7372632F02
:103E2000636F72652F697076342F65746861727084
:103E30002E63000074797065206F766572666C6F12
:103E400077000000417373657274696F6E202225DC
:103E50007322206661696C6564206174206C696EF0
:103E60006520256420696E2025730A0060C6002045
:103E70006172705F7461626C655B695D2E73746101
:103E80007465203D3D2050454E44494E47206F7299
:103E900020535441424C45007120213D204E554C49
:103EA0004C000000780100206E6F207061636B652C
:103EB000742071756575657320616C6C6F776564CE
:103EC000210000002DE9FC5F06460F46904699460A
:103ED000DDE90CAB0020019000BF002E08D100BF2F
:103EE00031A340F257423EA141A0FFF785F800BF41
:103EF00000BF4FF420721C210E2003F0F9FE05468E
:103F00001DB94FF0FF30BDE8FC9F00BF68891C2839
:103F100008DA00BF24A340F262423FA134A0FFF7B9
:103F20006BF800BF00BF6C680F9802F04EF9E0809C
:103F300000BF96F83000062808D000BF1AA340F250
:103F4000694242492AA0FFF757F800BF00BFD9F8DD
:103F50000000A060B9F80400A081DBF80000C4F8FC
:103F60001200BBF80400E082DAF80000C4F80E008A
:103F70000E980068A0614FF4807020800820608057
:103F8000062020710420607140F6060043463A4640
:103F900029460090304600F067FA284604F03EFBC0
:103FA00000250198AFE700002E2E2F4D6964646C48
:103FB0006577617265732F54686972645F506172CE
:103FC00074792F4C7749502F7372632F636F72652A
:103FD0002F697076342F6574686172702E630000EB
:103FE0006E6574696620213D204E554C4C000000E2
:103FF000417373657274696F6E2022257322206687
:1040000061696C6564206174206C696E652025644B
:1040100020696E2025730A00636865636B207468ED
:1040200061742066697273742070627566206361C2
:104030006E20686F6C64207374727563742065748D
:10404000686172705F68647200000000702B010884
:1040500070B504460D46034A2946204600F004F890
:1040600070BD0000CC2801087FB504460D461646F9
:104070000121074A201D04F12A038DE82500039140
:10408000324619462046FFF71DFF04B070BD000000
:10409000D228010870B5002464E004EB44003349E1
:1040A00001EBC000057D002D5BD004EB440001EB6B
:1040B000C000408A401C04EB44012C4A02EBC101C1
:1040C000488204EB4400114601EBC000408AB0F581
:1040D000967F0DDA04EB440001EBC000007D01285F
:1040E0000AD104EB440001EBC000408A052803DB41
:1040F0002046FFF711FB34E004EB44001B4901EBC1
:10410000C000007D032807D1042004EB4401174AB6
:1041100002EBC101087524E004EB4400134901EBF4
:10412000C000007D042807D1022004EB44010F4A9F
:1041300002EBC101087514E004EB44000B4901EBEC
:10414000C000007D01280CD104EB44020B4603EBB8
:10415000C202111D04EB440203EBC2029068FFF798
:1041600077FF641C0A2C98DB70BD000060C600203D
:104170002DE9F84305460E461746984600BF95F8C8
:104180003000062808D000BF2EA340F2A9123BA1A0
:1041900043A0FEF731FF00BF00BF5EB1306848B1F9
:1041A0002946306800F041FD20B9307800F0F00079
:1041B000E02803D16FF00F00BDE8F8832A4641469E
:1041C0003046FFF729F90446002C01DA60B2F3E724
:1041D000022004EB44013C4A02EBC101087504EBE8
:1041E0004400114601EBC000856004EB440001EB84
:1041F000C0003968C160B9880182002004EB440125
:1042000002EBC101488204EB4400114651F8300032
:10421000B0B104EB440051F83090002004EB4401AD
:1042200042F831004FF400603B4605F12A0249464E
:104230000090284600F018F9484604F0EFF900BF56
:104240000020B9E72E2E2F4D6964646C657761728A
:1042500065732F54686972645F50617274792F4C72
:104260007749502F7372632F636F72652F69707671
:10427000342F6574686172702E6300006E65746916
:10428000662D3E6877616464725F6C656E203D3DAB
:10429000204554485F4857414444525F4C454E00C6
:1042A000417373657274696F6E20222573222066D4
:1042B00061696C6564206174206C696E6520256499
:1042C00020696E2025730A0060C600202DE9F041A8
:1042D00004460E464FF00E0860890E2800DC4FE0C1
:1042E000E07B18B996F83400401CE0736568AF892C
:1042F000287800F00100B0B12878012809D1687849
:1043000088B9A8785E280ED1607B40F010006073F9
:1043100009E006221D492846FCF72AF818B9607BF7
:1043200040F008006073082F03D0B7F5C16F22D1A9
:1043300010E096F8310000F0080000B920E0414696
:10434000204604F0CFFB00B11AE03146204600F0D1
:10435000F9FD11E096F8310000F0080000B90FE017
:104360004146204604F0BEFB00B109E0314620463C
:10437000FFF7F2F900E003E000BF0020BDE8F081A4
:10438000204604F04BF90020F8E70000CC28010893
:10439000704700009AB00646642101A8FBF7DDFFD4
:1043A00000240027A046A146354600BF2C48FEF752
:1043B0001EF9044695F83100C0F3800058B1012C75
:1043C00009DC2848FCF7D8FF284603F0A7F8284660
:1043D00003F01CF93FE095F83100C0F3800000289D
:1043E00039D1012C37DD022C06D0032C0AD0042C45
:1043F0000ED0052C17D111E04FF400694FF480481E
:10440000012711E04FF000094FF4804801270BE02D
:104410004FF400694FF00008012705E04FF0000954
:10442000C846012700E000BF00BFA7B101A90D48A1
:10443000FCF786FBCDF81C90CDF8188001A909483F
:10444000FCF7E2FE0748FCF72BFF284603F0C2F911
:10445000284603F04BF9642003F02AFAA6E700008F
:10446000A0500020B84F00202DE9F04705460E4629
:1044700017469846DDF82090484601F0A6FE824691
:104480000E21304603F0B7FB00B122E07468A4F8B7
:104490000CA0D8F800002060B8F80400A0803868AC
:1044A000C4F80600B888608100BF95F8300006287F
:1044B00008D000BF08A34FF4997215A121A0FEF700
:1044C0009BFD00BF00BF31462846AA699047BDE862
:1044D000F0876FF00100FAE72E2E2F4D6964646CAF
:1044E0006577617265732F54686972645F50617299
:1044F00074792F4C7749502F7372632F6E657469EE
:10450000662F65746865726E65742E630000000026
:104510006E657469662D3E6877616464725F6C6570
:104520006E206D757374206265203620666F722070
:1045300065746865726E65745F6F757470757421EB
:1045400000000000417373657274696F6E2022254C
:104550007322206661696C6564206174206C696EE9
:104560006520256420696E2025730A0010B5044675
:1045700000BF44B900BF0CA34FF4F17211A115A004
:10458000FEF73AFD00BF00BF732084F832007421AB
:1045900033200155194860611948A061204601F097
:1045A00075FC002010BD00002E2E2F4C5749502FB7
:1045B0005461726765742F65746865726E6574699D
:1045C000662E63006E6574696620213D204E554C51
:1045D0004C000000417373657274696F6E20222570
:1045E0007322206661696C6564206174206C696E59
:1045F0006520256420696E2025730A00953800081F
:10460000A160000806460024354600BF4FF0FF3188
:104610000B48006803F08CFA0028F7D100BF284649
:1046200001F02CFD04463CB1294620462A699047FA
:1046300010B1204603F0F2FF002CF0D1E6E70000B5
:104640001800002038B504468DF8000069460320A4
:10465000ABBE204638BD000070B50546102D69D2AE
:10466000DFE805F0080E141A20262C32383E444AA2
:1046700050565C6210213248FDF764F804465BE056
:1046800020212F48FDF75EF8044655E040212C48D4
:10469000FDF758F804464FE080212948FDF752F80D
:1046A000044649E008212748FDF74CF8044643E05A
:1046B00010212448FDF746F804463DE0202121481A
:1046C000FDF740F8044637E040211E48FDF73AF870
:1046D000044631E080211B48FDF734F804462BE006
:1046E00001211948FDF72EF8044625E0022116485D
:1046F000FDF728F804461FE004211348FDF722F8CF
:10470000044619E008211048FDF71CF8044613E0A0
:1047100010210D48FDF716F804460DE020210A4847
:10472000FDF710F8044607E040210748FDF70AF8B6
:10473000044601E0002400BF00BF204670BD000019
:10474000000C0240000402400010024070B5044614
:104750000D4600224FF480613F48FDF705F8102C0C
:1047600076D2DFE804F0080F161D242B32394047BB
:104770004E555C62686F2A464FF480613748FCF7FB
:10478000F3FF66E02A464FF400613448FCF7ECFF83
:104790005FE02A464FF480513048FCF7E5FF58E0CF
:1047A0002A464FF400512D48FCF7DEFF51E02A461F
:1047B0004FF480412948FCF7D7FF4AE02A464FF4DE
:1047C00000412648FCF7D0FF43E02A464FF4007131
:1047D0002348FCF7C9FF3CE02A464FF4807121488A
:1047E000FCF7C2FF35E02A464FF400611D48FCF794
:1047F000BBFF2EE02A464FF480511A48FCF7B4FF65
:1048000027E02A464FF400411648FCF7ADFF20E0B0
:104810002A464FF480511248FCF7A6FF19E02A46B9
:1048200001210E48FCF7A0FF13E02A4602210B48A5
:10483000FCF79AFF0DE02A4604210848FCF794FF94
:1048400007E005E02A4608210448FCF78DFF00E058
:1048500000BF00BF70BD000000040240000C024019
:10486000000802400000024070B505460C46224692
:104870000321284600F03AF970BD00002DE9FF5FE2
:1048800005468A46654880680390039800780007CB
:10489000860E142E00DAB7E06889042800D2B3E04F
:1048A0006868047814B1082C70D100E0A6E0DFF845
:1048B0006C9109F114095948007D00F0F000E028DE
:1048C00000D1A5E0554A1168506900F0AEF900B179
:1048D0009EE02889082800D296E006F10E012846BD
:1048E00003F089F9002840D0288930441FFA80FB62
:1048F0002889584500DD8BE04FF4207259460E2080
:1049000003F0F6F9074607B982E0798906F1080055
:10491000814203D2384603F081FE79E0324678685E
:104920000399FBF7F3FC3146384604F0DBF8002826
:104930000DD000BF00BF3AA3B62247A154A0FEF796
:104940005BFB00BF00BF384603F068FE60E029460D
:10495000384603F0AFFC18B1384603F05FFE57E06D
:10496000284603F05BFE3D4611E006F10E012846A5
:1049700004F0B8F858B100BF00BF29A3C7224EA168
:1049800043A0FEF739FB00BF00BF41E024E0D5F8AB
:1049900004803146284603F02EF9E0B96F68D9F853
:1049A0000000F8601D4800693861002088F80000A8
:1049B000A8F80200FF203872002078810120002131
:1049C000FF230A46CDE9010A00914946284600F036
:1049D00099FB834600BF11E0032C0ED00B2C0CD0AA
:1049E0000C2C0AD0042C08D0052C06D00D2C04D099
:1049F0000E2C02D0112C00D000BF00BF00BF2846F3
:104A000003F00CFEBDE8FF9F284603F007FEF9E720
:104A1000284603F003FE00BFF4E70000DC8F00200F
:104A20002E2E2F4D6964646C6577617265732F5407
:104A3000686972645F50617274792F4C7749502FA6
:104A40007372632F636F72652F697076342F696399
:104A50006D702E630000000069636D705F696E7099
:104A600075743A206D6F76696E6720722D3E7061A5
:104A7000796C6F616420746F2069636D7020686564
:104A800061646572206661696C65640A00000000FB
:104A9000417373657274696F6E20222573222066DC
:104AA00061696C6564206174206C696E65202564A1
:104AB00020696E2025730A0069636D705F696E70EE
:104AC00075743A20726573746F72696E67206F72C5
:104AD0006967696E616C20702D3E7061796C6F61E1
:104AE00064206661696C65640A0000002DE9FF4777
:104AF0000746884691464FF420722421222003F075
:104B0000F7F805460DB9BDE8FF8700BF688924287E
:104B100008D200BF19A34FF4B47226A130A0FEF74B
:104B20006BFA00BF00BFD7F804A06C6884F800805F
:104B300084F801900020A080E08079686A6802F122
:104B400008001C22FBF7E2FBDAF80C00039003A834
:104B500000F040FD06465EB100206080012000218B
:104B6000FF2303AACDE901060091284600F0CAFA06
:104B7000284603F053FD00BFC5E700002E2E2F4D41
:104B80006964646C6577617265732F5468697264D7
:104B90005F50617274792F4C7749502F7372632F75
:104BA000636F72652F697076342F69636D702E6341
:104BB00000000000636865636B20746861742066A0
:104BC0006972737420706275662063616E20686F0D
:104BD0006C642069636D70206D6573736167650037
:104BE000417373657274696F6E202225732220668B
:104BF00061696C6564206174206C696E6520256450
:104C000020696E2025730A0070B505460C462246C1
:104C10000B212846FFF76AFF70BD00BFEFF3058048
:104C200008B1012070470020FCE718B50246009249
:104C3000D04300B10AB9012018BD91F8310000F04D
:104C4000020008B90020F7E74868904201D100202F
:104C5000F2E700988B681840D1E90134234098426C
:104C600008D1886822EA00008C68E343984201D1A9
:104C70000120E1E70020DFE72DE9F74F8CB0044683
:104C80000F464FF00008398DA1F11400C11700EB59
:104C90005171C1F3CF0A1420059060680990DDF8C6
:104CA000249099F8000000F00F001421B1EB800F60
:104CB00004D06FF005000FB0BDE8F08F00BF608931
:104CC00014280BDA00BF72A34FF43F727FA186A0B5
:104CD000FEF792F900BF6FF00500ECE700BFB9F8EE
:104CE000060001F072FA04900498C0F30C000790DB
:104CF000049800F400500390208914381FFA80FBB8
:104D0000BDE04FF6FF7000EACA00584501DD584685
:104D100003E04FF6FF7000EACA0008904FF42072DB
:104D200014210E2002F0E4FF054605B9ADE000BFF6
:104D30006889142808DA00BF55A34FF4497274A19A
:104D400069A0FEF759F900BF00BF142268680999ED
:104D5000FBF7DCFAD5F8049008980A9054E06189D2
:104D60000598081A80B2029000BF618905988142B7
:104D700008DA00BF46A340F22D326DA15AA0FEF71B
:104D80003BF900BF00BF02990A98884201DA0A98ED
:104D900000E002988046B8F1000F03D10020059092
:104DA000246831E000F060FC06461EB9284603F096
:104DB00035FC6AE061680598084433464122414663
:104DC000CDE90008002003F041F90B900B9830B9B1
:104DD000304600F04FFC284603F020FC55E020460A
:104DE00003F02CFE74615648306128460B9903F09D
:104DF00057F90A98A0EB080080B20A900A9810B1FF
:104E000000200590246800BF0A980028A7D10598C3
:104E1000404480B20590388D1438584501DB01209C
:104E200000E0002006900798C0F30C00049006985C
:104E300008B1039818B1049840F400500490049805
:104E400001F0C3F9A9F806000899143188B201F0FD
:104E5000BCF9A9F802000020A9F80A007B692946DC
:104E600038460E9A9847284603F0D8FB0898ABEBD3
:104E700000001FFA80FB0798504480B20790BBF1F6
:104E8000000F7FF43EAF002015E74FF0FF3012E730
:104E90002E2E2F4D6964646C6577617265732F5493
:104EA000686972645F50617274792F4C7749502F32
:104EB0007372632F636F72652F697076342F697018
:104EC000345F667261672E63000000006970345FB2
:104ED0006672616728293A207062756620746F6F68
:104EE0002073686F72740000417373657274696F28
:104EF0006E2022257322206661696C6564206174CE
:104F0000206C696E6520256420696E2025730A0077
:104F100074686973206E65656473206120706275C2
:104F20006620696E206F6E6520706965636521007B
:104F3000702D3E6C656E203E3D20706F66660000F1
:104F4000C55D00082DE9F04707460E467D682878C4
:104F50000421B1EB201F05D0384603F05FFB002091
:104F6000BDE8F087287800074FEA9068688801F06C
:104F70002CF981463989494503DD4946384603F015
:104F8000A9FC7889404505DB3889484502DBB8F142
:104F9000140F04DA384603F041FB0020E0E72869EB
:104FA00049494861E86808610846007D00F0F00062
:104FB000E0280AD196F8310000F0010018B17068BD
:104FC00008B134461CE000241AE0304600F080F8B6
:104FD00008B1344614E000243B48007D7F280FD000
:104FE0003A48046809E0B44200D105E0204600F0E8
:104FF0006FF800B103E000BF2468002CF3D100BFBC
:10500000314908693146FFF710FE28B92E48007C67
:1050100000F0F000E02804D1384603F0FFFA002049
:105020009EE724B9384603F0F9FA002098E7E888AB
:105030004FF63F71084038B1384600F04DF9074649
:105040000FB900208CE77D681F48046046608560CA
:1050500028780007800E1C4988814146384603F0B5
:1050600041FD687A012806D0062809D13146384624
:1050700005F088FE1DE031463846FFF7FFFB18E0DB
:10508000114948692146FFF7D0FD70B90E48007DEF
:1050900000F0F000E02808D00FFA88F1384603F05D
:1050A000CEFB02213846FFF7DFFB384603F0B6FAA5
:1050B00000BF00BF00200449086048608860888104
:1050C0000861486100BF4BE7DC8F00201801002019
:1050D00010B5044694F8310000F0010070B160682A
:1050E00060B1074840696168884205D00449486951
:1050F0002146FFF79AFD08B1012010BD0020FCE712
:10510000DC8F00202DE9FE4F07460C4615469846D9
:10511000DDE90C9A0E9EA34625B10CB1206808B9B2
:1051200006F1040B43462A4659463846CDE9009A13
:10513000029600F003F8BDE8FE8F00002DE9F84F5D
:1051400005460F4690469A46DDF828B00C9E00BFF3
:10515000A87B012808D000BF37A34FF4557243A1A4
:1051600045A0FDF749FF00BF00BFB8F1000F46D0D2
:105170004FF014091421284602F03DFD18B16FF0DC
:105180000100BDE8F88F6C6800BF6889142808D258
:1051900000BF29A34FF4627241A137A0FDF72CFF95
:1051A00000BF00BF84F808A00B986072D8F8000018
:1051B000206148464FEAE97109EB9171C1F387011B
:1051C00041F04001217084F801B0288900F0FDFF12
:1051D00060800020E0803E48008800F0F6FFA0805C
:1051E0003B480088401C3A4908801FB9394800688C
:1051F000E06001E03868E0600020608109E06889D3
:10520000142802DA6FF00100BBE76C682069009097
:10521000E846308D48B12889318D884205DD424607
:1052200031462846FFF728FDABE74246294630467F
:1052300073699847A5E700002E2E2F4D6964646CB2
:105240006577617265732F54686972645F5061722B
:1052500074792F4C7749502F7372632F636F726587
:105260002F697076342F6970342E6300702D3E7272
:105270006566203D3D203100417373657274696F2E
:105280006E2022257322206661696C65642061743A
:10529000206C696E6520256420696E2025730A00E4
:1052A000636865636B2074686174206669727374E7
:1052B00020706275662063616E20686F6C64207375
:1052C00074727563742069705F6864720000000016
:1052D0007A010020042A01082DE9F14F84B00498D6
:1052E0004568287800F00F001421B1EB800F00D042
:1052F00011E1E88800F069FFC0F30C004FF6FF7180
:1053000001EAC00A688800F060FF074628780007B5
:10531000810E02910299B94200DDFCE00298381A30
:1053200087B2049802F064FF06467D480188881918
:105330000A280ADD3146284600F0E6FC20B178480C
:10534000008830440A2800DDE5E07648046811E072
:105350006069E968884209D1A0692969884205D154
:10536000A089A988884201D1012000E0002000B175
:1053700002E02468002CEBD100BF34B93146284646
:1053800000F0A8FB044694B9C5E0E88800F01DFFD2
:10539000C0F30C0058B9E08900F017FFC0F30C000F
:1053A00028B11422294604F10800FAF7AFFFE88873
:1053B000012121EA50100190019850B10AEB070138
:1053C00088B2504503DB4FF6EB71884200DD80E088
:1053D00000BF2046019A049900F098F983460BF12A
:1053E000010000B975E04E48008830444C490880FF
:1053F000019840B10AEB070188B2A083A17F41F078
:105400000101A17700BFBBF1010F60D1A08B143067
:1054100080B2009060684068D0F80090606845688D
:10542000142204F108012846FAF770FF009800F0F2
:10543000CCFE68800020E8806881606804900DE000
:10544000D9F8040003901421484603F04BFB494669
:10545000049802F025FE0398D0F80090B9F1000FEF
:10546000EED130480068844202D14FF000080EE0CF
:105470002C48D0F8008006E0D8F80000A04200D107
:1054800004E0D8F80080B8F1000FF5D100BF414624
:10549000204600F0BDFA049802F0AAFE064600BFBE
:1054A0001F480088B04208DA00BF1FA340F29B22C9
:1054B0002CA133A0FDF7A0FD00BF00BF1848008855
:1054C000801B17490880049805B0BDE8F08F0020C4
:1054D000FAE700BF44B900BF13A34FF42A7232A108
:1054E00027A0FDF789FD00BF00BF606890B900BF2D
:1054F0000C480068844208D000BF0BA340F2AB22E6
:105500002CA11FA0FDF778FD00BF00BF00212046A1
:1055100000F07EFA00BF049803F080F80020D3E783
:10552000800100207C0100202E2E2F4D6964646CC8
:105530006577617265732F54686972645F50617238
:1055400074792F4C7749502F7372632F636F726594
:105550002F697076342F6970345F667261672E63CD
:105560000000000069705F72656173735F7062753F
:1055700066636F756E74203E3D20636C656E00003F
:10558000417373657274696F6E20222573222066E1
:1055900061696C6564206174206C696E65202564A6
:1055A00020696E2025730A0069707220213D204E0B
:1055B000554C4C006E6F74206669727374616C7424
:1055C000686F756768206A75737420656E7175659C
:1055D0007565640010B502462148016821E091F824
:1055E000310000F00100D8B191F83100C0F3800023
:1055F000B0B14868A0B110688B681840D1E9013497
:105600002340984201D1084610BD91F8310000F0C6
:10561000020028B91068CB68984201D10846F3E728
:1056200009680029DBD10F480068A0B10D48006867
:1056300090F8310000F0010068B10A48006890F865
:105640003100C0F3800030B106480068406810B1F6
:1056500010787F2801D10020D6E702480068D3E700
:10566000180100201C01002010B5042001F024FBCB
:1056700010BD000010B5044600BF002C08D100BFCB
:1056800006A34FF4317214A116A0FDF7B5FC00BFBC
:1056900000BF2146042001F041FA10BD2E2E2F4DEF
:1056A0006964646C6577617265732F5468697264AC
:1056B0005F50617274792F4C7749502F7372632F4A
:1056C000636F72652F697076342F6970345F66720C
:1056D00061672E63000000007020213D204E554C74
:1056E0004C000000417373657274696F6E2022254F
:1056F0007322206661696C6564206174206C696E38
:105700006520256420696E2025730A002DE9F74F76
:1057100084B006468846002501200190D8F8040090
:1057200002900299488800F050FD83460298007864
:105730000007800E03900398584503DD681E07B0EC
:10574000BDE8F08F0398ABEB00001FFA80FB0299D5
:10575000C88800F03AFDC0F30C004FF6FF7101EA73
:10576000C00A00BF00BFD8F8044000202060A4F8A1
:1057700004A00AEB0B00E080E088504502DA4FF00D
:10578000FF30DCE7D6F804903EE0D9F80470A0883A
:10579000B988884220DAC4F800909DB1A088E988D1
:1057A000884203DBE088B988884202DD4FF0FF3091
:1057B000C5E7C5F80080E888A18888420BD00020A2
:1057C000019008E0E088B988884202DD4FF0FF30A0
:1057D000B5E7C6F804801AE0A088B988884202D1EB
:1057E0004FF0FF30ABE7A088F988884202DA4FF02B
:1057F000FF30A4E72DB1E888B988884201D00020A5
:105800000190D7F800903D46B9F1000FBDD100BF1F
:10581000B9F1000F28D1002D17D000BFE888A1886A
:10582000884208DD00BF3EA34FF4DB724BA153A0BA
:10583000FDF7E2FB00BF00BFC5F80080E888A18843
:10584000884211D0002001900EE000BF706840B186
:1058500000BF33A34FF4DF7252A148A0FDF7CCFB89
:1058600000BF00BFC6F80480069820B9B07F00F0E2
:105870000100002851D00198002848D0706818B164
:1058800070684068808810B1002001903FE0254694
:10589000D4F800900BE0D9F80440E888A188884249
:1058A00002D00020019005E02546D4F80090B9F11F
:1058B000000FF0D100BF0198002828D000BF706809
:1058C00040B900BF16A340F2DF1244A12BA0FDF7A0
:1058D00093FB00BF00BF00BF70684068A04208D1C2
:1058E00000BF0FA34FF4F0723CA124A0FDF784FB8E
:1058F00000BF00BF00BF206840B100BF08A34FF445
:10590000F1723AA11DA0FDF777FB00BF00BF01981F
:1059100008B1012013E7002011E700200FE7000085
:105920002E2E2F4D6964646C6577617265732F54F8
:10593000686972645F50617274792F4C7749502F97
:105940007372632F636F72652F697076342F69707D
:10595000345F667261672E630000000063686563F0
:105960006B20667261676D656E747320646F6E275D
:1059700074206F7665726C6170000000417373650E
:105980007274696F6E2022257322206661696C65CE
:1059900064206174206C696E6520256420696E2026
:1059A00025730A006E6F2070726576696F757320BB
:1059B000667261676D656E742C2074686973206D02
:1059C00075737420626520746865206669727374EB
:1059D00020667261676D656E7421000073616E6987
:1059E000747920636865636B0000000076616C6900
:1059F000646174655F646174616772616D3A6E655C
:105A000078745F70627566213D4E554C4C00000005
:105A100070B504460D460E480068A04203D10C49FB
:105A2000206808600EE000BF002D08D100BF09A368
:105A300040F2451216A11DA0FDF7DEFA00BF00BF1F
:105A4000206828602146032001F068F870BD00003E
:105A50007C0100202E2E2F4D6964646C6577617285
:105A600065732F54686972645F50617274792F4C4A
:105A70007749502F7372632F636F72652F69707649
:105A8000342F6970345F667261672E630000000016
:105A900073616E69747920636865636B206C696EED
:105AA0006B6564206C69737400000000417373655A
:105AB0007274696F6E2022257322206661696C659D
:105AC00064206174206C696E6520256420696E20F5
:105AD00025730A0070B505460E46032001F0ECF868
:105AE000044664B93146284600F00EF9B04203DBA3
:105AF000032001F0E1F804460CB9002070BD20211C
:105B00002046FAF72AFC0F20E0770648006820605C
:105B1000044804601422294604F10800FAF7F6FB51
:105B20002046EBE77C0100202DE9F047044688463B
:105B3000002500BFA04507D100BF40A3AB224EA166
:105B400050A0FDF759FA00BF00BFB8F1000F0DD00B
:105B500000BFD8F80000A04207D000BF37A3AD2295
:105B600052A148A0FDF748FA00BF00BF6068D0F816
:105B70000490B9F80400002824D16768D9F800001F
:105B80006060142204F108017868FAF7BFFB012174
:105B90003846FFF739F8384602F02AFB064600BFC0
:105BA000A819B0F5803F07DB00BF24A3BC2244A1A5
:105BB00034A0FDF721FA00BF00BFA81985B238460E
:105BC00002F02CFD67681CE0D7F80490BA46D9F8BB
:105BD0000070504602F00CFB064600BFA819B0F555
:105BE000803F07DB00BF15A3CC2235A125A0FDF720
:105BF00003FA00BF00BFA81985B2504602F00EFD9F
:105C000000BF002FE0D141462046FFF701FF00BF53
:105C100033480088A84207DA00BF08A3D22231A186
:105C200018A0FDF7E9F900BF00BF2D480088401B10
:105C30002B4908802846BDE8F08700002E2E2F4D06
:105C40006964646C6577617265732F546869726406
:105C50005F50617274792F4C7749502F7372632FA4
:105C6000636F72652F697076342F6970345F667266
:105C700061672E63000000007072657620213D2070
:105C800069707200417373657274696F6E202225AA
:105C90007322206661696C6564206174206C696E92
:105CA0006520256420696E2025730A007072657670
:105CB0002D3E6E657874203D3D20697072000000B5
:105CC00070627566735F6672656564202B20636C15
:105CD000656E203C3D2030786666666600000000F8
:105CE0008001002069705F72656173735F70627517
:105CF00066636F756E74203E3D2070627566735FDB
:105D000066726565640000002DE9F84F0546894616
:105D1000002700BF0026B2460020009083461B48A3
:105D2000046821E06069E968884207D1A0692969AF
:105D3000884203D1A089A988884201D0012000E0CF
:105D4000002068B10BF1010B1EB92646CDF800A06A
:105D500006E0E07FF17F884202DC2646CDF800A015
:105D6000206800B1A2462468002CDBD12EB1304659
:105D70000099FFF7D9FE804647444F4502DABBF150
:105D8000010FC7DC3846BDE8F88F00007C01002019
:105D900070B500250A4804680FE0E07F002805DDA3
:105DA000E07F401EE0772546246806E0264624680A
:105DB00029463046FFF7B8FE00BF002CEDD170BD7C
:105DC0007C01002070B505462C4600BF002C08D190
:105DD00000BF0FA340F2CE221CA11FA0FDF70CF9BB
:105DE00000BF00BF00BFAC4208D000BF08A340F214
:105DF000CF2223A118A0FDF7FFF800BF00BF606904
:105E000010B1606902F00AFC2046FFF733FC70BD58
:105E10002E2E2F4D6964646C6577617265732F5403
:105E2000686972645F50617274792F4C7749502FA2
:105E30007372632F636F72652F697076342F697088
:105E4000345F667261672E63000000007063722029
:105E5000213D204E554C4C00417373657274696F3F
:105E60006E2022257322206661696C65642061744E
:105E7000206C696E6520256420696E2025730A00F8
:105E8000706372203D3D2070000000002DE9F0415C
:105E9000A2B004460027B8460026642109A8FAF7F4
:105EA0005CFA6B486B49086000208DF81C0080206C
:105EB0008DF81D00E1208DF81E0000208DF81F00D8
:105EC0008DF8200001208DF8210007A848604FF4CC
:105ED0000001604881606049C160604901614FF420
:105EE000C0614161FBF74CFCC0B28DF81F00FBF7AD
:105EF0004DFCC0B28DF82000FBF74EFCC0B28DF80F
:105F0000210007A8534948600846FAF72BFF0746C7
:105F100038215348FAF721FA2120514908604FF4FB
:105F200040004861002008614E4800F0AFFE0620A6
:105F300084F8300047484068007884F82A004548D3
:105F4000406841782B2001554248406881782C20D8
:105F5000015540484068C1782D2001553D484068B2
:105F600001792E2001553B48406841792F20015589
:105F700040F2DC50208594F8310040F00A0084F8AB
:105F800031000322002101200BF070FC364908602B
:105F90000322002101200BF069FC344908601C2217
:105FA00033496846FAF7B2F92146684601F0F4FD34
:105FB00030493148FCF7FFFB2F48FCF78DFB002FE1
:105FC00041D12D48FCF713FB0646012E06DC204686
:105FD00001F01CFB204601F0A1FA36E0022E06D0AB
:105FE000032E09D0042E0BD0052E11D10DE04FF455
:105FF00000654FF4804810E000254FF480480CE025
:106000004FF400654FF0000807E00025A84604E0C3
:106010004FF400654FF4804800BF00BF09A90D4848
:10602000FAF78EFD0F95CDF8388009A90948FBF7DE
:10603000EBF80848FBF734F9204601F0CBFB20468B
:1060400001F054FB01E0FAF74FFD22B0BDE8F0810A
:1060500000800240B84F0020184F0020784E0020EA
:106060006850002070280108180000201C00002043
:106070007C28010820000020A050002038B50446EC
:10608000002000900448007818B969460348FAF7E0
:106090007EFF009838BD000014000020B84F00209B
:1060A0002DE9F0418CB080460D46002400260027E3
:1060B00030216846FAF751F930216846FAF74DF970
:1060C0002E4629E0042C04D36FF00B000CB0BDE881
:1060D000F08104EB440170684DF82100708904EBF5
:1060E00044016A4602EB8101486054B104EB44006C
:1060F000694601EB8001601E00EB400002EB80006E
:106100008160306830B9002004EB44016A4602EB3C
:1061100081018860641C3668002ED3D128890D491E
:106120004860C1F808D008464563284602F086FC5E
:1061300008490948FBF77EF900BF4FF0FF310748D7
:10614000006801F0F5FC0028F7D10348FAF7D5FF05
:106150003846BBE768500020B84F00201C000020E4
:106160002DE9F041044625466868804703F07AFB34
:1061700006460D49286809684718B81BB0F1004F5A
:1061800001D3012000E0002030B12968881922469F
:10619000064903F0EFFB04E022460449384603F0C9
:1061A000E9FBBDE8F081000070010020616100089A
:1061B0000146080601F47F4240EA022001F47F0212
:1061C00040EA122040EA1160704701460806000CC0
:1061D00040EA11207047000008B50020009000BF81
:1061E0006846804208D000BF0BA340F25112164906
:1061F00016A0FCF701FF00BF00BF00BF00BF03F007
:10620000D9FA00F057F900F031FD01F05FF804F021
:10621000ADFD03F04FFC08BD2E2E2F4D6964646C5C
:106220006577617265732F54686972645F5061723B
:1062300074792F4C7749502F7372632F636F726597
:106240002F696E69742E63005C2A010841737365BF
:106250007274696F6E2022257322206661696C65F5
:1062600064206174206C696E6520256420696E204D
:1062700025730A00FBF7A2FAFCF7A2FDFCF7E2FA8D
:10628000FCF744FDFCF70EFDFCF7ACFA01F01CFB3B
:1062900000BFFEE701460020842901D0CA1C10443B
:1062A0007047000070B5054605B970BD05F00300E4
:1062B000002813D000BF00BF3DA340F2732248A1C5
:1062C00050A0FCF799FE00BF00BF00BF03F032FAF8
:1062D0000646304603F03AFA00BFE6E7A5F10804A7
:1062E00052480068844205D305F10C005049096802
:1062F000884213D900BF00BF2DA340F27F224DA1D9
:1063000040A0FCF779FE00BF00BF00BF03F012FA07
:106310000646304603F01AFA00BFC6E74C4803F0C1
:1063200083FA2079002816D100BF00BF20A34FF4C4
:10633000237248A133A0FCF75FFE00BF00BF4448B2
:1063400003F08AFA00BF03F0F5F90646304603F081
:10635000FDF900BFA9E7204600F026F9002816D174
:1063600000BF00BF12A340F2952244A125A0FCF774
:1063700043FE00BF00BF364803F06EFA00BF03F0D3
:10638000D9F90646304603F0E1F900BF8DE7002059
:10639000207147480068844201D245480460204685
:1063A00002F01AFC2A4803F057FA00BF7DE700000C
:1063B0002E2E2F4D6964646C6577617265732F545E
:1063C000686972645F50617274792F4C7749502FFD
:1063D0007372632F636F72652F6D656D2E6300009E
:1063E0006D656D5F667265653A2073616E6974797B
:1063F00020636865636B20616C69676E6D656E74A0
:1064000000000000417373657274696F6E2022256D
:106410007322206661696C6564206174206C696E0A
:106420006520256420696E2025730A00D4000020B1
:10643000D80000206D656D5F667265653A20696CF5
:106440006C6567616C206D656D6F7279000000008E
:10645000DC0000206D656D5F667265653A20696CD1
:106460006C6567616C206D656D6F72793A20646F41
:1064700075626C6520667265650000006D656D5F14
:10648000667265653A20696C6C6567616C206D6544
:106490006D6F72793A206E6F6E2D6C696E6B6564EC
:1064A0003A20646F75626C65206672656500000055
:1064B000E000002010B500BF00BF194820F0030025
:1064C00018490860084604684FF4C860208000201E
:1064D000608020714FF4C86002F086FF12490860A6
:1064E0000120096808714FF4C8600F4909680880E5
:1064F0000D49096848800B4800680C4908600C4841
:1065000003F09AF900280AD000BF00BF09A340F2A7
:106510001F2214A11AA0FCF76FFD00BF00BF10BD21
:10652000F78F0020D4000020D8000020E0000020D9
:10653000DC0000202E2E2F4D6964646C657761723B
:1065400065732F54686972645F50617274792F4C5F
:106550007749502F7372632F636F72652F6D656D6E
:106560002E6300006661696C656420746F2063723D
:1065700065617465206D656D5F6D7574657800008B
:10658000417373657274696F6E20222573222066D1
:1065900061696C6564206174206C696E6520256496
:1065A00020696E2025730A002DE9F041044620463B
:1065B00000F084F90546208802F016FF0646608840
:1065C00002F012FF07462088B0F5C86F10D8608827
:1065D000B0F5C86F0CD86088A84202D03888A842AD
:1065E00006D106480068864205D07088A84202D0CD
:1065F0000020BDE8F0810120FBE70000D80000206A
:106600002DE9F0478146B9F1000F02D10020BDE825
:10661000F08709F1030020F0030085B20C2D00D2B1
:106620000C25B5F5C86F01D84D4501DA0020EEE71D
:106630005C4803F0F9F85C48006800F03FF9064652
:10664000A6E0304602F0D0FE0446207900287CD136
:10665000218806F10800081AA84276D3218806F19D
:106660000800091A05F11400814229D306F1080037
:1066700028441FFA80F800BFB8F5C86F08D100BFE2
:106680004AA340F2873255A159A0FCF7B5FC00BFE0
:1066900000BF404602F0A8FE07460021397121885C
:1066A00039807E80A4F80080012020713888B0F500
:1066B000C86F07D0388802F097FEA0F8028001E08A
:1066C0000120207138480068844227D13648D0F82C
:1066D00000A004E0BAF8000002F086FE82469AF8B4
:1066E000040018B14C4800688245F3D12E48C0F828
:1066F00000A000BF00684849096888420CD02A48B9
:106700000068007940B100BF28A340F2B53243A130
:1067100037A0FCF771FC00BF00BF00BF214803F0A9
:106720009BF800BF04F1080028443B4909688842EF
:1067300008D900BF1DA340F2B9323FA12CA0FCF73D
:106740005BFC00BF00BF00BF00E01DE004F00300E1
:1067500040B100BF15A340F2BB3243A124A0FCF717
:106760004BFC00BF00BF00BF04F0030040B100BFFE
:106770000EA340F2BD3248A11DA0FCF73DFC00BFB6
:1067800000BF04F1080042E7304602F02DFE068803
:10679000C5F5C860B0423FF654AF024803F05CF85C
:1067A000002034E7DC000020E00000202E2E2F4DDA
:1067B0006964646C6577617265732F54686972648B
:1067C0005F50617274792F4C7749502F7372632F29
:1067D000636F72652F6D656D2E630000696E766163
:1067E0006C6964206E65787420707472000000001B
:1067F000417373657274696F6E202225732220665F
:1068000061696C6564206174206C696E6520256423
:1068100020696E2025730A00D80000206D656D5F29
:106820006D616C6C6F633A20216C667265652D3EFC
:1068300075736564000000006D656D5F6D616C6C63
:106840006F633A20616C6C6F6361746564206D6581
:106850006D6F7279206E6F742061626F7665207241
:10686000616D5F656E642E006D656D5F6D616C6C52
:106870006F633A20616C6C6F6361746564206D6551
:106880006D6F72792070726F7065726C7920616CB7
:1068900069676E65642E00006D656D5F6D616C6C7F
:1068A0006F633A2073616E69747920636865636B06
:1068B00020616C69676E6D656E7400000146024868
:1068C0000088081A80B27047D40000202DE9F84FE4
:1068D00081468B460BF1030020F0030085B20C2D9E
:1068E00000D20C25B5F5C86F01D85D4502DA00204D
:1068F000BDE8F88F00BF5C480068814503D35B4862
:106900000068814508D300BF59A340F2D12264A199
:1069100069A0FCF771FB00BF00BF534800688145C8
:1069200003D352480068814509D300BF02F002FF3B
:106930000090009802F00AFF00BF4846D8E7A9F18E
:1069400008063046FFF7BAFF07463188C81B0838EB
:106950001FFA80FA00BF554508DD00BF44A34FF47D
:1069600039725FA154A0FCF747FB00BF00BF55453B
:1069700001DD0020BCE7554501D14846B8E7604835
:1069800002F052FF308802F02FFD044620790028E3
:1069900033D100BF3088B0F5C86F08D100BF34A331
:1069A00040F2F52257A144A0FCF726FB00BF00BF30
:1069B0002088009007F1080028441FFA80F8564804
:1069C0000068A04204D1404602F00EFD5249086022
:1069D000404602F009FD0446002020710098208006
:1069E0006780A6F800802088B0F5C86F04D02088A2
:1069F00002F0FAFCA0F8028031E005F114005045E5
:106A00002DD807F1080028441FFA80F800BF30880D
:106A1000B0F5C86F08D100BF15A340F2163239A1F6
:106A200025A0FCF7E9FA00BF00BF404602F0DCFCFD
:106A3000044639480068844201D237480460002087
:106A40002071308820806780A6F800802088B0F50B
:106A5000C86F04D0208802F0C7FCA0F80280284844
:106A600002F0FAFE484643E7D4000020D800002098
:106A70002E2E2F4D6964646C6577617265732F5497
:106A8000686972645F50617274792F4C7749502F36
:106A90007372632F636F72652F6D656D2E630000D7
:106AA0006D656D5F7472696D3A206C6567616C200D
:106AB0006D656D6F72790000417373657274696FF3
:106AC0006E2022257322206661696C6564206174E2
:106AD000206C696E6520256420696E2025730A008C
:106AE0006D656D5F7472696D2063616E206F6E6C91
:106AF0007920736872696E6B206D656D6F727900B5
:106B0000DC000020696E76616C6964206E657874C3
:106B10002070747200000000E000002070B5044690
:106B20000D4600BF0C2C09DB00BF0AA34FF4D57241
:106B300014A11BA0FCF760FA00BF70BD00BF05B92F
:106B4000FBE7214951F824002946FCF787FB00BFE9
:106B5000F3E700002E2E2F4D6964646C6577617237
:106B600065732F54686972645F50617274792F4C39
:106B70007749502F7372632F636F72652F6D656D48
:106B8000702E63006D656D705F667265653A207486
:106B9000797065203C204D454D505F4D41580000B7
:106BA000417373657274696F6E20222573222066AB
:106BB00061696C6564206174206C696E6520256470
:106BC00020696E2025730A006829010870B5044603
:106BD0000D4600BF002C08D100BF09A340F295125A
:106BE00013A118A0FCF708FA00BF00BF04B105B953
:106BF00070BD29462046FCF731FB00BFF8E70000D6
:106C00002E2E2F4D6964646C6577617265732F5405
:106C1000686972645F50617274792F4C7749502FA4
:106C20007372632F636F72652F6D656D702E6300D5
:106C3000696E76616C696420706F6F6C2064657337
:106C400063000000417373657274696F6E202225C2
:106C50007322206661696C6564206174206C696EC2
:106C60006520256420696E2025730A0010B5002474
:106C700006E0054951F8240000F008F8601C84B2D1
:106C80000C2CF6D310BD00006829010810B50023B4
:106C9000846823604368DB1C23F00301002207E0C3
:106CA00083681B680B608368196003881944521C51
:106CB00043889342F4DC10BD70B5044600BF0C2C31
:106CC0000ADB00BF09A340F2571214A11BA0FCF776
:106CD00093F900BF002070BD00BF224951F8240085
:106CE000FCF71AFB05462846F5E700002E2E2F4D2F
:106CF0006964646C6577617265732F546869726446
:106D00005F50617274792F4C7749502F7372632FE3
:106D1000636F72652F6D656D702E63006D656D70AC
:106D20005F6D616C6C6F633A2074797065203C20F4
:106D30004D454D505F4D4158000000004173736553
:106D40007274696F6E2022257322206661696C65FA
:106D500064206174206C696E6520256420696E2052
:106D600025730A006829010810B5044600BF002CED
:106D700008D100BF07A34FF49E7212A116A0FCF722
:106D80003BF900BF00BF0CB9002010BD2046FCF746
:106D9000C3FAFAE72E2E2F4D6964646C6577617231
:106DA00065732F54686972645F50617274792F4CF7
:106DB0007749502F7372632F636F72652F6D656D06
:106DC000702E6300696E76616C696420706F6F6C01
:106DD0002064657363000000417373657274696FAA
:106DE0006E2022257322206661696C6564206174BF
:106DF000206C696E6520256420696E2025730A0069
:106E00002DE9F05F04460E4617469846DDE90AB9BB
:106E100000BF002C0BD100BF4CA340F2271258A199
:106E20005EA0FCF7E9F800BF0020BDE8F09F00BFBE
:106E300000BFB9F1000F0AD100BF44A34FF4947210
:106E400060A156A0FCF7D8F800BF0020EDE700BF16
:106E500006B9654E07B9644FB8F1000F01D1DFF8EC
:106E6000888100206060A060E06060486061002070
:106E7000208584F83100E0612062C4F824B05C48C9
:106E8000007884F834000C98206143463A46314635
:106E9000204600F0E9FA2046C84708B10020C4E7C0
:106EA00000BF94F83400FF2802D1002084F8340099
:106EB0004FF0000A4F48056829E000BFA54208D1FD
:106EC00000BF22A340F28B124BA134A0FCF794F830
:106ED00000BF00BF0AF1010A00BFBAF1FF0F08DDD1
:106EE00000BF1AA340F28D1248A12CA0FCF784F831
:106EF00000BF00BF95F8340094F83410884205D1E3
:106F000094F83400401C84F8340002E02D68002D11
:106F1000D3D100BF002DC4D194F83400FE2803D192
:106F200000203349087004E094F83400401C3049D4
:106F300008703048006820602E480460002201215B
:106F4000204600F0C5F920466FE700002E2E2F4D99
:106F50006964646C6577617265732F5468697264E3
:106F60005F50617274792F4C7749502F7372632F81
:106F7000636F72652F6E657469662E630000000092
:106F80006E657469665F6164643A20696E76616CEF
:106F90006964206E65746966000000004173736562
:106FA0007274696F6E2022257322206661696C6598
:106FB00064206174206C696E6520256420696E20F0
:106FC00025730A006E657469665F6164643A204ED9
:106FD0006F20696E69742066756E6374696F6E20C8
:106FE000676976656E000000042A01086174000874
:106FF00020010020180100206E6574696620616C14
:10700000726561647920616464656400746F6F20E7
:107010006D616E79206E65746966732C206D617880
:107020002E20737570706F72746564206E756D625A
:1070300065722069732032353500000070B5044652
:107040000D462946204604F095FE70BD70B50446F5
:107050000D4616462868E168884201D1012000E00B
:107060000020002814D100BF46B900BF09A34FF487
:10707000147215A118A0FBF7BFFF00BF00BFE068A6
:1070800030600DB9002000E02868E060012070BD8C
:107090000020FCE72E2E2F4D6964646C65776172C9
:1070A00065732F54686972645F50617274792F4CF4
:1070B0007749502F7372632F636F72652F6E6574FB
:1070C00069662E6300000000696E76616C69642059
:1070D000706F696E74657200417373657274696F65
:1070E0006E2022257322206661696C6564206174BC
:1070F000206C696E6520256420696E2025730A0066
:10710000F8B504460D46164600BF002D08D100BF55
:107110001CA340F2CB1228A12BA0FBF76DFF00BFF0
:1071200000BF00BF46B900BF16A34FF4E67222A10C
:1071300025A0FBF761FF00BF00BF28686168884297
:1071400001D1012000E00020C8B9286800906068E3
:10715000306069463046FFF771FF0DB9002000E04E
:10716000286860600121204600F00EF900BFE06948
:1071700010B12046E169884700BF0120F8BD00201A
:10718000FCE700002E2E2F4D6964646C65776172F8
:1071900065732F54686972645F50617274792F4C03
:1071A0007749502F7372632F636F72652F6E65740A
:1071B00069662E6300000000696E76616C69642068
:1071C000706F696E74657200417373657274696F74
:1071D0006E2022257322206661696C6564206174CB
:1071E000206C696E6520256420696E2025730A0075
:1071F00070B504460D4616462868A168884201D13C
:10720000012000E00020002814D100BF46B900BFD3
:1072100009A34FF4047215A118A0FBF7EDFE00BFFF
:1072200000BFA06830600DB9002000E02868A060B1
:10723000012070BD0020FCE72E2E2F4D6964646C88
:107240006577617265732F54686972645F5061720B
:1072500074792F4C7749502F7372632F636F726567
:107260002F6E657469662E6300000000696E76619A
:107270006C696420706F696E746572004173736528
:107280007274696F6E2022257322206661696C65B5
:1072900064206174206C696E6520256420696E200D
:1072A00025730A0002466AB10748016808E091F8B0
:1072B0003400401CC0B2904201D1084670470968B2
:1072C0000029F4D10020F9E71801002070470000E0
:1072D0002DE9F04105460E4617460D48046800BFEB
:1072E000002D08D100BF0BA340F2FC6216A11CA028
:1072F000FBF782FE00BF00BF05E03A463146284654
:10730000236898476468002CF7D1BDE8F08100003D
:10731000140100202E2E2F4D6964646C6577617214
:1073200065732F54686972645F50617274792F4C71
:107330007749502F7372632F636F72652F6E657478
:1073400069662E63000000006E65746966206D75C5
:10735000737420626520213D204E554C4C00000086
:10736000417373657274696F6E20222573222066E3
:1073700061696C6564206174206C696E65202564A8
:1073800020696E2025730A0070B504460D4600BFC3
:10739000002C08D100BF12A340F26D321DA126A01F
:1073A000FBF72AFE00BF00BF94F8310000F0040094
:1073B00020B194F8310000F0010000B970BD05F073
:1073C000010050B1606840B194F8310000F008004D
:1073D00018B1211D2046FCF73BFE00BFEEE7000080
:1073E0002E2E2F4D6964646C6577617265732F541E
:1073F000686972645F50617274792F4C7749502FBD
:107400007372632F636F72652F6E657469662E6386
:10741000000000006E657469665F69737375655F6F
:107420007265706F7274733A20696E76616C69640C
:10743000206E657469660000417373657274696FCC
:107440006E2022257322206661696C656420617458
:10745000206C696E6520256420696E2025730A0002
:1074600003466FF00B0070472DE9F04F87B083465D
:107470000D4616461F4600240DF10C080DF10809B3
:1074800005B9224D06B9214E07B9204F0DB1286824
:1074900008B9012000E000208246BAF1000F09D0AF
:1074A00001AA29465846FFF72BFE18B144F01004F4
:1074B00001A80490424631465846FFF799FE18B19C
:1074C00044F04004CDF814804A4639465846FFF748
:1074D000BDFD18B144F02004CDF81890BAF1000FAA
:1074E00009D101AA29465846FFF70AFE18B144F00F
:1074F000100401A8049034B144F0800404AA214689
:107500005846FFF7E5FE07B0BDE8F08F042A0108F2
:1075100001490860704700001C0100203EB5044688
:1075200000BF002C09D100BF17A340F29B3223A15A
:107530002AA0FBF761FD00BF3EBD00BF94F83100FB
:1075400000F00100F0B100208DF800006A4608212B
:107550002046FFF7BDFE00BF94F8310000F0FE00AA
:1075600084F8310000BF94F8310000F0080010B139
:107570002046FBF735FF00BFE06910B12046E16906
:10758000884700BF00BFD7E72E2E2F4D6964646C7B
:107590006577617265732F54686972645F506172B8
:1075A00074792F4C7749502F7372632F636F726514
:1075B0002F6E657469662E63000000006E65746945
:1075C000665F7365745F646F776E3A20696E76618B
:1075D0006C6964206E6574696600000041737365B0
:1075E0007274696F6E2022257322206661696C6552
:1075F00064206174206C696E6520256420696E20AA
:1076000025730A0000B10162704700003EB50446D0
:1076100000BF002C09D100BF14A340F2064220A1F4
:1076200028A0FBF7E9FC00BF3EBD00BF94F8310085
:1076300000F00400B8B100BF94F8310000F0FB0086
:1076400084F8310000BF00BF206A10B12046216AD3
:10765000884700BF00208DF800006A4604212046BC
:10766000FFF736FE00BF00BFDEE700002E2E2F4DD5
:107670006964646C6577617265732F5468697264BC
:107680005F50617274792F4C7749502F7372632F5A
:10769000636F72652F6E657469662E63000000006B
:1076A0006E657469665F7365745F6C696E6B5F6449
:1076B0006F776E3A20696E76616C6964206E6574CE
:1076C00069660000417373657274696F6E202225CC
:1076D0007322206661696C6564206174206C696E38
:1076E0006520256420696E2025730A003EB5044696
:1076F00000BF002C09D100BF16A34FF4787222A15D
:107700002AA0FBF779FC00BF3EBD00BF94F8310012
:1077100000F00400D8B900BF94F8310040F0040034
:1077200084F8310000BF03212046FFF72DFE00BF83
:10773000206A10B12046216A884700BF01208DF8D9
:1077400000006A4604212046FFF7C2FD00BF00BFCB
:10775000DAE700002E2E2F4D6964646C6577617244
:1077600065732F54686972645F50617274792F4C2D
:107770007749502F7372632F636F72652F6E657434
:1077800069662E63000000006E657469665F73654C
:10779000745F6C696E6B5F75703A20696E76616CB0
:1077A0006964206E6574696600000000417373654A
:1077B0007274696F6E2022257322206661696C6580
:1077C00064206174206C696E6520256420696E20D8
:1077D00025730A003EB5044600BF002C09D100BF46
:1077E00015A34FF4547221A127A0FBF705FC00BF9D
:1077F0003EBD00BF94F8310000F00100D0B900BFD9
:1078000094F8310040F0010084F8310000BF00BF5F
:10781000E06910B12046E169884700BF01208DF87A
:1078200000006A4608212046FFF752FD032120464A
:10783000FFF7AAFD00BFDBE72E2E2F4D6964646CB5
:107840006577617265732F54686972645F50617205
:1078500074792F4C7749502F7372632F636F726561
:107860002F6E657469662E63000000006E65746992
:10787000665F7365745F75703A20696E76616C69D6
:1078800064206E6574696600417373657274696F14
:107890006E2022257322206661696C656420617404
:1078A000206C696E6520256420696E2025730A00AE
:1078B00070B5044625460DB1294600E00121084671
:1078C00009F086FD002070BD10B509F04FFE0020C4
:1078D00010BD10B5FDF7A1F910B10AF055FD10BDAE
:1078E0000AF04CFDFBE7F8B504460D46A06840B130
:1078F000E06830B10020009094E80F0009F0E3FF49
:10790000F8BD0022D4E9000109F0B0FFF8E700005B
:107910002DE9FF4107460D461446029500200190CF
:107920003DB9802000909DE8070087E80700BDE88A
:10793000FF81002003900026601C08B9761E03E03A
:1079400014B1264606B90126FDF767F9B0B103AABE
:1079500001A928460AF0EAFA012802D11020009075
:1079600001E0002000900398B8B14FF080500E491C
:107970000860BFF34F8FBFF36F8F0EE0324601A94F
:1079800028460AF01FFA012802D11020009004E0D6
:107990000EB9002000E0402000909DE8070087E835
:1079A000070000BFC3E7000004ED00E077B581B039
:1079B0000646144600200090254605B90125FDF72E
:1079C0002CF9A8B100236A4602A930460AF00CF946
:1079D000012802D0FF2004B070BD009890B14FF094
:1079E000805009490860BFF34F8FBFF36F8F09E0E4
:1079F00000232A4602A930460AF022F8012801D0C5
:107A0000FF20E8E70020E6E704ED00E010B50446BB
:107A1000606820B10120616809F013FF10BD0120EA
:107A200009F0FEFEFAE7000038B504460025002004
:107A30000090FDF7F2F890B1694620460AF052F93D
:107A4000012801D0FF2038BD009888B14FF0805048
:107A500008490860BFF34F8FBFF36F8F08E0002322
:107A60001A461946204609F0EBFF012800D0FF25F1
:107A70002846E8E704ED00E0F8B506460C4600208D
:107A800000900EB98020F8BD0025601C08B96D1E5D
:107A900003E014B1254605B90125FDF7BEF898B1FC
:107AA0006A46002130460AF041FA012801D0FF2041
:107AB000E9E7009880B14FF0805008490860BFF3B3
:107AC0004F8FBFF36F8F07E0294630460AF094FAD4
:107AD000012801D0FF20D6E70020D4E704ED00E024
:107AE00038B50446002500200090FDF796F890B1C7
:107AF000694620460AF0F6F8012801D0FF2038BD7B
:107B0000009888B14FF0805008490860BFF34F8F4C
:107B1000BFF36F8F08E000231A461946204609F08C
:107B20008FFF012800D0FF252846E8E704ED00E09C
:107B3000F8B506460C46002000900EB98020F8BD2E
:107B40000025601C08B96D1E03E014B1254605B977
:107B50000125FDF762F898B16A46002130460AF027
:107B6000E5F9012801D0FF20E9E7009880B14FF046
:107B7000805008490860BFF34F8FBFF36F8F07E055
:107B8000294630460AF038FA012801D0FF20D6E70E
:107B90000020D4E704ED00E07FB504460D4660699F
:107BA00098B1A06988B1B4F90800FEF773FB0646E6
:107BB000D4E90510CDE9006102902B462269D4E991
:107BC00000100AF06DFB039013E0B4F90800FEF713
:107BD00061FB064603A8CDE90060238A9AB22B46D2
:107BE000D4E900100AF02AFB012802D0002004B0DA
:107BF00070BD0398FBE770B504460D460022294688
:107C0000204600F001F870BD2DE9F04704460D460E
:107C1000904600BF44B900BF1CA340F2DF1227A169
:107C200029A0FBF7E9F900BF00BF14B1B5F5803F0B
:107C300002D30120BDE8F0870DB90020FAE7AEB20B
:107C40002089304480B2B04201DA0120F2E794F892
:107C50000C9009F0800038B16068471B04F11000F7
:107C6000874209D20120E5E7B8F1000F02D0606831
:107C7000471B01E00120DDE76760608930446081D7
:107C80002089304420810020D4E700002E2E2F4D83
:107C90006964646C6577617265732F546869726496
:107CA0005F50617274792F4C7749502F7372632F34
:107CB000636F72652F706275662E63007020213DC0
:107CC000204E554C4C000000417373657274696F0F
:107CD0006E2022257322206661696C6564206174C0
:107CE000206C696E6520256420696E2025730A006A
:107CF0002DE9FE4F82460E4690465746B8F1010FD9
:107D00000AD0B8F1410F06D0B8F5C17F0BD0B8F555
:107D1000207F7DD16AE000BF42463146002000F05E
:107D200037F90446AEE0002400200290B14600BFBF
:107D30000B20FEF7C1FF054645B900F0A9FD14B1BF
:107D4000204600F06BFC0020BDE8FE8FF81C20F000
:107D50000300C0F5147080B2484501DD484605E0D7
:107D6000F81C20F00300C0F5147080B28346002098
:107D7000CDE9008005F110003844C01C20F003015B
:107D80005B464A46284600F074FD00BF287900F0A3
:107D90000300002808D000BF3CA34FF4807247A125
:107DA00052A0FBF729F900BF00BF00BFF81C20F06C
:107DB0000300C0F51470002808D100BF33A34FF4AE
:107DC000817254A149A0FBF717F900BF00BF0CB99D
:107DD0002C4601E0029805600295A9EB0B001FFA02
:107DE00080F90027B9F1000FA2DC4BE0F81C20F06D
:107DF0000301F01C20F00300084485B205F11000D7
:107E00001FFA80F9F01C20F00300A84206D800E019
:107E10002BE0F01C20F00300484501D9002093E737
:107E20004846FEF7EDFB04460CB900208CE7002025
:107E3000CDE9008004F110003844C01C20F003019B
:107E400033463246204600F014FD00BF207900F092
:107E5000030040B100BF0DA34FF491723AA123A0DB
:107E6000FBF7CAF800BF00BF0CE000BF00BF07A3CC
:107E700040F227123FA11DA0FBF7BEF800BF00BFD4
:107E8000002061E700BF20465EE700002E2E2F4D48
:107E90006964646C6577617265732F546869726494
:107EA0005F50617274792F4C7749502F7372632F32
:107EB000636F72652F706275662E630070627566FF
:107EC0005F616C6C6F633A207062756620712D3E45
:107ED0007061796C6F61642070726F7065726C791B
:107EE00020616C69676E6564000000004173736512
:107EF0007274696F6E2022257322206661696C6539
:107F000064206174206C696E6520256420696E2090
:107F100025730A00504255465F504F4F4C5F425503
:107F20004653495A45206D75737420626520626915
:107F300067676572207468616E204D454D5F414CE6
:107F400049474E4D454E5400706275665F616C6CDA
:107F50006F633A20706275662D3E7061796C6F6157
:107F6000642070726F7065726C7920616C69676EE5
:107F700065640000706275665F616C6C6F633A20C7
:107F80006572726F6E656F7573207479706500002D
:107F90002DE9FC4107460D46144600BF412C0AD08E
:107FA000012C08D000BF0EA34FF4A57218A11DA08C
:107FB000FBF722F800BF00BF0A20FEF77DFE064651
:107FC00016B90020BDE8FC8100202B462A46394620
:107FD000CDE90040304600F04CFC3046F2E70000AE
:107FE0002E2E2F4D6964646C6577617265732F5412
:107FF000686972645F50617274792F4C7749502FB1
:108000007372632F636F72652F706275662E6300E3
:10801000696E76616C696420706275665F747970F0
:1080200065000000417373657274696F6E202225CC
:108030007322206661696C6564206174206C696ECE
:108040006520256420696E2025730A002DE9FC5FF8
:1080500005460C4617469846DDE90C9BAA460AF1F0
:10806000030020F003002044584502D90020BDE859
:10807000FC9FB9F1000F06D00AF1030020F00300C5
:1080800000EB090600E00026022023462246314686
:10809000CDE90070404600F0ECFB4046E7E7000009
:1080A00070B506460D4600BF0EB1002D09D100BFC8
:1080B0001BA340F2593226A133A0FAF79DFF00BF5F
:1080C00070BD00BF344604E020892989084420811E
:1080D000246820680028F7D100BF20896189884280
:1080E00008D000BF0EA340F2623231A126A0FAF7F9
:1080F00083FF00BF00BF00BF206840B100BF08A3DE
:1081000040F2633236A120A0FAF776FF00BF00BF2D
:108110002089298908442081256000BFD0E700001C
:108120002E2E2F4D6964646C6577617265732F54D0
:10813000686972645F50617274792F4C7749502F6F
:108140007372632F636F72652F706275662E6300A2
:10815000286820213D204E554C4C292026262028D9
:108160007420213D204E554C4C29202870726F6799
:1081700072616D6D65722076696F6C6174657320D4
:108180004150492900000000417373657274696FA2
:108190006E2022257322206661696C6564206174FB
:1081A000206C696E6520256420696E2025730A00A5
:1081B000702D3E746F745F6C656E203D3D20702D98
:1081C0003E6C656E20286F66206C6173742070624F
:1081D000756620696E20636861696E290000000081
:1081E000702D3E6E657874203D3D204E554C4C0000
:1081F0000146002002E0421C90B209680029FAD131
:10820000704700002DE9F04180460E461446218952
:1082100032464046FFF76CFD074617B90020BDE81F
:10822000F0812146384600F045F8054600BF45B1CB
:1082300000BF05A340F224520FA114A0FAF7DCFE00
:1082400000BF00BF3846EAE72E2E2F4D6964646CEC
:108250006577617265732F54686972645F506172EB
:1082600074792F4C7749502F7372632F636F726547
:108270002F706275662E6300706275665F636F7043
:1082800079206661696C6564000000004173736564
:108290007274696F6E2022257322206661696C6595
:1082A00064206174206C696E6520256420696E20ED
:1082B00025730A002DE9F04105460C4600260027EB
:1082C00000BF25B11CB12889218988420CDA00BF82
:1082D00044A340F2C9324FA15AA0FAF78DFE00BF65
:1082E0006FF00F00BDE8F08100BF00BF6889801B00
:1082F0006189C91B884203D36089A0EB070802E0AB
:108300006889A0EB06086268D1196A68901942462C
:10831000F7F7FCFF4644474400BF6889B04208D2E3
:1083200000BF30A340F2D93250A146A0FAF764FE54
:1083300000BF00BF00BF6089B84208D200BF29A3B8
:1083400040F2DA324FA13FA0FAF756FE00BF00BF5D
:108350006089B84201D8002724686889B04211D1E9
:1083600000262D6800BF65B95CB100BF1DA34FF4A6
:1083700079724BA133A0FAF73FFE00BF6FF00F00F8
:10838000B0E700BF002C13D06089218988420FD14B
:1083900000BF206858B100BF12A340F2E93244A1E7
:1083A00028A0FAF729FE00BF6FF005009AE700BF8A
:1083B000002D13D06889298988420FD100BF286811
:1083C00058B100BF07A340F2EE3239A11DA0FAF761
:1083D00013FE00BF6FF0050084E700BF002C85D1BD
:1083E00000207FE72E2E2F4D6964646C65776172E3
:1083F00065732F54686972645F50617274792F4C91
:108400007749502F7372632F636F72652F70627597
:10841000662E6300706275665F636F70793A2074D0
:108420006172676574206E6F742062696720656E83
:108430006F75676820746F20686F6C6420736F7548
:1084400072636500417373657274696F6E202225D3
:108450007322206661696C6564206174206C696EAA
:108460006520256420696E2025730A006F66667397
:1084700065745F746F203C3D20705F746F2D3E6C9F
:10848000656E00006F66667365745F66726F6D205F
:108490003C3D20705F66726F6D2D3E6C656E000016
:1084A000705F746F20213D204E554C4C0000000041
:1084B000706275665F636F7079282920646F6573D9
:1084C000206E6F7420616C6C6F77207061636B65D8
:1084D0007420717565756573210000002DE9F05FEA
:1084E0008046894616461D464FF0000AD34600BF17
:1084F000B8F1000F0BD100BF21A340F20A422CA11A
:1085000033A0FAF779FD00BF0020BDE8F09F00BF5F
:1085100000BFB9F1000F0AD100BF19A340F20B420E
:1085200035A12BA0FAF768FD00BF0020EDE700BFE2
:10853000444620E035B16089A84203DC6089281AEE
:1085400085B217E06089401B87B2B74200DD37462D
:108550006268511909EB0A003A46F7F7D7FE0BEBB0
:1085600007001FFA80FB0AEB07001FFA80FAF01BD6
:1085700086B2002524680EB1002CDBD15846C4E732
:108580002E2E2F4D6964646C6577617265732F546C
:10859000686972645F50617274792F4C7749502F0B
:1085A0007372632F636F72652F706275662E63003E
:1085B000706275665F636F70795F70617274696114
:1085C0006C3A20696E76616C6964206275660000A1
:1085D000417373657274696F6E2022257322206661
:1085E00061696C6564206174206C696E6520256426
:1085F00020696E2025730A00706275665F636F7074
:10860000795F7061727469616C3A20696E76616C31
:108610006964206461746170747200002DE9F04730
:108620000446002C0ED100BF44B900BF38A34FF45C
:10863000377243A145A0FAF7DFFC00BF00BF00205E
:10864000BDE8F08700265EE001F074F8824600BFC6
:10865000A07B002808DC00BF2DA340F2F12245A139
:108660003AA0FAF7C9FC00BF00BFA07B401E00F093
:10867000FF0884F80E80504601F068F8B8F1000F4A
:108680003FD12768207B00F00F05607B00F00200DF
:10869000002814D0A14600BFD9F81000002808D146
:1086A00000BF1BA340F2FF2238A128A0FAF7A4FCC8
:1086B00000BF00BF2046D9F8101088471DE0022DEA
:1086C00004D121460B20FEF729FA16E0012D04D132
:1086D00021460A20FEF722FA0FE01DB92046FDF7D9
:1086E000E1FD0AE000BF00BF09A340F20F3230A154
:1086F00016A0FAF781FC00BF00BF701CC6B23C4652
:1087000000E0002400BF002C9ED1304698E7000016
:108710002E2E2F4D6964646C6577617265732F54DA
:10872000686972645F50617274792F4C7749502F79
:108730007372632F636F72652F706275662E6300AC
:108740007020213D204E554C4C0000004173736554
:108750007274696F6E2022257322206661696C65D0
:1087600064206174206C696E6520256420696E2028
:1087700025730A00706275665F667265653A2070DF
:108780002D3E726566203E203000000070632D3E55
:10879000637573746F6D5F667265655F66756E6332
:1087A00074696F6E20213D204E554C4C0000000036
:1087B000696E76616C696420706275662074797088
:1087C0006500000070B50446254629460748FEF7B7
:1087D000FDF907480078012806D1002004490870F7
:1087E00004480068FFF77CF970BD0000702801089C
:1087F000140000201800002070B500BF00F09AFFA0
:108800000546002009490870284600F09FFF00BF78
:108810000748046806E0606F18B1204602F05EFA6F
:1088200070BDE468002CF6D100BFF9E721010020FB
:108830003401002010B50446FFF7DEFF10BD70B50F
:1088400004460D4601222946204600F001F870BD7D
:1088500070B505460C461646002C04DA61422846DF
:1088600000F040F970BD324621462846FFF7CCF9AA
:10887000F8E770B5DDE90445002606604160028135
:10888000438104734573012686730026C67370BD49
:1088900070B500F04FFF05460C48047801200B49E5
:1088A0000870284600F052FF7CB900BF002108483C
:1088B00008F08EFB40B100F03DFF05460020034963
:1088C0000870284600F042FF00BF70BD2101002063
:1088D000358800082DE9F04106460F4600BF002EFE
:1088E00008D100BF2CA34FF4CC7237A13CA0FAF7FB
:1088F00083FB00BF00BF3089B84201DCBDE8F081D6
:108900003089C01B1FFA80F83D46344613E0608969
:10891000281A85B22089A0EB08002081246800BFB6
:1089200044B900BF1CA340F2AF1237A12CA0FAF744
:1089300063FB00BF00BF6089A842E8DB207B00F03A
:108940000F0000281BD16089A84218D0607B00F07E
:108950000200002813D1A088001B284481B22046C1
:10896000FDF7B4FF044600BF44B900BF0AA340F2BC
:10897000BD122BA11AA0FAF73FFB00BF00BF658113
:1089800060892081206810B12068FFF747FE002031
:10899000206000BFB2E700002E2E2F4D6964646C8A
:1089A0006577617265732F54686972645F50617294
:1089B00074792F4C7749502F7372632F636F7265F0
:1089C0002F706275662E6300706275665F726561F6
:1089D0006C6C6F633A207020213D204E554C4C004A
:1089E000417373657274696F6E202225732220664D
:1089F00061696C6564206174206C696E6520256412
:108A000020696E2025730A00706275665F72656169
:108A10006C6C6F633A207120213D204E554C4C0008
:108A20006D656D5F7472696D2072657475726E65C7
:108A3000642071203D3D204E554C4C0070B50446DD
:108A4000002C18D000BF00F075FE0546A07B401C2E
:108A5000A073284600F07AFE00BF00BFA07B00286C
:108A600008DC00BF04A340F242320FA113A0FAF7C2
:108A7000C3FA00BF00BF70BD2E2E2F4D6964646C19
:108A80006577617265732F54686972645F506172B3
:108A900074792F4C7749502F7372632F636F72650F
:108AA0002F706275662E630070627566207265664F
:108AB000206F766572666C6F770000004173736596
:108AC0007274696F6E2022257322206661696C655D
:108AD00064206174206C696E6520256420696E20B5
:108AE00025730A002DE9F04104460D4600BF44B944
:108AF00000BF18A340F24B2222A125A0FAF77CFA6E
:108B000000BF00BF14B1B5F5803F02D30120BDE81E
:108B1000F0810DB90020FAE7AEB200BF6089B04223
:108B20000ADA00BF0BA340F2552223A118A0FAF7DE
:108B300063FA00BF0120EAE700BF67686068284465
:108B400060606089801B60812089801B20810020FB
:108B5000DDE700002E2E2F4D6964646C657761722D
:108B600065732F54686972645F50617274792F4C19
:108B70007749502F7372632F636F72652F70627520
:108B8000662E63007020213D204E554C4C000000A5
:108B9000417373657274696F6E202225732220669B
:108BA00061696C6564206174206C696E6520256460
:108BB00020696E2025730A00696E6372656D656EAB
:108BC000745F6D61676E6974756465203C3D2070EB
:108BD0002D3E6C656E0000002DE9F041044600BF9B
:108BE0003B480068844208D200BF3AA340F2DF123B
:108BF00044A14AA0FAF700FA00BF00BF00BF5148E5
:108C00000068844208D300BF32A34FF4F0724EA133
:108C100042A0FAF7F1F900BF00BF00BF2079002899
:108C200008D000BF2BA340F2E1124EA13BA0FAF7FF
:108C3000E3F900BF00BF00BF2088B0F5C86F08D9B6
:108C400000BF24A34FF4F2724DA134A0FAF7D4F977
:108C500000BF00BF208800F0C7FB0546AC4219D01A
:108C60002879B8B937480068854213D04F48006862
:108C7000A84201D14D480460288820802888B0F59A
:108C8000C86F07D02046FDF719FE0746288800F078
:108C9000ABFB4780608800F0A7FB0646A64215D0D4
:108CA000307998B941480068A04201D13F48066038
:108CB000208830802088B0F5C86F07D03046FDF797
:108CC000FDFD0746208800F08FFB4780BDE8F0815E
:108CD000D40000202E2E2F4D6964646C657761727C
:108CE00065732F54686972645F50617274792F4C98
:108CF0007749502F7372632F636F72652F6D656DA7
:108D00002E630000706C75675F686F6C65733A2046
:108D10006D656D203E3D2072616D0000417373658D
:108D20007274696F6E2022257322206661696C65FA
:108D300064206174206C696E6520256420696E2052
:108D400025730A00D8000020706C75675F686F6C2F
:108D500065733A206D656D203C2072616D5F656EB4
:108D600064000000706C75675F686F6C65733A2013
:108D70006D656D2D3E75736564203D3D20300000AE
:108D8000706C75675F686F6C65733A206D656D2DEB
:108D90003E6E657874203C3D204D454D5F53495AE9
:108DA000455F414C49474E4544000000E00000202B
:108DB0002DE9F04105460E461C4807681C4800682E
:108DC000001D08F0C4F950B91948006890F82C103B
:108DD0000120884017490968814316480160681CD2
:108DE00038B936B112480168091D134808F0FAF97C
:108DF0001AE07C190E4800684460BC4207D20C4857
:108E00000168091D0D48006808F0D2F90CE0084817
:108E10000168091D0A48006808F0CAF90948006895
:108E2000844201D207480460BDE8F0817000002050
:108E30005C00002074000020C85300206400002063
:108E4000600000208C00002010B5044608F0D6F920
:108E500023480068401C224908602248006840B945
:108E6000204804600846006801280DD100F0BEF9D2
:108E70000AE01D48006838B91A480068C06AE16A0B
:108E8000884201D81748046018480068401C1749F8
:108E9000086094F82C10012088401549096808439F
:108EA00013490860E16A01EB8101124A02EB81007B
:108EB000211D08F097F908F0CBF90B48006868B15C
:108EC00008480068C06AE16A884207D24FF08050C3
:108ED00009490860BFF34F8FBFF36F8F10BD0000CB
:108EE0006C0000205C00002078000020880000203A
:108EF00074000020F850002004ED00E010B516E0EA
:108F000008F07CF90C48C068C468201D08F01FF9FF
:108F10000A480068401E0949086009480068401E68
:108F20000749086008F094F9204600F05FF804480B
:108F300000680028E4D110BDB45300206C0000206C
:108F40006800002070B504460D46206C70B1216C9D
:108F5000E0680144E160D4E90210884201D321684D
:108F6000E1602846226CE168F7F7D0F970BD2DE981
:108F7000F04104460F4615464FF00008A66B206CE2
:108F800048B9206800282CD1A06809F0ABFA8046C7
:108F90000020A06025E07DB93946226C6068F7F7B3
:108FA000B5F9216C606808446060D4E90101884229
:108FB00017D32068606014E03946226CE068F7F748
:108FC000A5F9216CE068411AE1602168E0688842F7
:108FD00003D2216CA068411AE160022D01D106B1D3
:108FE000761E701CA0634046BDE8F08110B50446B3
:108FF00094F8590030B9206B08F048F9204608F081
:1090000045F91AE094F85900012803D1204608F0E8
:109010003DF912E094F85900022801D1012000E046
:10902000002050B900BF502080F31188BFF34F8F4C
:10903000BFF36F8F00BF00BFFEE710BD01464A6A55
:1090400022B10A6B1268C2F1200000E000207047D4
:1090500030B54FF47053174800F007042CB1C01D11
:1090600020F00700134C041B1B1B0246124C22600D
:109070000024114D6C60D018083820F007000F4C08
:10908000206000240D4D2D686C600C4D2D682C6007
:109090001146441A4C60094C24680C60084D4C6819
:1090A0002C60084D4C682C604FF00044064D2C603D
:1090B00030BD0000DC53002098000020A0000020FC
:1090C000A8000020A4000020B400002000BFFFF78B
:1090D00015FF064800680128F9D94FF0805004496F
:1090E0000860BFF34F8FBFF36F8FF0E7F850002099
:1090F00004ED00E010B5044654B10020A0602060EB
:109100000021E16000231A461946204608F098FC29
:1091100010BD2DE9F04106460D4617469846069CBF
:109120000DB9246000E02760E66325640121204634
:1091300008F03AFCBDE8F0812DE9FF5F81460E465C
:109140009246DDE90E7B109CAAF10100216B01EB38
:10915000800828F0070808F0070008B9012000E09F
:10916000002050B900BF502080F31188BFF34F8F0B
:10917000BFF36F8F00BF00BFFEE786B1002507E099
:10918000715D04F134004155705D00B902E06D1C61
:10919000182DF5D300BF00214B20015502E000201F
:1091A00084F83400202F00D31F27E762E7640020F3
:1091B0002065201D07F0F9FF04F1180007F0F5FF06
:1091C0002461C7F12000A06164620020606584F81A
:1091D000580049464046039A00F0C4F92060BBF1AC
:1091E000000F01D0CBF80040BDE8FF9F10B5002470
:1091F00007E004EB84010F4A02EB810007F0C8FF8F
:10920000641C202CF5D30C4807F0C2FF0B4807F074
:10921000BFFF0B4807F0BCFF0A4807F0B9FF0A4838
:1092200007F0B6FF04480949086004480849086087
:1092300010BD0000F8500020785300208C5300200F
:10924000A0530020B4530020C85300206000002029
:109250006400002010B50146164800E0006803686D
:109260008B42FBD30246436813448B4204D14368CC
:109270004C682344436001460A464B681344046823
:10928000A34211D10C4C03682468A34208D04B6858
:109290000468646823444B6003681B680B6005E046
:1092A000054B1B680B6001E003680B60884200D02F
:1092B000016010BD98000020A000002070B5054698
:1092C00007F09CFFA86B08B9012400E0002407F018
:1092D000BFFF204670BD70B5054607F08FFFA86B35
:1092E000E96B884201D1012400E0002407F0B0FFBF
:1092F000204670BD0A490968096809B9012100E0E2
:10930000002121B14FF0FF31064A116006E0044907
:109310000968C968C868034A41681160704700005D
:10932000600000208C0000200E480068401C08B936
:10933000012000E0002050B900BF502080F31188C8
:10934000BFF34F8FBFF36F8F00BF00BFFEE700BFBB
:10935000502080F31188BFF34F8FBFF36F8F00BF92
:1093600000BFFEE7B800002070B5044607F046FFD6
:1093700094F9455010E0606A08B9012000E000202F
:1093800038B904F1240009F06DF918B108F05AF861
:1093900000E003E0681E45B2002DECDC00BFFF20BA
:1093A00084F8450007F054FF07F028FF94F9445073
:1093B00010E0206908B9012000E0002048B904F15C
:1093C000100009F04FF908B108F03CF8681E45B2EA
:1093D00000E001E0002DECDC00BFFF2084F8440039
:1093E00007F036FF70BD00000146024800680844DF
:1093F00070470000D40000202DE9F04104464FF0F2
:10940000000808F00BF94948006808B9FFF720FE8A
:10941000474800682040002870D1D4B1083404F0D7
:109420000700B0B104F00700C0F10800044404F0E4
:10943000070008B9012000E0002050B900BF50200B
:1094400080F31188BFF34F8FBFF36F8F00BF00BF52
:10945000FEE7002C52D03748006884424ED8364E82
:109460003046056801E02E462D686868A04202D2A9
:1094700028680028F7D12D48006885423ED0306822
:1094800000F10808286830606868001B102819D9A6
:109490002F1907F0070008B9012000E0002050B99B
:1094A00000BF502080F31188BFF34F8FBFF36F8F41
:1094B00000BF00BFFEE76868001B78606C6038463C
:1094C000FFF7C8FE1B4968680968081A194908604F
:1094D0000846006819490968884203D2154800689F
:1094E00016490860124968680968084368600020E6
:1094F000286013480068401C1149086009F0FEF814
:1095000008F0070008B9012000E0002050B900BFB2
:10951000502080F31188BFF34F8FBFF36F8F00BFD0
:1095200000BFFEE74046BDE8F0810000A00000203B
:10953000B4000020A400002098000020A800002013
:10954000AC0000200648006830B10549096801F107
:109550005000096D491C0160014800687047000017
:109560005C000020001F4FF080730360001F21F09B
:1095700001030360001F054B036014380260001FE5
:109580006FF0020303602038704700002993000841
:1095900088B000BF0024172520216846F6F7DDFEBD
:1095A000AA208DF8000000208DF801008DF802003F
:1095B00004208DF8030010208DF8040000BF17E090
:1095C0002046FBF749F81E4908551E48005D095D15
:1095D000884206D01A48005D1A49085501201A49E8
:1095E00008701748015D601D0DF80010601CC4B2C2
:1095F000102CE5DB14480078E8B114480078012805
:1096000019D1E81E81B20DF1010009F0F9F88DF8C9
:1096100015003C208DF816002946684607F06CFDC1
:1096200009480078401C084908700846007803285B
:1096300001DD00200870642007F0CAFEAAE70000E0
:10964000B0010020A0010020010000200000002047
:1096500000BF04210348F8F77DF84FF4FA7007F0D3
:10966000B7FEF6E70004024008B5F9F7EBF900F0A1
:10967000BDFF00BF002000901248007801281DD1D6
:109680006B46012200211048F7F702FD0098C0F355
:10969000800068B90D48FDF7B9FF0C48FDF73EFFA3
:1096A0000B48006800F06AFB00200649087005E0DE
:1096B0000648FEF71BF80548FEF78CF8012007F076
:1096C00087FED7E700000020B84F0020C0500020E0
:1096D0008C010020F0B587B004460D461646FEF713
:1096E000F8F80746AEB1324601A82168FEF710F936
:1096F00001A807C804AB07C30498102806D1059831
:109700002860FEF7E6F8C01B07B0F0BD4FF0FF3051
:10971000FAE74FF0FF3201A82168FEF7F9F801A837
:1097200007C804AB07C305982860FEF7D2F8C01B32
:10973000EAE7000010B54FF0FF3103480068FEF77C
:109740009BF9012010BD00008801002010B50446DF
:1097500002480068FEF768F910BD0000880100208B
:109760002DE9F04100F07EF8074600BF0F4804687D
:109770000CB9BDE8F0816068381AB0F1004F01D330
:10978000012000E0002000B1F3E7084920680860EC
:10979000A568E66806496068086021460920FDF76B
:1097A000BDF90DB13046A847E0E700006C0100208C
:1097B0007001002010B50348FEF728F9024908603F
:1097C00010BD00000C2A0108880100207FB5044666
:1097D0000D46094B0FCB8DE80F0000950021684620
:1097E000FEF781F82060206818B94FF0FF3004B010
:1097F00070BD0020FBE70000142A010870B5054683
:109800000E46002231462868FEF7D0F808B9002439
:1098100001E04FF0FF34204670BD0146086808B9EA
:10982000002070470120FCE710B504464FF0FF31DF
:109830002068FEF721F910BD1CB5044600200090F9
:1098400001906846FEF7E2F82060206810B94FF0FA
:10985000FF301CBD0020FCE710B504462068FEF771
:10986000E3F810BD10B5F7F785FF10BD2DE9F04105
:1098700088B004460D4616461F46DDF838801C2188
:1098800001A8F6F76AFD019402950FFA88F0ADF889
:109890000C000597314601A8FEF77EF908B0BDE837
:1098A000F08100002DE9F04104460E46174600BF46
:1098B000B4F1804F08D300BF09A340F2291215A1CB
:1098C00022A0F9F799FB00BF00BFFFF7CBFF0519F6
:1098D0003A463146284600F04DF8BDE8F0810000D8
:1098E0002E2E2F4D6964646C6577617265732F54F9
:1098F000686972645F50617274792F4C7749502F98
:109900007372632F636F72652F74696D656F757401
:10991000732E630054696D656F75742074696D658D
:1099200020746F6F206C6F6E672C206D61782069DA
:1099300073204C5749505F55494E5433325F4D4167
:10994000582F34206D736563730000004173736595
:109950007274696F6E2022257322206661696C65BE
:1099600064206174206C696E6520256420696E2016
:1099700025730A002DE9F04106460F46904609205E
:10998000FDF79AF90446002C0CD100BF07D100BFA7
:1099900020A3BE222CA13CA0F9F72EFB00BF00BFE4
:1099A000BDE8F08100202060A760C4F80C806660EC
:1099B0003F48006810B93E480460F1E73C496068E0
:1099C00009684968401AB0F1004F01D3012000E056
:1099D000002028B13648006820603548046017E050
:1099E0003348056811E0286850B160682968496803
:1099F000401AB0F1004F01D3012000E0002018B15F
:109A0000286820602C6002E02D68002DEBD100BF9B
:109A100000BFC5E72E2E2F4D6964646C65776172B7
:109A200065732F54686972645F50617274792F4C4A
:109A30007749502F7372632F636F72652F74696D4E
:109A4000656F7574732E63007379735F74696D65E8
:109A50006F75743A2074696D656F757420213D20AF
:109A60004E554C4C2C20706F6F6C204D454D505F07
:109A70005359535F54494D454F55542069732065E0
:109A80006D70747900000000417373657274696FC2
:109A90006E2022257322206661696C6564206174E2
:109AA000206C696E6520256420696E2025730A008C
:109AB0006C01002010B5012408E0064901EBC40246
:109AC00051F834000449FFF7EDFE641C032CF4D375
:109AD00010BD0000E82901086161000870B5154853
:109AE000006810B94FF0FF3070BDFFF7BBFE0446B1
:109AF000104800684068001BB0F1004F01D30120FE
:109B000000E0002008B10020EEE70A480068406845
:109B1000051B00BFB5F1004F08D300BF06A34FF4EB
:109B2000DC7212A116A0F9F767FA00BF00BF284641
:109B3000DAE700006C0100202E2E2F4D6964646C62
:109B40006577617265732F54686972645F506172E2
:109B500074792F4C7749502F7372632F636F72653E
:109B60002F74696D656F7574732E6300696E76610D
:109B70006C696420736C65657074696D65000000C4
:109B8000417373657274696F6E202225732220669B
:109B900061696C6564206174206C696E6520256460
:109BA00020696E2025730A002DE9FF5F04460E46EA
:109BB00000BF002C0AD100BF42A340F23D224DA1BC
:109BC00053A0F9F719FA00BFBDE8FF9F00BF00BF1F
:109BD000207D012808D100BF3AA34FF4107256A18E
:109BE0004BA0F9F709FA00BF00BF207D0A2807D172
:109BF00021465E4803F078F9204600F029FF5FE037
:109C00004FF0000AD346276DD4F82480D4F8905042
:109C1000D4F81090207DE8B9E08A38B300BF5448EA
:109C20000068A04205D152480068C06850490860E9
:109C30000DE04F49086806E0C168A14202D1E16821
:109C4000C16002E0C0680028F6D100BF00BF00205C
:109C5000E0600BE0B246B4F816B000BF21464548BC
:109C600003F042F901204449087000BF206F10B191
:109C7000206F05F08EF9E06E10B1E06E05F089F905
:109C8000606F10B1606F05F084F9BAF1000F0AD06F
:109C9000208B211D23464246CDE9001B0290394608
:109CA000204605F07BF8207D0390204600F0D0FE92
:109CB00000BF1DB16FF00C014846A84700BF00BFB0
:109CC00000BF81E72E2E2F4D6964646C6577617249
:109CD00065732F54686972645F50617274792F4C98
:109CE0007749502F7372632F636F72652F7463709F
:109CF0002E6300007463705F6162616E646F6E3A20
:109D000020696E76616C69642070636200000000F7
:109D1000417373657274696F6E2022257322206609
:109D200061696C6564206174206C696E65202564CE
:109D300020696E2025730A00646F6E2774206361AA
:109D40006C6C207463705F61626F72742F746370E7
:109D50005F6162616E646F6E20666F72206C697302
:109D600074656E2D7063627300000000380100207E
:109D70002C010020340100203C01002010B50446D5
:109D800001212046FFF710FF10BD28B1027D012AF6
:109D900002D10246916100BF7047000070B50546D0
:109DA0000C46164600BF002C08D100BF07A340F2A6
:109DB0000F3212A119A0F9F71FF900BF00BF20460A
:109DC000FFF7DCFF6FF00C0070BD00002E2E2F4D52
:109DD0006964646C6577617265732F546869726435
:109DE0005F50617274792F4C7749502F7372632FD3
:109DF000636F72652F7463702E6300007463705F0D
:109E00006163636570745F6E756C6C3A20696E7621
:109E1000616C6964207063620000000041737365C7
:109E20007274696F6E2022257322206661696C65E9
:109E300064206174206C696E6520256420696E2041
:109E400025730A0070B505460020FCF735FF04466F
:109E50001CBB00F071FF01F01FFD0020FCF72CFF80
:109E60000446CCB9092001F0AFFC0020FCF724FF28
:109E7000044684B9082001F0A7FC0020FCF71CFF71
:109E800004463CB9284601F06BFC0020FCF714FFA7
:109E9000044600BF00BF00BF00BF44B39C21204662
:109EA000F6F75BFA0C3465724FF48660A4F858003C
:109EB0004000E083A083FF2004F8010C4FF40670FB
:109EC000E0840620A0866086C01FA0840120A087B1
:109ED00008480068606108480078A0744FF4866004
:109EE000E0870648A0670648C4F888000C3C204676
:109EF00070BD0000280100203E01002061E600083E
:109F000000DD6D002DE9F04705460C4617464FF081
:109F1000040904B92E4C00BF002D0CD100BF2DA3A5
:109F200040F2A92237A13DA0F9F766F800BF6FF013
:109F30000F00BDE8F08700BF00BF287D00280BD0D0
:109F400000BF24A340F2AB223EA134A0F9F754F89D
:109F500000BF6FF00500ECE700BF37B901F09EFFCE
:109F600007460FBB6FF00100E3E74FF0000819E070
:109F70003E4850F82800066810E0F08AB8420CD13C
:109F800046B1306830B12CB1206818B13068216812
:109F9000884202D16FF00700CBE7F668002EECD1C3
:109FA00008F10108C845E3DB34B1206820B10CB9E1
:109FB000002000E020682860EF8200BF2C48006885
:109FC000E8602B48056005F003FE00BF0020B0E705
:109FD000042A01082E2E2F4D6964646C6577617226
:109FE00065732F54686972645F50617274792F4C85
:109FF0007749502F7372632F636F72652F7463708C
:10A000002E6300007463705F62696E643A20696E4B
:10A0100076616C696420706362000000417373654F
:10A020007274696F6E2022257322206661696C65E7
:10A0300064206174206C696E6520256420696E203F
:10A0400025730A007463705F62696E643A2063610D
:10A050006E206F6E6C792062696E6420696E207369
:10A060007461746520434C4F53454400D82901085E
:10A070002C01002010B5044600BF002C0BD100BFFE
:10A080000CA34FF4F47217A11CA0F8F7B5FF00BFA2
:10A090006FF00F0010BD00BF207D012805D000BF6C
:10A0A000608B40F01000608300BF0121204600F06B
:10A0B00039F8EFE72E2E2F4D6964646C6577617275
:10A0C00065732F54686972645F50617274792F4CA4
:10A0D0007749502F7372632F636F72652F746370AB
:10A0E0002E6300007463705F636C6F73653A206960
:10A0F0006E76616C69642070636200004173736501
:10A100007274696F6E2022257322206661696C6506
:10A1100064206174206C696E6520256420696E205E
:10A1200025730A003EB504460D4600BF002C08D139
:10A1300000BF55A34FF4AF725FA167A0F8F75CFFB3
:10A1400000BF00BF002D56D0207D042802D0207D06
:10A15000072850D1A06F18B9208DB0F5066F4AD0EE
:10A1600000BFA07E00F0100040B900BF46A34FF42E
:10A17000B27263A158A0F8F73FFF00BF00BF208B69
:10A18000E18A221DCDE90021029023462046626A21
:10A19000216D04F003FE204602F038FE00BF00BF30
:10A1A0005E480068A04205D15C480068C0685B4911
:10A1B00008600DE05949086806E0C168A14202D173
:10A1C000E168C16002E0C0680028F6D100BF00BFAE
:10A1D0000020E06000BF01205149087000BF5148D5
:10A1E0000068A04202D105F0C3FD02E0204600F065
:10A1F0002FFC00203EBD207D20B1012824D0022864
:10A200003AD12CE0E08AD8B100BF47480068A042AC
:10A2100005D145480068C068434908600DE04249DF
:10A22000086806E0C168A14202D1E168C16002E0AD
:10A23000C0680028F6D100BF00BF0020E06000BF6A
:10A24000204600F005FC1BE0204601F043FB2146C0
:10A25000364802F049FE204600F0F2FC10E000BF54
:10A2600021462E4802F040FE01202D49087000BF13
:10A27000204600F0EDFB03E0204600F059F8B9E776
:10A2800000BF0020B6E700002E2E2F4D6964646CDD
:10A290006577617265732F54686972645F5061728B
:10A2A00074792F4C7749502F7372632F636F7265E7
:10A2B0002F7463702E6300007463705F636C6F7340
:10A2C000655F73687574646F776E3A20696E766146
:10A2D0006C69642070636200417373657274696FA6
:10A2E0006E2022257322206661696C65642061748A
:10A2F000206C696E6520256420696E2025730A0034
:10A300007063622D3E666C61677320262054465F41
:10A310005258434C4F534544000000003401002084
:10A320003C010020680100202C01002030010020A9
:10A3300070B5054600BF45B900BF1EA34FF4CE72ED
:10A3400028A12BA0F8F758FE00BF00BF287D0328E6
:10A3500004D004280AD0072818D10FE0284604F0BA
:10A36000C5FE04460CB90520287511E0284604F006
:10A37000BDFE04460CB90520287509E0284604F006
:10A38000B5FE04460CB90920287501E0002070BD17
:10A3900000BF1CB9284601F0A3FE09E0601C38B9D3
:10A3A00000BF688B40F00800688300BF0020EEE724
:10A3B0002046ECE72E2E2F4D6964646C6577617240
:10A3C00065732F54686972645F50617274792F4CA1
:10A3D0007749502F7372632F636F72652F746370A8
:10A3E0002E63000070636220213D204E554C4C00CE
:10A3F000417373657274696F6E2022257322206623
:10A4000061696C6564206174206C696E65202564E7
:10A4100020696E2025730A002DE9F05F80460D4605
:10A4200091469A460A9F00BFB8F1000F07D100BFBE
:10A4300040A3A3224CA154A0F8F7DEFD00BF00BF4B
:10A4400000BF002D07D100BF3AA3A42258A14EA0FF
:10A45000F8F7D2FD00BF00BF07F0010008B10420EB
:10A4600000E0002007F0020109B1002100E0002116
:10A47000084407F0080109B1002100E00021084468
:10A4800007F0100109B1002100E000214618022068
:10A49000FCF712FC041E05D12846FEF7BFF8002089
:10A4A000BDE8F09FA77200202060656000BF28898A
:10A4B000B04207DA00BF1FA3B02246A132A0F8F7CE
:10A4C0009BFD00BF00BF2889801B208114212846E6
:10A4D000FDF791FB20B1204604F04EFD0020DFE7A0
:10A4E00060684068E060B8F81600FBF76EFEE1684F
:10A4F0000880B8F81800FBF768FEE168488050460D
:10A50000FBF756FEE1684860B346F11706EB917120
:10A510008910491D4FF6FF7202EA013141EA090034
:10A52000FBF753FEE16888810020E16848822046FD
:10A53000B6E700002E2E2F4D6964646C657761725A
:10A5400065732F54686972645F50617274792F4C1F
:10A550007749502F7372632F636F72652F74637026
:10A560005F6F75742E6300007463705F6372656162
:10A5700074655F7365676D656E743A20696E7661A8
:10A580006C69642070636200417373657274696FF3
:10A590006E2022257322206661696C6564206174D7
:10A5A000206C696E6520256420696E2025730A0081
:10A5B0007463705F6372656174655F7365676D6511
:10A5C0006E743A20696E76616C696420706275669B
:10A5D00000000000702D3E746F745F6C656E203E4D
:10A5E0003D206F70746C656E0000000010B5002493
:10A5F00001F04EFC044641F28B3207492046FFF73A
:10A6000081FCFF21204601F0C9FA04460349204697
:10A61000FFF7BBFB10BD0000042A0108E509010893
:10A620002DE9F04106460D46174600BF002F08D120
:10A6300000BF10A340F6C5021AA124A0F8F7DCFC65
:10A6400000BF00BF15B93046BDE8F0812C8D74B154
:10A650002820844202DD211A89B200E000218846C8
:10A66000464501DA314600E041460E4600BF30461D
:10A67000EAE700002E2E2F4D6964646C65776172E5
:10A6800065732F54686972645F50617274792F4CDE
:10A690007749502F7372632F636F72652F746370E5
:10A6A0002E6300007463705F6566665F73656E6439
:10A6B0005F6D73735F6E657469663A20696E76616B
:10A6C0006C6964206473745F697000004173736522
:10A6D0007274696F6E2022257322206661696C6531
:10A6E00064206174206C696E6520256420696E2089
:10A6F00025730A002DE9F84304460D460027B946A4
:10A7000000BF05F0030040B900BF60A340F2114252
:10A710006B496CA0F8F770FC00BF00BF00BF002CB5
:10A7200008D100BF59A340F2134270A165A0F8F709
:10A7300063FC00BF00BF05F0020000B1012707F075
:10A74000010008B1042000E0002007F0020109B177
:10A75000002100E00021084407F0080109B10021B0
:10A7600000E00021084407F0100109B1002100E0D9
:10A77000002100EB01094FF4207249463620FDF715
:10A78000B7FAB0F1000809D100BF608B40F080003B
:10A79000608300BF4FF0FF30BDE8F88300BFB8F81A
:10A7A0000A00484508DA00BF38A340F2394257A1F1
:10A7B00044A0F8F721FC00BF00BF00972A4641469D
:10A7C0002046E36DFFF728FE061E07D100BF608B11
:10A7D00040F08000608300BF701EDDE700BF307B6B
:10A7E00000F0030040B100BF28A340F2424256A14E
:10A7F00034A0F8F701FC00BF00BF00BF308940B1B2
:10A8000000BF22A340F2434255A12EA0F8F7F4FB6B
:10A8100000BF00BFE06E08B9E66607E0E06E00E04A
:10A82000006801680029FBD1066000BF0020A4F881
:10A83000680005F0020010B905F0010010B1E06DEC
:10A84000401CE06505F0010028B100BF608B40F0BE
:10A850002000608300BF7068FDF7CAFC34F8661FF3
:10A860000844208034F8660970B100BF206F50B9E9
:10A87000E06E40B900BF05A340F2654243A111A0BC
:10A88000F8F7BAFB00BF00BF002085E72E2E2F4D42
:10A890006964646C6577617265732F54686972646A
:10A8A0005F50617274792F4C7749502F7372632F08
:10A8B000636F72652F7463705F6F75742E63000031
:10A8C000182B0108417373657274696F6E2022251D
:10A8D0007322206661696C6564206174206C696E06
:10A8E0006520256420696E2025730A007463705FFB
:10A8F000656E71756575655F666C6167733A206931
:10A900006E76616C69642070636200007463705FCE
:10A91000656E71756575655F666C6167733A206316
:10A920006865636B20746861742066697273742053
:10A93000706275662063616E20686F6C64206F7052
:10A94000746C656E000000007365672D3E74637063
:10A95000686472206E6F7420616C69676E65640054
:10A960007463705F656E71756575655F666C616750
:10A97000733A20696E76616C6964207365676D65F2
:10A980006E74206C656E6774680000007463705F9D
:10A99000656E71756575655F666C6167733A206990
:10A9A0006E76616C6964207175657565206C656E85
:10A9B0006774680070B523480078401C214908700E
:10A9C00000BF2148046839E0A07F1E490978884209
:10A9D00033D01C480078A077A07E00F0010078B149
:10A9E00000BF608B40F00200608300BF204601F092
:10A9F00077FB00BF608B4FF6FC710840608300BF9F
:10AA0000A07E00F0080048B100BF608B4FF6F771E0
:10AA10000840608300BF2046FFF78AFCE568A06F0E
:10AA200048B1002009490870204602F0EBFE0748B3
:10AA3000007800B1C5E72C4600E0E468002CC3D1E3
:10AA400070BD00003E010020340100203C010020C8
:10AA500010B5044600BF207D012807D100BF06A322
:10AA6000D42211A115A0F8F7C7FA00BF00BF2146F4
:10AA70000020FCF753F810BD2E2E2F4D6964646C36
:10AA80006577617265732F54686972645F50617293
:10AA900074792F4C7749502F7372632F636F7265EF
:10AAA0002F7463702E6300007463705F6672656557
:10AAB0003A204C495354454E0000000041737365E1
:10AAC0007274696F6E2022257322206661696C653D
:10AAD00064206174206C696E6520256420696E2095
:10AAE00025730A002DE9F04705460C469146984625
:10AAF00035E0264624687068FDF77AFB074600BFFC
:10AB0000B5F86600B84208DA00BF22A340F2574207
:10AB10002DA137A0F8F770FA00BF00BF35F8660F17
:10AB2000C01B288030893C49098808443A4908807C
:10AB3000304604F021FA35F8660900280FD000BF2E
:10AB4000002C0BD1B8F1000F08D100BF11A340F2C7
:10AB5000614232A126A0F8F74FFA00BF00BFB4B19E
:10AB6000E1684868FBF724FB8246E1688889FBF7C7
:10AB70002CFB00F0030008B1012000E00020218937
:10AB8000084450442D490968401A0028B1DD204688
:10AB9000BDE8F0872E2E2F4D6964646C6577617275
:10ABA00065732F54686972645F50617274792F4CB9
:10ABB0007749502F7372632F636F72652F746370C0
:10ABC0005F696E2E630000007063622D3E736E64D9
:10ABD0005F71756575656C656E203E3D20706275B0
:10ABE000665F636C656E286E6578742D3E70290013
:10ABF000417373657274696F6E202225732220661B
:10AC000061696C6564206174206C696E65202564DF
:10AC100020696E2025730A005C0100207463705F58
:10AC2000726563656976653A2076616C6964207146
:10AC300075657565206C656E677468005801002045
:10AC400010B5044600BF207D012807D100BF06A330
:10AC5000DF2211A117A0F8F7CFF900BF00BF2146EE
:10AC60000120FBF75BFF10BD2E2E2F4D6964646C35
:10AC70006577617265732F54686972645F506172A1
:10AC800074792F4C7749502F7372632F636F7265FD
:10AC90002F7463702E6300007463705F6672656565
:10ACA0005F6C697374656E3A20214C495354454E6C
:10ACB00000000000417373657274696F6E20222575
:10ACC0007322206661696C6564206174206C696E12
:10ACD0006520256420696E2025730A0010B504469E
:10ACE000606F20B1606F04F054F90020606710BD00
:10ACF0000D4801880088401C0B4A10800B480068F2
:10AD000018B10B480088814205DA0A48006800F152
:10AD10001402505C704706480078081AC2B2034813
:10AD20000068805CF6E70000500100204C01002024
:10AD30004A0100204401002070B50B48046810E06F
:10AD4000E568A07E00F0080048B100BF608B4FF6B8
:10AD5000F7710840608300BF2046FFF7E9FA2C46F0
:10AD600000BF002CECD170BD3401002010B5F5F708
:10AD7000BBFAC0F30D0000F540400149088010BD4A
:10AD8000240100202DE9FE4F05468B4600BF002D13
:10AD900007D100BFE2A38322EEA1F4A0F8F72CF9BB
:10ADA00000BF00BFFB49686808606889142800DAA2
:10ADB000C8E3F94A11685069F9F737FF28B9F6482E
:10ADC000007D00F0F000E02800D1BBE3F149096804
:10ADD0008889FBF7FAF900138700142F02DB288912
:10ADE000B84200DAAEE3A7F11400EC490880002075
:10ADF000EB4908606889B84208DBE8480088E949FF
:10AE0000088039462846FDF76DFE4AE000BF2868F5
:10AE100038B900BFC2A3C222E3A1D4A0F8F7ECF86E
:10AE200000BF00BF14212846FDF75CFE6889DD499C
:10AE30000880DA4800880988401A1FFA80FAD94841
:10AE400001882846FDF74EFE28684089504500DA03
:10AE500078E328684068D249086051462868FDF7C1
:10AE600041FE2889A0EB0A00288100BF688938B11B
:10AE700000BFABA3DF22D0A1BCA0F8F7BDF800BF94
:10AE800000BF00BF288929680989884207D000BF10
:10AE9000A3A3E022CBA1B5A0F8F7AEF800BF00BF96
:10AEA00000BFBC4909680888FBF78FF9B9490968F0
:10AEB0000880B84909684888FBF787F9B5490968E7
:10AEC0004880B44909684868FBF772F9B1490968D4
:10AED0004860C4490860AF4909688868FBF768F9A9
:10AEE000AC4909688860C0490860AA490968C889EE
:10AEF000FBF76BF9A7490968C881A64909688889E1
:10AF0000FBF763F900F03F00B84908702889B84999
:10AF10000880B648007800F0030040B10846008879
:10AF2000401C088028890988884200DD0AE34FF028
:10AF30000009B048046873E000BF207D38B900BF45
:10AF400077A3FB22ACA189A0F8F756F800BF00BF99
:10AF500000BF207D0A2807D100BF71A3FC22B0A149
:10AF600082A0F8F749F800BF00BF00BF207D01288C
:10AF700007D100BF6AA3FD22B4A17CA0F8F73CF87A
:10AF800000BF00BF207A50B1217A8348406890F812
:10AF90003400401CC0B2814201D0A1463FE0208B6A
:10AFA0007C4909680988884237D1E08A794909686B
:10AFB0004988884231D178496068096988422CD132
:10AFC000754920684969884227D100BFE068A042DE
:10AFD00008D100BF52A340F20D12A6A163A0F8F75A
:10AFE0000BF800BF00BFB9F1000F07D0E068C9F847
:10AFF0000C0080480068E0607E48046000BFE068A4
:10B00000A04208D100BF46A340F21512A4A157A048
:10B01000F7F7F2FF00BF00BF04E0A14600BFE468FD
:10B02000002C89D100BF002C78D1A848046839E0F1
:10B0300000BF207D0A2808D000BF39A340F21F12AC
:10B04000A3A14AA0F7F7D8FF00BF00BF207A48B1FC
:10B05000217A5148406890F83400401CC0B28142C7
:10B0600000D01EE0208B4B4909680988884217D11F
:10B07000E08A484909684988884211D14649606890
:10B08000096988420CD1444920684969884207D13E
:10B09000204604F0B9FD2846FDF7C0FABDE8FE8F52
:10B0A00000BFE468002CC3D1A146954806681FE0A4
:10B0B000307A50B1317A3848406890F83400401CFA
:10B0C000C0B2814201D0B14611E0F08A314909682D
:10B0D0004988884209D1304930684969884200D19D
:10B0E00008E00EB1306800B904E0B14600BFF66870
:10B0F000002EDDD100BF8EB1B9F1000F07D0F0688E
:10B10000C9F80C007E480068F0607D480660304653
:10B1100000F04AFC2846FDF781FABFE7F2E00000A4
:10B120002E2E2F4D6964646C6577617265732F54A0
:10B13000686972645F50617274792F4C7749502F3F
:10B140007372632F636F72652F7463705F696E2E05
:10B15000630000007463705F696E7075743A2069F3
:10B160006E76616C69642070627566004173736508
:10B170007274696F6E2022257322206661696C6586
:10B1800064206174206C696E6520256420696E20DE
:10B1900025730A0044010020DC8F002048010020B4
:10B1A0004C0100204A010020702D3E6E657874200D
:10B1B000213D204E554C4C00702D3E6C656E203D5F
:10B1C0003D203000702D3E746F745F6C656E203DC5
:10B1D0003D20702D3E6E6578742D3E746F745F6CEB
:10B1E000656E00005401002058010020600100201D
:10B1F0005E010020340100207463705F696E707519
:10B20000743A20616374697665207063622D3E73C1
:10B210007461746520213D20434C4F534544000028
:10B220007463705F696E7075743A206163746976D7
:10B2300065207063622D3E737461746520213D202A
:10B2400054494D452D574149540000007463705FC7
:10B25000696E7075743A20616374697665207063F5
:10B26000622D3E737461746520213D204C49535416
:10B27000454E00007463705F696E7075743A20709B
:10B2800063622D3E6E65787420213D2070636220DC
:10B29000286265666F7265206361636865290000D6
:10B2A0007463705F696E7075743A207063622D3ECE
:10B2B0006E65787420213D20706362202861667479
:10B2C0006572206361636865290000003801002011
:10B2D0007463705F696E7075743A2054494D452DE2
:10B2E00057414954207063622D3E73746174652028
:10B2F0003D3D2054494D452D574149540000000023
:10B3000030010020002C73D000209149086028896A
:10B310000881084645608F480068C86000208E4953
:10B3200008608E4908708E4908808E48007800F0C9
:10B33000080018B1687B40F001006873A06F80B10D
:10B34000204602F05FFA0D3028B1A06F48B1864860
:10B350000088002805DD608D10B9204603F026FE28
:10B36000BCE082480460204601F0AAFE804608F155
:10B370000D00002816D07948007800F0080090B140
:10B3800000BFD4F8900028B16FF00D01D4F89020E0
:10B390002069904700BF2146754801F0A5FD204671
:10B3A000FFF756FB99E04FF000086D480088002831
:10B3B00019DD6B48B0F800A000BFD4F8800038B1A8
:10B3C00052462146D4F8803020699847804601E0F3
:10B3D0004FF0000800BF08F10D0000B97EE000202A
:10B3E0005F49088000BF204600F0D8F808B175E03A
:10B3F00084E059480068A8B300BFA06F50B100BFF7
:10B40000AFF2E4234FF4F3725AA1AFF2A020F7F7A2
:10B41000F3FD00BF00BFA07E00F0100038B14E4821
:10B420000068FDF7FBF82046FEF7A8FC56E000BFD9
:10B43000D4F8840048B100234749D4F884C0206977
:10B440000A682146E047804607E00023424821463B
:10B450000268184603F004F9804600BF08F10D00A9
:10B4600008B93BE005E0B8F1000F02D03A480068A7
:10B47000A0673A48007800F0200018B3A06F30B100
:10B48000A06F407B40F02000A16F48731AE0208D30
:10B49000B0F5066F02D0208D401C208500BFD4F887
:10B4A000840040B100231A462146D4F884C02069A4
:10B4B000E047804601E04FF0000800BF08F10D00B2
:10B4C00000B90BE0002029490860204600F066F82A
:10B4D00000B103E0204600F003FE00BF0020234936
:10B4E00008601D4908601A48406840B31849486818
:10B4F000FDF794F800201649486020E015490968D6
:10B500008889FAF762FE00F00400A8B911480068C3
:10B5100000881049096849881D4ACDE90021029038
:10B520001C480068104909884218194B1B1D1A480D
:10B530000168002003F032FC2846FDF76FF800BFD9
:10B5400000BFABE52846FDF769F800BFA6E500009F
:10B5500050C6002044010020640100206101002049
:10B560005C010020600100205E01002068010020D5
:10B57000340100207063622D3E72656675736564E8
:10B580005F64617461203D3D204E554C4C000000CD
:10B59000EC8F0020540100205801002010B5044613
:10B5A00000BF002C08D100BF13A340F25A221FA1F4
:10B5B00028A0F7F721FD00BF00BF3048007800F059
:10B5C0001000B8B1A07E00F0100050B900BFD4F850
:10B5D000900028B16FF00E01D4F8902020699047B8
:10B5E00000BF2146264801F07FFC2046FFF730FAD5
:10B5F000012010BD0020FCE72E2E2F4D6964646CE5
:10B600006577617265732F54686972645F50617207
:10B6100074792F4C7749502F7372632F636F726563
:10B620002F7463705F696E2E630000007463705F37
:10B63000696E7075745F64656C617965645F636C75
:10B640006F73653A20696E76616C6964207063621D
:10B6500000000000417373657274696F6E202225CB
:10B660007322206661696C6564206174206C696E68
:10B670006520256420696E2025730A006101002081
:10B68000340100202DE9F0410446002600BF002CC3
:10B6900008D100BF14A340F6240220A126A0F7F78A
:10B6A000ABFC00BF00BF216D481EFAF781FD80464C
:10B6B000434600223146204600F0C4FE05461DB92F
:10B6C0004FF0FF30BDE8F081334600222946204686
:10B6D00001F036F8231D22462946204600F0B2FF2D
:10B6E00007463846EEE700002E2E2F4D6964646C45
:10B6F0006577617265732F54686972645F50617217
:10B7000074792F4C7749502F7372632F636F726572
:10B710002F7463705F6F75742E6300007463705FC5
:10B720006B656570616C6976653A20696E76616CEF
:10B730006964207063620000417373657274696F9D
:10B740006E2022257322206661696C656420617415
:10B75000206C696E6520256420696E2025730A00BF
:10B760002DE9F04107467F2F01DD7F2000E03846BC
:10B7700006460EB9BDE8F081701EC6B24FF0000853
:10B7800000250F48046813E0607DB04208DB607D4F
:10B79000B0420CD10B49206A0968081A404506D30B
:10B7A0000849206A0968A1EB00082546667DE4681F
:10B7B000002CE9D115B12846FEF7E0FA00BFD9E721
:10B7C00034010020280100202DE9F041054600BF8A
:10B7D000082D0AD0092D08D000BF13A340F2DD6266
:10B7E0001DA121A0F7F708FC00BF00BF002700261D
:10B7F000274804680EE0207DA8420AD12549206A26
:10B800000968081AB84204D32249206A09680F1A45
:10B810002646E468002CEED11EB100213046FEF72A
:10B82000C3F9BDE8F08100002E2E2F4D6964646CD1
:10B830006577617265732F54686972645F506172D5
:10B8400074792F4C7749502F7372632F636F726531
:10B850002F7463702E630000696E76616C696420DA
:10B860007374617465000000417373657274696F6D
:10B870006E2022257322206661696C6564206174E4
:10B88000206C696E6520256420696E2025730A008E
:10B89000340100202801002070B5002600250B4847
:10B8A00004680BE00A49206A0968081AB04204D308
:10B8B0000749206A09680E1A2546E468002CF1D170
:10B8C00015B12846FEF75AFA70BD00003801002075
:10B8D0002801002070B5044600BF44B900BF12A380
:10B8E00040F211121CA11FA0F7F786FB00BF00BF9A
:10B8F00000BF207D012808D000BF0BA34FF4897240
:10B9000022A118A0F7F778FB00BF00BF012507E0D0
:10B91000244951F825100868214602F091FF6D1C5A
:10B92000042DF5D370BD00002E2E2F4D6964646C7C
:10B930006577617265732F54686972645F506172D4
:10B9400074792F4C7749502F7372632F636F726530
:10B950002F7463702E63000070636220213D204EBF
:10B96000554C4C00417373657274696F6E202225CB
:10B970007322206661696C6564206174206C696E55
:10B980006520256420696E2025730A007063622D8E
:10B990003E7374617465203D3D204C495354454EBF
:10B9A00000000000D82901082DE9FE43054654484F
:10B9B000007800F0040008B1BDE8FE8300BF002D50
:10B9C00008D100BF4FA340F281225BA162A0F7F72C
:10B9D00013FB00BF00BF4A48007800F01000B0B170
:10B9E000674800680088664909684988654ACDE962
:10B9F0000021029064480068644909884218614B3C
:10BA00001B1D63480168284603F0C8F975E03C48EF
:10BA1000007800F0020000286FD0687DFEF712FA6F
:10BA2000044674B900BFA86938B14FF0FF32002155
:10BA3000AB6928699847804601E06FF00F0800BFA6
:10BA4000BAE750481038406920604E481038006905
:10BA50006060E88AE0824A4800680088208303200A
:10BA6000207549480068401C6062606AE0622046B8
:10BA700000F048FA0646A66526656664E665424813
:10BA80000068401E606528692061E567687A00F0FB
:10BA90000C006072287A207200BF00BF3D48006829
:10BAA000E0603C48046004F093F800BF01203A498C
:10BAB000087000BF204601F055F831480068C08981
:10BAC00024F8600F20886080603C201DF9F782FD1B
:10BAD0008046608E221D4146FEF7A2FD608612213F
:10BAE0002046FEF707FE074627B100212046FEF755
:10BAF0005BF861E7204600F0F3FA00BF5CE7000066
:10BB0000600100202E2E2F4D6964646C6577617290
:10BB100065732F54686972645F50617274792F4C39
:10BB20007749502F7372632F636F72652F74637040
:10BB30005F696E2E630000007463705F6C697374DC
:10BB4000656E5F696E7075743A20696E76616C69B6
:10BB50006420706362000000417373657274696FE2
:10BB60006E2022257322206661696C6564206174F1
:10BB7000206C696E6520256420696E2025730A009B
:10BB800044010020EC8F0020540100205E010020C1
:10BB900058010020340100203C01002070B504460B
:10BBA0000D4600222946204600F002F870BD000034
:10BBB0002DE9F041044688461746002500BF002CB9
:10BBC0000BD100BF38A340F2593243A14EA0F7F782
:10BBD00013FA00BF6FF00F0660E000BF00BF207DCA
:10BBE00000280BD000BF30A340F25A3250A146A02B
:10BBF000F7F702FA00BF6FF00E064FE000BF207D9E
:10BC0000012803D125466FF0080647E00120FBF725
:10BC100053F8054615B94FF0FF363FE0206928611B
:10BC2000E08AE88201202875607D6875607A687214
:10BC300000202872E07AE872A07AA8722068286052
:10BC4000E08AD8B100BF48480068A04205D1464804
:10BC50000068C068444908600DE04349086806E090
:10BC6000C168A14202D1E168C16002E0C068002859
:10BC7000F6D100BF00BF0020E06000BF2046FEF705
:10BC8000E7FE3A48A86100BF39480068E8603848D4
:10BC9000056003F09DFF00BF002600BF07B13E70A6
:10BCA0002846BDE8F08100002E2E2F4D6964646C9B
:10BCB0006577617265732F54686972645F50617251
:10BCC00074792F4C7749502F7372632F636F7265AD
:10BCD0002F7463702E6300007463705F6C697374FB
:10BCE000656E5F776974685F6261636B6C6F675FD5
:10BCF000616E645F6572723A20696E76616C696428
:10BD00002070636200000000417373657274696F94
:10BD10006E2022257322206661696C65642061743F
:10BD2000206C696E6520256420696E2025730A00E9
:10BD30007463705F6C697374656E5F776974685F54
:10BD40006261636B6C6F675F616E645F6572723AAC
:10BD50002070636220616C726561647920636F6E2C
:10BD60006E656374656400002C0100209D9D0008D1
:10BD70003001002070B506460D46D6B13068C0B11E
:10BD80000C480168304600F01BF80B48016830464B
:10BD900000F016F86DB1286858B10848046806E04C
:10BDA00020683168884201D128682060E468002C4E
:10BDB000F6D170BD340100202C010020300100209C
:10BDC0002DE9F04105460E46344600BF002D08D14E
:10BDD00000BF0CA34FF4106216A123A0F7F70CF9D3
:10BDE00000BF00BF0AE020682968884205D1E768E3
:10BDF0002046FDF7C3FF3C4600E0E468002CF2D18A
:10BE0000BDE8F0812E2E2F4D6964646C65776172F8
:10BE100065732F54686972645F50617274792F4C36
:10BE20007749502F7372632F636F72652F7463703D
:10BE30002E6300007463705F6E657469665F69707D
:10BE40005F616464725F6368616E6765645F70639D
:10BE5000626C6973743A20696E76616C6964206FF4
:10BE60006C645F6164647200417373657274696FBE
:10BE70006E2022257322206661696C6564206174DE
:10BE8000206C696E6520256420696E2025730A0088
:10BE900010B54020FDF7D6FF10BD000010B50023FF
:10BEA00000BF16480088401C144C208020460088A3
:10BEB0004FF6FF74A04203D14FF440400F4C208056
:10BEC000002116E00E4850F8210002680DE0D08AEB
:10BED0000A4C2488A04207D1581C83B2B3F5804F86
:10BEE00001DB002010BDDCE7D268002AEFD1481C3E
:10BEF000C1B20429E6DB01480088F3E724010020F1
:10BF0000D829010810B5044600BF002C08D100BF95
:10BF100009A340F6AF0214A11AA0F7F76DF800BF0D
:10BF200000BF224800682249096808441F49086088
:10BF30000846006810BD00002E2E2F4D6964646C09
:10BF40006577617265732F54686972645F506172BE
:10BF500074792F4C7749502F7372632F636F72651A
:10BF60002F7463702E6300007463705F6E65787465
:10BF70005F6973733A20696E76616C6964207063DF
:10BF800062000000417373657274696F6E20222530
:10BF90007322206661696C6564206174206C696E2F
:10BFA0006520256420696E2025730A004001002069
:10BFB0002801002070B505460C4600BF002D08D1B1
:10BFC00000BF25A340F21F4230A13AA0F7F714F8B2
:10BFD00000BF00BFE9688889FAF7F7F800F00100B0
:10BFE00020B1204602F0D5FF002433E013E0E168E1
:10BFF0008889FAF7EAF800F0010038B10120FAF771
:10C00000E4F8E96889890843E96888812646246854
:10C01000304602F0B1FF4CB1E06840682189084425
:10C0200029892E4A12681144081AE0D594B128894A
:10C030002A4909680844E1684968401A002809DD6E
:10C04000E068808825490988401A2881298968681C
:10C05000FCF740FC2C6070BD2E2E2F4D6964646C83
:10C060006577617265732F54686972645F5061729D
:10C0700074792F4C7749502F7372632F636F7265F9
:10C080002F7463705F696E2E630000007463705FCD
:10C090006F6F735F696E736572745F7365676D65EB
:10C0A0006E743A20696E76616C69642063736567AB
:10C0B00000000000417373657274696F6E20222561
:10C0C0007322206661696C6564206174206C696EFE
:10C0D0006520256420696E2025730A005401002024
:10C0E0002DE9F84F044600BF002C08D100BFA7A3DC
:10C0F00040F2E142B2A1B8A0F6F77EFF00BF00BF58
:10C1000000BF207D012808D100BFA0A340F2E34278
:10C11000BBA1B1A0F6F770FF00BF00BFC248006826
:10C12000A04202D10020BDE8F88FB4F86000B4F856
:10C130004810884202DAB4F8600001E0B4F8480020
:10C140008146E56E45B9A07E00F0020018B1204698
:10C1500002F02CFFE7E710E1221D2146204602F005
:10C160000DFE074617B96FF00300DCE70CB120683D
:10C1700058B90FB1381D00E00020014611B96FF029
:10C180000300D0E70868206000BFE9684868FAF754
:10C190000FF8616C401A29890844484519D9B4F848
:10C1A000600048450CD1206F50B994F8990038B917
:10C1B000002004F8980F012060700020A070983CC7
:10C1C000A07E00F0020018B1204602F0EFFEAAE7C0
:10C1D000D3E0002084F89900266F26B100E036688D
:10C1E00030680028FBD1B5E000BFE9688889F9F71D
:10C1F000ECFF00F0040040B100BF64A340F23652EF
:10C200008AA175A0F6F7F8FE00BF00BF206FA0B1AD
:10C21000A07E00F0440080B9E06E38B1E06E0068A6
:10C2200058B9E06E0089618E884206DAB4F864007D
:10C2300018B1B4F86600092801DB012000E00020F5
:10C2400020B9A07E00F0A00000B98FE0207D022878
:10C2500007D01020F9F7B9FFE96889890843E96830
:10C2600088813A462146284600F0FCFA0090009862
:10C2700038B100BF608B40F08000608300BF009841
:10C2800051E72868E066207D022806D000BF608B59
:10C290004FF6FC710840608300BFE9684868F9F711
:10C2A00087FF8046E9688889F9F78FFF00F003006F
:10C2B00008B1012000E000202989084408EB000AA9
:10C2C000206DB0EB0A0001D5C4F850A0E968888958
:10C2D000F9F77BFF00F0030008B1012000E0002027
:10C2E0002989084488B300202860206F10B9256789
:10C2F0002E462EE0E9684868F9F75AFF8046F16853
:10C300004868F9F755FFB8EB00001BD504F1700839
:10C3100001E0D8F80080D8F8000068B1D8F8001023
:10C32000C9684868F9F744FF8346E9684868F9F73F
:10C330003FFFBBEB0000ECD4D8F800002860C8F841
:10C34000005006E03560366803E0FFE7284602F05B
:10C3500013FEE56E55B1E9684868F9F729FF616C8D
:10C36000401A2989084448457FF63EAF00BFE06E79
:10C3700010B90020A4F8680000BF00BF608B4FF622
:10C380007F710840608300BF0020CCE62E2E2F4D29
:10C390006964646C6577617265732F54686972644F
:10C3A0005F50617274792F4C7749502F7372632FED
:10C3B000636F72652F7463705F6F75742E63000016
:10C3C0007463705F6F75747075743A20696E76610E
:10C3D0006C69642070636200417373657274696F85
:10C3E0006E2022257322206661696C656420617469
:10C3F000206C696E6520256420696E2025730A0013
:10C40000646F6E27742063616C6C207463705F6F5F
:10C41000757470757420666F72206C697374656EC4
:10C420002D70636273000000680100205253542095
:10C430006E6F7420657870656374656420686572DA
:10C44000652100002DE9FF4104460E461746984637
:10C4500000BF002C08D100BF10A340F242721CA103
:10C4600025A0F6F7C9FD00BF00BF608D1023218B0A
:10C47000E28ACDE901130092039043463A463146E1
:10C48000606A00F04DF805461DB1618D606A084490
:10C49000E062284604B0BDE8F08100002E2E2F4D4A
:10C4A0006964646C6577617265732F54686972643E
:10C4B0005F50617274792F4C7749502F7372632FDC
:10C4C000636F72652F7463705F6F75742E63000005
:10C4D0007463705F6F75747075745F616C6C6F639B
:10C4E0005F6865616465723A20696E76616C696443
:10C4F0002070636200000000417373657274696F9D
:10C500006E2022257322206661696C656420617447
:10C51000206C696E6520256420696E2025730A00F1
:10C520002DE9F05F82460D4617469846DDF830B09B
:10C5300005F11400384481B24FF420722220FBF739
:10C54000D7FB0646002E34D000BF718905F11400D8
:10C55000814208DA00BF18A340F2237223A12FA062
:10C56000F6F74AFD00BF00BF74680A98F9F72DFE80
:10C5700020800B98F9F729FE6080C4F804805046AB
:10C58000F9F716FEA060A946E91705EB917189102D
:10C59000491D4FF6FF7202EA013141EA0B00F9F73B
:10C5A00014FEA0810D98F9F710FEE0810020208292
:10C5B00060823046BDE8F09F2E2E2F4D6964646C7A
:10C5C0006577617265732F54686972645F50617238
:10C5D00074792F4C7749502F7372632F636F726594
:10C5E0002F7463705F6F75742E63000063686563FA
:10C5F0006B20746861742066697273742070627550
:10C60000662063616E20686F6C642073747275635A
:10C6100074207463705F6864720000004173736516
:10C620007274696F6E2022257322206661696C65C1
:10C6300064206174206C696E6520256420696E2019
:10C6400025730A002DE9FE4F04460E4692469B468E
:10C6500000BF002E08D100BF17A340F2877223A1AC
:10C660002DA0F6F7C9FC00BF00BF5A465146204630
:10C6700002F084FB054615B96FF0030715E024B1FD
:10C6800094F80B8094F80A9003E04FF0FF084FF005
:10C690000009062043465A465146CDE900900295CE
:10C6A0003046F8F72FFD074600BF3046FBF7B6FFD0
:10C6B0003846BDE8FE8F00002E2E2F4D6964646C55
:10C6C0006577617265732F54686972645F50617237
:10C6D00074792F4C7749502F7372632F636F726593
:10C6E0002F7463705F6F75742E6300007463705FE6
:10C6F0006F75747075745F636F6E74726F6C5F7357
:10C7000065676D656E743A20696E76616C69642048
:10C710007062756600000000417373657274696F22
:10C720006E2022257322206661696C656420617425
:10C73000206C696E6520256420696E2025730A00CF
:10C740002DE9F04781460D4614469A464FF0000801
:10C7500000BF002D08D100BF1CA340F2567228A1D3
:10C7600031A0F6F749FC00BF00BF6E6806F1140760
:10C7700000BF384600EB880004F0010109B1042134
:10C7800000E00021084404F0020109B1002100E0AA
:10C790000021084404F0080109B1002100E0002153
:10C7A000084404F0100109B1002100E00021084410
:10C7B000B84208D000BF05A340F2757224A11AA0A8
:10C7C000F6F71AFC00BF00BFBDE8F0872E2E2F4DF4
:10C7D0006964646C6577617265732F54686972640B
:10C7E0005F50617274792F4C7749502F7372632FA9
:10C7F000636F72652F7463705F6F75742E630000D2
:10C800007463705F6F75747075745F66696C6C5F6C
:10C810006F7074696F6E733A20696E76616C6964CB
:10C820002070627566000000417373657274696FF1
:10C830006E2022257322206661696C656420617414
:10C84000206C696E6520256420696E2025730A00BE
:10C850006F7074696F6E73206E6F742066696C6C94
:10C86000656400002DE9FE4F04460D46164600BFE4
:10C87000002C08D100BF58A34FF4B76263A16BA08E
:10C88000F6F7BAFB00BF00BF00BF002D08D100BF04
:10C8900051A340F2B9526FA164A0F6F7ADFB00BFFF
:10C8A00000BF00BF002E08D100BF4BA340F2BA5218
:10C8B00070A15EA0F6F7A0FB00BF00BF204600F00D
:10C8C000F7F810B10020BDE8FE8F686AF9F770FC38
:10C8D000E1688860688DF9F778FCE168C881698D46
:10C8E000686A0844E862E06800F11407A07A00F082
:10C8F000010068B12A1D31464FF40670FDF790FE25
:10C9000082464AF00170F9F753FC38603F1D00BFC2
:10C91000B5F93000002801DA00202886686B38B9A4
:10C920005D4800686863E1684868F9F741FCA863FE
:10C93000A08961688988401A1FFA80F86068408978
:10C94000A0EB08006168488160680089A0EB0800DE
:10C95000616808816168E06848600020E1680882D9
:10C9600000BFE0681430A17A01F0010109B104218F
:10C9700000E000210844A17A01F0020109B1002180
:10C9800000E000210844A17A01F0080109B100216A
:10C9900000E000210844A17A01F0100109B1002152
:10C9A00000E000210844B84208D000BF0AA340F2CA
:10C9B0001C623AA11DA0F6F71FFB00BF00BF0621B5
:10C9C000A87A8DE84300EB7A2A1D29466068F8F7BB
:10C9D00099FB8146484676E72E2E2F4D6964646C9C
:10C9E0006577617265732F54686972645F50617214
:10C9F00074792F4C7749502F7372632F636F726570
:10CA00002F7463705F6F75742E6300007463705FC2
:10CA10006F75747075745F7365676D656E743A20B9
:10CA2000696E76616C696420736567004173736534
:10CA30007274696F6E2022257322206661696C65AD
:10CA400064206174206C696E6520256420696E2005
:10CA500025730A007463705F6F75747075745F730B
:10CA600065676D656E743A20696E76616C696420E5
:10CA7000706362007463705F6F75747075745F7358
:10CA800065676D656E743A20696E76616C696420C5
:10CA90006E65746966000000280100206F7074697B
:10CAA0006F6E73206E6F742066696C6C6564000035
:10CAB00010B5044600BF002C08D100BF08A340F207
:10CAC0009A5214A11DA0F6F797FA00BF00BF606844
:10CAD000807B012801D0012010BD0020FCE7000070
:10CAE0002E2E2F4D6964646C6577617265732F54C7
:10CAF000686972645F50617274792F4C7749502F66
:10CB00007372632F636F72652F7463705F6F7574D8
:10CB10002E6300007463705F6F75747075745F735B
:10CB200065676D656E745F627573793A20696E76BC
:10CB3000616C696420736567000000004173736570
:10CB40007274696F6E2022257322206661696C659C
:10CB500064206174206C696E6520256420696E20F4
:10CB600025730A002DE9F041054600BF002D08D1CC
:10CB700000BF28A340F27D7233A13AA0F6F73CFA39
:10CB800000BF00BF41480088002840D00020404935
:10CB9000088036E0FEF7ACF8074627B1012F04D035
:10CBA000022F1FD102E0BDE8F08128E0FEF7A0F8D7
:10CBB000042806D136480088801C344909888842F8
:10CBC00000DDF0E7FEF794F80602FEF791F8064361
:10CBD000B6F5067F00DC16B94FF4067000E030466B
:10CBE00068860CE0FEF784F80446022C00DADAE7E7
:10CBF000A01E2749098808442549088000BF00BFB6
:10CC000000BF23480088214909888842C2DB00BF51
:10CC1000C9E700002E2E2F4D6964646C6577617240
:10CC200065732F54686972645F50617274792F4C18
:10CC30007749502F7372632F636F72652F7463701F
:10CC40005F696E2E630000007463705F70617273C1
:10CC5000656F70743A20696E76616C6964207063E8
:10CC600062000000417373657274696F6E20222543
:10CC70007322206661696C6564206174206C696E42
:10CC80006520256420696E2025730A004801002074
:10CC9000500100202DE9F84F81460C461746984672
:10CCA000DDE90BAB0A9E009400BFB8F1000F07D17D
:10CCB00000BF29A3E82235A13DA0F6F79DF900BFEA
:10CCC00000BF00BF002E07D100BF23A3E92242A16D
:10CCD00037A0F6F791F900BF00BFBC421BDA0AF09B
:10CCE000020050B9B07E00F04000A0B9BBF1000FC7
:10CCF00003D0F06E08B9306F68B104F21B2020F049
:10CD00000300B84201D9384603E004F21B2020F0AA
:10CD1000030080B200904FF4207248460099FAF761
:10CD2000E7FF054615B90020BDE8F88F00BF286869
:10CD300040B100BF08A340F20B122FA11CA0F6F7D0
:10CD40005BF900BF00BF6889001BA8F800002C81B8
:10CD50006C812846E8E700002E2E2F4D6964646C34
:10CD60006577617265732F54686972645F50617290
:10CD700074792F4C7749502F7372632F636F7265EC
:10CD80002F7463705F6F75742E6300007463705F3F
:10CD9000706275665F707265616C6C6F633A206972
:10CDA0006E76616C6964206F76657273697A65006E
:10CDB000417373657274696F6E2022257322206639
:10CDC00061696C6564206174206C696E65202564FE
:10CDD00020696E2025730A007463705F7062756647
:10CDE0005F707265616C6C6F633A20696E76616C1E
:10CDF00069642070636200006E65656420756E630F
:10CE00006861696E656420706275660010B50446DD
:10CE100000BF002C09D100BF16A340F6510221A18A
:10CE200027A0F6F7E9F800BF10BD00BF207DF8B1DC
:10CE3000207D0A281CD0207D012819D0A06F20B1A8
:10CE4000A06FFBF7EBFB0020A067606F10B12046DE
:10CE5000FDF744FF4FF0FF302086E06E02F099F8B6
:10CE6000206F02F096F80020E0662067A4F86800C2
:10CE700000BFD9E72E2E2F4D6964646C657761720F
:10CE800065732F54686972645F50617274792F4CB6
:10CE90007749502F7372632F636F72652F746370BD
:10CEA0002E6300007463705F7063625F70757267F9
:10CEB000653A20696E76616C696420706362000077
:10CEC000417373657274696F6E2022257322206628
:10CED00061696C6564206174206C696E65202564ED
:10CEE00020696E2025730A0070B505460C4600BF08
:10CEF000002C08D100BF3AA340F6830244A14BA006
:10CF0000F6F77AF800BF00BF00BF002D08D100BFC0
:10CF100033A340F684024FA144A0F6F76DF800BF9A
:10CF200000BF00BF2868A04203D12868C0682860FD
:10CF30000CE0286806E0C168A14202D1E168C16046
:10CF400002E0C0680028F6D100BF00BF0020E0600A
:10CF500000BF2046FFF75AFF207D0A280FD0207D12
:10CF600001280CD0A07E00F0010040B100BF608B12
:10CF700040F00200608300BF2046FFF7B1F8207D3B
:10CF8000012826D000BFE06E40B100BF14A340F6D8
:10CF9000930238A125A0F6F72FF800BF00BF00BF0D
:10CFA000206F40B100BF0EA340F6940237A11FA02E
:10CFB000F6F722F800BF00BF00BF606F40B100BFAE
:10CFC00007A340F6960238A118A0F6F715F800BF9F
:10CFD00000BF00202075E08200BF00BF70BD0000D0
:10CFE0002E2E2F4D6964646C6577617265732F54C2
:10CFF000686972645F50617274792F4C7749502F61
:10D000007372632F636F72652F7463702E630000F9
:10D010007463705F7063625F72656D6F76653A20EE
:10D02000696E76616C696420706362004173736538
:10D030007274696F6E2022257322206661696C65A7
:10D0400064206174206C696E6520256420696E20FF
:10D0500025730A007463705F7063625F72656D6F41
:10D0600076653A20696E76616C6964207063626CE3
:10D0700069737400756E73656E74207365676D6592
:10D080006E7473206C65616B696E6700756E6163A9
:10D090006B6564207365676D656E7473206C656184
:10D0A0006B696E67000000006F6F736571207365B8
:10D0B000676D656E7473206C65616B696E670000E7
:10D0C0002DE9FE4304460027002600BF002C08D1AE
:10D0D00000BFE5A34FF44772F0A1F7A0F5F78CFF6E
:10D0E00000BF00BFFE48007800F00400002845D0D3
:10D0F000207D022806D1FB49206D096888421BD19A
:10D10000012719E0F849606A0968884201D10127BE
:10D1100012E0F549606A0968081A0DD4218D606A29
:10D120000844F1490968081A002805DC00BF608B33
:10D1300040F00200608300BF002F1DD000BF207DA3
:10D1400040B900BFC8A34FF44E72E8A1DAA0F5F7CA
:10D1500053FF00BF00BFED48007840F00800EB49E6
:10D16000087000BF608B4FF6FE710840608300BFFF
:10D170006FF00D00BDE8FE830020FBE7D848007883
:10D1800000F0020068B1207D02280AD0207D03282B
:10D1900007D000BF608B40F00200608300BF00201A
:10D1A000E8E7A07E00F0100010B9D94800682062BE
:10D1B000002084F89B0084F89A002046FFF7D2FCF8
:10D1C000207D801E082875D2DFE800F004CDF4F33E
:10D1D000F2F1F0EFC248007800F0100000286AD0A9
:10D1E000BF48007800F002000028F8D0606C401CB6
:10D1F000BC49096888425ED1BB480068401C606237
:10D20000606AE062B74800686064C2480068C0892C
:10D21000A4F86000B4F86000A4F86200B2480068A6
:10D22000401E606504202075201DF8F7D3F9804664
:10D23000608E221D4146FDF7F3F96086608E810005
:10D24000400041F21C12904202D9608E400001E081
:10D2500041F21C10814202D2608E80000AE0608E92
:10D26000400041F21C11884202D9608E400001E06A
:10D2700041F21C10A4F8480000BFB4F86600002872
:10D2800008DC00BF78A34FF45B72A3A18AA0F5F776
:10D29000B3FE00BF00BFB4F86600401EA4F86600ED
:10D2A000256F95B9E56E00BF5DB900BF6EA34FF461
:10D2B0005D7201E08DE231E09DA17FA0F5F79CFE5B
:10D2C00000BF00BF2868E06601E0286820672846A4
:10D2D00001F052FE206F18B94FF0FF30208603E0B6
:10D2E0000020208684F8420000BFD4F8880038B1BE
:10D2F00000222146D4F8883020699847064600E08D
:10D30000002600BF06F10D0010B96FF00C0031E7E8
:10D3100000BF608B40F00200608323E0704800781B
:10D3200000F01000F0B17B48006800887949096876
:10D330004988844ACDE9002102906B4800688249FF
:10D34000098842187F4B1B1D66480168204601F082
:10D3500025FD94F84200062804DA002020862046A5
:10D3600001F0D0FB36E25E48007800F010000028A3
:10D3700076D0606C401C5B490968081A71D4594921
:10D38000206D0968081A00286BDC04202075E06F06
:10D3900010B96FF0050623E000BFE06F806978B92F
:10D3A00000BF31A34FF46A7205E0FCE1BCE107E184
:10D3B0007CE117E105E165A13FA0F5F71DFE00BF87
:10D3C00000BF00BFE06F806938B1E16F20690022C3
:10D3D0008B6921469847064601E06FF00F0600BFB3
:10D3E00046B106F10D0010B12046FCF7C7FC6FF006
:10D3F0000C00BFE6204600F09FFA5C48008820B190
:10D400005A480088401E59490880608E81004000BB
:10D4100041F21C12904202D9608E400001E041F2BC
:10D420001C10814202D2608E80000AE0608E4000B3
:10D4300041F21C11884202D9608E400001E041F2A5
:10D440001C10A4F848003148007800F0200048B1D2
:10D4500000BF608B40F00200608300BF072087E0C0
:10D460009FE087E0ABE000002E2E2F4D6964646CD6
:10D470006577617265732F54686972645F50617279
:10D4800074792F4C7749502F7372632F636F7265D5
:10D490002F7463705F696E2E630000007463705FA9
:10D4A00070726F636573733A20696E76616C69643C
:10D4B0002070636200000000417373657274696FCD
:10D4C0006E2022257322206661696C656420617478
:10D4D000206C696E6520256420696E2025730A0022
:10D4E0006001002058010020540100207463705F27
:10D4F000696E7075743A207063622D3E7374617446
:10D500006520213D20434C4F5345440061010020DC
:10D5100028010020440100207063622D3E736E6478
:10D520005F71756575656C656E203E20300000008A
:10D530006E6F207365676D656E7420746F20667200
:10D5400065650000EC8F00205E0100207063622D95
:10D550003E6C697374656E65722D3E6163636570C0
:10D560007420213D204E554C4C0000005C010020F1
:10D57000207524E099480068018898480068408830
:10D58000974ACDE90020029196480068964909889B
:10D590004218934B1B1D95480168204601F0FEFB85
:10D5A0000DE09348007800F0020040B1606A401E30
:10D5B0008C490968884202D1204601F09BF909E1B3
:10D5C00000BF204600F0B8F98A48007800F020003B
:10D5D00038B100BF608B40F00200608300BF0720BD
:10D5E0002075F7E0204600F0A7F98248007800F0A7
:10D5F0002000E8B37E48007800F01000C8B37B49F3
:10D60000206D0968884239D1E06E90BB00BF608B05
:10D6100040F00200608300BF2046FFF7F7FB00BF29
:10D6200000BF75480068A04205D173480068C06813
:10D63000714908600DE07049086806E0C168A142C0
:10D6400002D1E168C16002E0C0680028F6D100BFE5
:10D6500000BF0020E06000BF01206849087000BFE3
:10D660000A20207500BF66480068E060644801E059
:10D670000DE003E0046002F0ABFA16E000BF608B3F
:10D6800040F00200608300BF082020750DE058487C
:10D69000007800F0100040B15449206D09688842BC
:10D6A00003D1E06E08B90620207593E0204600F013
:10D6B00043F95048007800F02000A0B300BF608B11
:10D6C00040F00200608300BF2046FFF79FFB00BFD1
:10D6D00000BF49480068A04205D147480068C068BB
:10D6E000454908600DE04449086806E0C168A14268
:10D6F00002D1E168C16002E0C0680028F6D100BF35
:10D7000000BF0020E06000BF01203C49087000BF5E
:10D710000A20207500BF3A480068E060384804607D
:10D7200002F056FA00BF55E0204600F005F93048F7
:10D73000007800F01000A8B32C49206D09688842D9
:10D7400030D1E06E70BB2046FFF760FB00BF00BF2A
:10D7500029480068A04205D127480068C0682649CA
:10D7600008600DE02449086806E0C168A14202D1C2
:10D77000E168C16002E0C0680028F6D100BF00BFC8
:10D780000020E06000BF01201C49087000BF0A2093
:10D79000207500BF1A480068E0601948046002F074
:10D7A00017FA00BF16E0204600F0C6F810480078CF
:10D7B00000F0100060B10D49206D0968884207D162
:10D7C000E06E28B90B48007840F010000949087055
:10D7D00000E000BF00BF0020CCE4000044010020B6
:10D7E000EC8F0020540100205E0100205801002031
:10D7F0006001002061010020340100203C01002074
:10D80000380100202DE9F041044600BF002C0CD166
:10D8100000BF29A340F2096233A13DA0F5F7ECFB5C
:10D8200000BF6FF00F00BDE8F08100BFA06F477B25
:10D83000A66F0020A06700BFD4F8840040B1002389
:10D8400032462146D4F884C02069E047054606E008
:10D85000002332462146184600F002FF054600BF6D
:10D86000F5B907F0200028B3208DB0F5066F02D07F
:10D87000208D401C208500BFD4F8840040B10023D7
:10D880001A462146D4F884C02069E047054600E0E6
:10D89000002500BF05F10D0060B96FF00C00C2E774
:10D8A00005F10D0010B96FF00C00BCE7A6676FF032
:10D8B0000400B8E70020B6E72E2E2F4D6964646C93
:10D8C0006577617265732F54686972645F50617225
:10D8D00074792F4C7749502F7372632F636F726581
:10D8E0002F7463702E6300007463705F70726F63D7
:10D8F0006573735F726566757365645F6461746197
:10D900003A20696E76616C69642070636200000081
:10D91000417373657274696F6E20222573222066CD
:10D9200061696C6564206174206C696E6520256492
:10D9300020696E2025730A002DE9F05F04464FF040
:10D94000000900BF002C08D100BFE5A340F27B42D4
:10D95000F0A1F7A0F5F750FB00BF00BF00BF207D8E
:10D96000042808DA00BFDEA340F27C42FAA1F0A04E
:10D97000F5F742FB00BF00BFFE48007800F0100042
:10D98000002870D0B4F86000A16D00EB0108FA49DE
:10D99000606D0968401A15D4F749606D09688842BE
:10D9A00004D1F649A06D0968401A0BD4F349A06D63
:10D9B000096888421AD1F2480068C089B4F860103A
:10D9C000884213D9EE480068C08924F8600F608847
:10D9D00034F86019884203DAB4F86000A4F86200F1
:10D9E000E54800686065E5480068A065E349606C4B
:10D9F0000968081A00284ADCE248008890BBB4F89D
:10DA00006010A06D084440453AD1B4F930000028B8
:10DA100036DBDA49606C0968884231D14FF0010980
:10DA200094F84300401CC0B294F84310884204DDCF
:10DA300094F84300401C84F8430094F84300032802
:10DA400017DD00BFB4F84800618E084480B2B4F816
:10DA50004810884208DBB4F84800618E0844A4F8F6
:10DA6000480005E00CE02AE14FF6FF70A4F84800FA
:10DA700000BF94F84300032802DB204600F0BCFFFF
:10DA8000B9F1000F02D1002084F84300EBE0606C94
:10DA9000401CBA490968081A7ED4B849206D096843
:10DAA000081A002878DCA07E00F0040060B100BFF6
:10DAB000608B4FF6FB710840608300BF483460887C
:10DAC000208000206084483C00202434A077608BB4
:10DAD000B4F9181000EBE10000B2A083208CA74934
:10DAE0000988081A85B20020E077A44800682062FF
:10DAF00014F8100C243C042865DBB4F84800B4F892
:10DB00004A10884227DA628B02F400620AB10122CD
:10DB100000E002221146628E4A4392B2AA4201DD1F
:10DB20002A4602E0628E4A4392B2104600BFB4F821
:10DB30004820024492B2B4F848309A4205DBB4F867
:10DB400048200244A4F8482003E04FF6FF72A4F8EE
:10DB5000482000BF37E000BFB4F86A00284480B214
:10DB6000B4F86A10884205DBB4F86A002844A4F8C7
:10DB70006A0003E04FF6FF70A4F86A0000BFB4F833
:10DB80006A00B4F8481088421DDB4834608C218854
:10DB9000401A6084483C00E062E000BFB4F84800EE
:10DBA000618E084480B2B4F84810884206DBB4F8AD
:10DBB0004800618E0844A4F8480003E04FF6FF7067
:10DBC000A4F8480000BF70A22046D4E91B31FCF73E
:10DBD00089FF20676EA22046D4E91B13FCF782FF61
:10DBE000E066206F18B94FF0FF30208601E000207A
:10DBF000208600202077E06E10B90020A4F868008D
:10DC0000B4F86400644909880844A4F86400608B8F
:10DC100000F4006018B3206F88B9E06E40B1E16E87
:10DC2000C9684868F8F7C4FAE16C081A002816DCDD
:10DC300000BF608B4FF2FF71084060830FE0216FDF
:10DC4000C9684868F8F7B4FAE16C081A002806DCDD
:10DC500000BF608B4FF2FF710840608300BF02E09D
:10DC6000204601F0A3F9606B48B34449A06B0968F2
:10DC7000401A24D5A08E49490988081A07B2B4F978
:10DC80003C00A7EBE00007B2A08F384400B2A087A9
:10DC9000002F01DA784207B2B4F93E00A7EBA000EA
:10DCA00007B2E08F384400B2E087E08FB4F93C104F
:10DCB00000EBE10000B2A4F84000002060633148AE
:10DCC000008800286CDD207D072869DA2A48616A0F
:10DCD0000068401C081A7CD42748616A006860E02C
:10DCE0002E2E2F4D6964646C6577617265732F54B5
:10DCF000686972645F50617274792F4C7749502F54
:10DD00007372632F636F72652F7463705F696E2E19
:10DD1000630000007463705F726563656976653ADD
:10DD200020696E76616C6964207063620000000097
:10DD3000417373657274696F6E20222573222066A9
:10DD400061696C6564206174206C696E652025646E
:10DD500020696E2025730A007463705F72656365C5
:10DD60006976653A2077726F6E67207374617465A7
:10DD70000000000060010020540100205801002034
:10DD8000440100205E010020756E61636B656400D4
:10DD9000756E73656E7400005C0100202801002020
:10DDA000D4E3F74A12881044401E081A00285FDCAA
:10DDB000F4484668F449606A0968A0EB010A00BFAC
:10DDC000F048406860B900BFAFF2EC0340F29452F3
:10DDD00000E04DE0EDA1AFF2A800F5F70DF900BFAE
:10DDE00000BF00BF4FF6FF7082450AD300BFAFF2FD
:10DDF000101340F29552E9A1AFF2CC00F5F7FCF810
:10DE000000BF00BF1FFA8AF500BFDE4840680089E6
:10DE1000A8420ADA00BFAFF2381340F29752E3A1EA
:10DE2000AFF2F400F5F7E8F800BF00BFD54800896D
:10DE3000401BD4490881084640680089401B1FFAEE
:10DE400080FB07E07089281A85B2A6F808B0002088
:10DE5000708136687089A842F4DB29463046FAF7AB
:10DE600041FEC949606A0860C649C96848600AE05D
:10DE7000C549606A0968081A05D500BF608B40F083
:10DE80000200608300BFC049606A0968081A7DD437
:10DE9000218D606A0844401EBB490968081A0028A1
:10DEA00074DCB949606A0968884270D1B549C968AB
:10DEB0008889F8F78AF900F0030008B1012000E032
:10DEC0000020B04909890844AD490880208D09889F
:10DED000884256DAAB49C9688889F8F776F900F0C4
:10DEE000010098B1A749C9688889F8F76EF900F070
:10DEF0003E052846F8F769F9A249C96889894CF2B4
:10DF0000FF02114008439F49C9688881208D9D49BF
:10DF10000881C9688889F8F758F900F0020020B133
:10DF200098480089401E97490881964A118950688F
:10DF3000FAF7D0FC9349C9688889F8F746F900F0E8
:10DF4000030008B1012000E000208E49098908443F
:10DF50008B49088000BF218D606A08448A4909689E
:10DF6000874A1288114488420AD000BFAFF290233A
:10DF700040F2CB5291A1AFF24820F5F73DF800BF37
:10DF800000BF606F002816D07E4901E0DAE2D3E1DD
:10DF9000C9688889F8F719F900F0010060B107E055
:10DFA000656F606F00686067284600F0E5FF00BF9E
:10DFB000606F0028F4D187E0656F2EE0E9688889FA
:10DFC000F8F703F900F0010008B36E49C9688889C1
:10DFD000F8F7FBF800F00200C8B90120F8F7F5F8EF
:10DFE0006849C968898908436649C968888165495B
:10DFF000C9688889F8F7E9F800F0030008B1012042
:10E0000000E000205F49098908445D4908802E46E8
:10E010002D68304600F0B0FF00BF55B1E868406899
:10E020002989084458490968554A12881144081A30
:10E03000C4D5002D46D05448006851490988084489
:10E04000E9684968401A00283CDDE86880884E4944
:10E050000988401A4B490881C9688889F8F7B5F8DA
:10E0600000F0020020B147480089401E4549088160
:10E07000444A11895068FAF72DFC4249C9688889D9
:10E08000F8F7A3F800F0030008B1012000E0002039
:10E090003C49098908443A49088000BF3A48006869
:10E0A00009880844E968496888420AD000BFAFF28D
:10E0B000D03340F2FC524FA1AFF28C30F4F79CFF0A
:10E0C00000BF00BF656700BF2F4800682C49098862
:10E0D0000844606200BF208D2949098888420ADA15
:10E0E00000BFAFF2044340F2076251A1AFF2C0306B
:10E0F000F4F782FF00BF00BF208D21490988401A34
:10E100002085204601F03EFE1E4840680089002818
:10E1100006DD1C4840684E490860002019494860E7
:10E120001849C9688889F8F750F800F0010028B14B
:10E130004848007840F0200046490870DAE0656FF2
:10E14000606FC068406810490860E9688889F8F71E
:10E150003CF800F0030008B1012000E0002029890C
:10E160000844616A0844606200BFE9688889F8F77A
:10E170002CF800F0030008B101206EE06CE0000014
:10E180005E01002050C6002054010020696E7365B6
:10E19000672E7020213D204E554C4C00696E7361F6
:10E1A0006E65206F66667365742100007062756627
:10E1B00020746F6F2073686F727421007463705FD6
:10E1C000726563656976653A207365676D656E741F
:10E1D000206E6F74207472696D6D656420636F7258
:10E1E000726563746C7920746F207263765F776EEA
:10E1F000640A00007463705F726563656976653AEE
:10E20000207365676D656E74206E6F74207472691B
:10E210006D6D656420636F72726563746C792074D0
:10E220006F206F6F7365712071756575650A0000E9
:10E230007463705F726563656976653A20746370B4
:10E240006C656E203E207263765F776E640A000014
:10E250006401002061010020002029890844218DEB
:10E2600088420AD900BFAFF2885340F22B62C2A1A4
:10E27000AFF24450F4F7C0FE00BF00BFE9688889E0
:10E28000F7F7A3FF00F0030008B1012000E0002031
:10E2900029890844218D081A2085204601F072FD45
:10E2A0006868008900280DDDBD48006828B1BC48B9
:10E2B00069680068F9F7F4FE02E0B9496868086027
:10E2C00000206860E9688889F7F77FFF00F00100A7
:10E2D00050B1B448007840F02000B2490870207D69
:10E2E000042801D10720207528686067284600F0BF
:10E2F00043FE00BF606F30B1606FC0684068616A04
:10E3000088423FF41CAF00BFA07E00F0010060B166
:10E3100000BF608B4FF6FE710840608300BF00BFF6
:10E32000608B40F00200608305E000BF608B40F02E
:10E330000100608300BF1DE1606F20B99A4800F0C2
:10E34000C1FD6067FAE00026656FF2E0E8684068AA
:10E3500096490968884217D19348008929898842DB
:10E3600011DD914800F0AEFD8246BAF1000F09D0F0
:10E3700016B1C6F800A001E0C4F874A029465046C2
:10E38000FDF718FED8E0D7E0A6B9E86840688749ED
:10E390000968081A0DD5844800F094FD8246BAF148
:10E3A000000F05D0C4F874A029465046FDF702FEC0
:10E3B000C2E030E0F0684068401C7C490968081AF7
:10E3C00028D4E8684068401E78490968081A00287F
:10E3D00020DC754800F076FD8246BAF1000F18D0B7
:10E3E000F06840683189084470490968401A00287B
:10E3F00009DDF06880886D490988081A3081318903
:10E400007068FAF767FAC6F800A029465046FDF78B
:10E41000D1FD91E000BF2E46286800287DD1E86834
:10E42000406862490968081A002876DDE968888929
:10E43000F7F7CBFE00F0010000B17DE05A4800F094
:10E4400041FD28602868002871D0E8684068298963
:10E45000084456490968401A002809DDE8688088A0
:10E4600052490988081A288129896868FAF732FA16
:10E47000218D606A08444E4909884C4A126811444B
:10E48000081A002853DD2968C9688889F7F79DFEB6
:10E4900000F0010098B12968C9688889F7F795FEEE
:10E4A00000F03E0A5046F7F790FE2968C96889894E
:10E4B0004CF2FF02114008432968C9688881A08C8A
:10E4C000218D084439490988401A296808812A6839
:10E4D00011895068FAF7FEF92968C9688889F7F741
:10E4E00074FE00F0030008B1012000E0002029685C
:10E4F000098908442E49088000BF218D606A0144C3
:10E500002A4800682A4A1288104481420ED000BF6F
:10E51000AFF634034FF4DF6201E009E007E0AFF249
:10E520006431AFF2F470F4F767FD00BF00BF03E0A1
:10E530002D68002D7FF40AAF00BF00BF204600F019
:10E5400035FD17E0204600F031FD13E01749606A01
:10E550000968081A08D4218D606A0844401E1349CE
:10E560000968081A002805DD00BF608B40F0020032
:10E57000608300BFBDE8F09F7463705F7265636580
:10E580006976653A206F6F736571207463706C658E
:10E590006E203E207263765F776E640A0000000092
:10E5A000640100206101002050C6002054010020B9
:10E5B0005E01002070B504460D46002C0FD000BF50
:10E5C000207D012808D100BF05A340F2DF7210A111
:10E5D00019A0F4F711FD00BF00BFC4F8845070BD4E
:10E5E0002E2E2F4D6964646C6577617265732F54AC
:10E5F000686972645F50617274792F4C7749502F4B
:10E600007372632F636F72652F7463702E630000E3
:10E61000696E76616C696420736F636B65742073D7
:10E620007461746520666F72207265637620636121
:10E630006C6C6261636B0000417373657274696F27
:10E640006E2022257322206661696C6564206174E6
:10E65000206C696E6520256420696E2025730A0090
:10E660002DE9F04107460D4614461E4600BF002D19
:10E670000CD100BF0EA34FF4D36219A11FA0F4F771
:10E68000BBFC00BF6FF00F00BDE8F08100BF3CB1E4
:10E690002189284600F046F82046F9F7BFFF04E03C
:10E6A0001EB92846FBF7E6FCEEE70020ECE7000089
:10E6B0002E2E2F4D6964646C6577617265732F54DB
:10E6C000686972645F50617274792F4C7749502F7A
:10E6D0007372632F636F72652F7463702E63000013
:10E6E0007463705F726563765F6E756C6C3A2069F7
:10E6F0006E76616C696420706362000041737365BB
:10E700007274696F6E2022257322206661696C65C0
:10E7100064206174206C696E6520256420696E2018
:10E7200025730A002DE9F04104460F4600BF002C76
:10E730000AD100BF1CA340F2CF3227A12CA0F4F7CE
:10E740005BFC00BFBDE8F08100BF00BF207D012859
:10E7500008D100BF14A340F2D2322FA124A0F4F7B5
:10E760004BFC00BF00BF208D384485B2B5F5066F65
:10E7700002DC208DA84203DD4FF40660208500E016
:10E780002585204601F0FEFA0646B6F5067F08D339
:10E7900000BF608B40F00200608300BF2046FDF7A1
:10E7A0009FFC00BFCEE700002E2E2F4D6964646CE5
:10E7B0006577617265732F54686972645F50617226
:10E7C00074792F4C7749502F7372632F636F726582
:10E7D0002F7463702E6300007463705F72656376DC
:10E7E00065643A20696E76616C69642070636200CA
:10E7F000417373657274696F6E20222573222066DF
:10E8000061696C6564206174206C696E65202564A3
:10E8100020696E2025730A00646F6E27742063617F
:10E820006C6C207463705F72656376656420666FDC
:10E8300072206C697374656E2D70636273000000E2
:10E8400070B506460D4600BF002D07D100BF09A3D5
:10E85000FF2214A11DA0F4F7CFFB00BF00BF344678
:10E8600005E0E06FA84201D10020E067E468002CD9
:10E87000F7D170BD2E2E2F4D6964646C657761727F
:10E8800065732F54686972645F50617274792F4C9C
:10E890007749502F7372632F636F72652F746370A3
:10E8A0002E6300007463705F72656D6F76655F6CD8
:10E8B000697374656E65723A20696E76616C69641D
:10E8C000206C697374656E65720000004173736536
:10E8D0007274696F6E2022257322206661696C65EF
:10E8E00064206174206C696E6520256420696E2047
:10E8F00025730A002DE9F041044600BF002C08D121
:10E9000000BF20A340F2C1622BA131A0F4F774FB39
:10E9100000BF00BF206F18B96FF00500BDE8F0819F
:10E92000256F2846FEF7C4F810B16FF00500F5E733
:10E930002868206704F16C0600E03668306858B13A
:10E940003168C9684868F7F733FC0746E9684868E2
:10E95000F7F72EFC381AF0D4306828603560286844
:10E9600010B90020A4F8680094F84200FF2804DAE7
:10E9700094F84200401C84F842000020606300BF0D
:10E98000CCE700002E2E2F4D6964646C65776172B0
:10E9900065732F54686972645F50617274792F4C8B
:10E9A0007749502F7372632F636F72652F74637092
:10E9B0005F6F75742E6300007463705F7265786DAD
:10E9C00069743A20696E76616C69642070636200D4
:10E9D000417373657274696F6E20222573222066FD
:10E9E00061696C6564206174206C696E65202564C2
:10E9F00020696E2025730A0010B5044600BF002C64
:10EA000008D100BF20A340F2F9622CA133A0F4F793
:10EA1000F3FA00BF00BF206FA0B3A07E00F0040097
:10EA200080BB2046FFF766FF60BBB4F84810B4F81F
:10EA30006020914202DAB4F8481001E0B4F86010A6
:10EA4000084601EBD071C1F34F01A4F84A10B4F8A5
:10EA50004A00618E4900884204D2608E4004000C56
:10EA6000A4F84A00B4F84A00618E032202FB0100B8
:10EA7000A4F8480000BF608B40F00400608300BF32
:10EA80000020208610BD00002E2E2F4D6964646C7E
:10EA90006577617265732F54686972645F50617243
:10EAA00074792F4C7749502F7372632F636F72659F
:10EAB0002F7463705F6F75742E6300007463705FF2
:10EAC0007265786D69745F666173743A20696E76F9
:10EAD000616C6964207063620000000041737365BB
:10EAE0007274696F6E2022257322206661696C65DD
:10EAF00064206174206C696E6520256420696E2035
:10EB000025730A0010B5044600BF002C08D100BFD1
:10EB100008A340F2AD6214A11AA0F4F76DFA00BF89
:10EB200000BF204600F09EF810B9204600F03EF8E5
:10EB300010BD00002E2E2F4D6964646C65776172E4
:10EB400065732F54686972645F50617274792F4CD9
:10EB50007749502F7372632F636F72652F746370E0
:10EB60005F6F75742E6300007463705F7265786DFB
:10EB700069745F72746F3A20696E76616C696420A3
:10EB800070636200417373657274696F6E20222531
:10EB90007322206661696C6564206174206C696E03
:10EBA0006520256420696E2025730A0010B504468F
:10EBB00000BF002C08D100BF0AA34FF4D36216A1F6
:10EBC0001EA0F4F719FA00BF00BF94F84200FF2816
:10EBD00004DA94F84200401C84F842002046FDF715
:10EBE0007FFA10BD2E2E2F4D6964646C65776172BB
:10EBF00065732F54686972645F50617274792F4C29
:10EC00007749502F7372632F636F72652F7463702F
:10EC10005F6F75742E6300007463705F7265786D4A
:10EC200069745F72746F5F636F6D6D69743A2069A8
:10EC30006E76616C69642070636200004173736575
:10EC40007274696F6E2022257322206661696C657B
:10EC500064206174206C696E6520256420696E20D3
:10EC600025730A0070B5044600BF002C08D100BF10
:10EC700022A340F263622EA136A0F4F7BDF900BFD3
:10EC800000BF206F10B96FF0050070BD256F07E061
:10EC90002846FDF70DFF10B16FF00500F5E72D6870
:10ECA00028680028F4D12846FDF702FF10B16FF064
:10ECB0000500EAE7E06E2860206FE066002020672C
:10ECC00000BF608B40F40060608300BFE968486863
:10ECD000F7F76EFA0646E9688889F7F776FA00F0E2
:10ECE000030008B1012000E00020298908443044D5
:10ECF000E0640020606300BFC7E700002E2E2F4DA8
:10ED00006964646C6577617265732F5468697264B5
:10ED10005F50617274792F4C7749502F7372632F53
:10ED2000636F72652F7463705F6F75742E6300007C
:10ED30007463705F7265786D69745F72746F5F7011
:10ED40007265706172653A20696E76616C696420E3
:10ED500070636200417373657274696F6E2022255F
:10ED60007322206661696C6564206174206C696E31
:10ED70006520256420696E2025730A0070B504465D
:10ED80000E4615462CB1207A18B1207AF8F78AFA87
:10ED900070BD2846F6F71EFCFAE700002DE9F04F9B
:10EDA00085B083460F4690461D46DDF8389000BF7B
:10EDB000002D08D100BF1EA340F2C47229A130A0CB
:10EDC000F4F71AF900BF00BF00BFB9F1000F08D176
:10EDD00000BF17A340F2C57233A129A0F4F70CF9C4
:10EDE00000BF00BF002646F2080A3846F7F7E0F9F0
:10EDF00014220490DDE90F018DE80704002231465A
:10EE00004046049BFDF78CFB044614B905B0BDE8F1
:10EE1000F08F3346002221465846FDF791FC4B46C1
:10EE20002A4621465846FDF70DFC00BFEEE70000DC
:10EE30002E2E2F4D6964646C6577617265732F5453
:10EE4000686972645F50617274792F4C7749502FF2
:10EE50007372632F636F72652F7463705F6F757465
:10EE60002E6300007463705F7273743A20696E766B
:10EE7000616C6964206C6F63616C5F697000000095
:10EE8000417373657274696F6E2022257322206648
:10EE900061696C6564206174206C696E652025640D
:10EEA00020696E2025730A007463705F7273743A70
:10EEB00020696E76616C69642072656D6F74655F40
:10EEC0006970000070B5054600BF002D08D100BF75
:10EED0000CA340F2826217A11DA0F4F78DF800BFC9
:10EEE00000BF0220F7F7E8FE04460CB9002070BD11
:10EEF00095E80F0084E80F006068F9F79FFD204651
:10EF0000F5E700002E2E2F4D6964646C6577617201
:10EF100065732F54686972645F50617274792F4C05
:10EF20007749502F7372632F636F72652F7463700C
:10EF30002E6300007463705F7365675F636F707941
:10EF40003A20696E76616C69642073656700000021
:10EF5000417373657274696F6E2022257322206677
:10EF600061696C6564206174206C696E652025643C
:10EF700020696E2025730A0010B5044644B160680C
:10EF800010B16068F9F74AFB21460220F7F7C6FD89
:10EF900010BD70B5044605E025682046FFF7ECFF7C
:10EFA0002C4600BF002CF7D170BD00002DE9F047C2
:10EFB00004460025A94600BF002C08D100BF2CA3A1
:10EFC00040F2EA7237A13FA0F4F716F800BF00BF85
:10EFD00005F0010008B1042000E0002005F0020166
:10EFE00009B1002100E00021084405F0080109B141
:10EFF000002100E00021084405F0100109B10021C2
:10F0000000E0002100EB0108206DF7F7D1F88246FF
:10F010005346002241462046FDF714FA06464EB9F3
:10F0200000BF608B40F00300608300BF6FF0010001
:10F03000BDE8F0874B462A4631462046FDF780FB67
:10F04000231D224631462046FDF7FCFA07462FB124
:10F0500000BF608B40F00300608306E000BF608B60
:10F060004FF6FC710840608300BF3846E0E70000BF
:10F070002E2E2F4D6964646C6577617265732F5411
:10F08000686972645F50617274792F4C7749502FB0
:10F090007372632F636F72652F7463705F6F757423
:10F0A0002E6300007463705F73656E645F656D70DE
:10F0B00074795F61636B3A20696E76616C69642074
:10F0C00070636200417373657274696F6E202225EC
:10F0D0007322206661696C6564206174206C696EBE
:10F0E0006520256420696E2025730A0070B50446EA
:10F0F00000BF002C08D100BF16A340F2EB3222A1C2
:10F1000028A0F3F779FF00BF00BFE06EE8B1E56E1D
:10F1100000E02D6828680028FBD1E9688889F7F7A6
:10F1200054F800F0070078B90120F7F74EF8E968C5
:10F1300089890843E968888100BF608B40F020001E
:10F14000608300BF002070BD00BF01212046FBF797
:10F15000D1FAF8E72E2E2F4D6964646C65776172E1
:10F1600065732F54686972645F50617274792F4CB3
:10F170007749502F7372632F636F72652F746370BA
:10F180005F6F75742E6300007463705F73656E64E7
:10F190005F66696E3A20696E76616C69642070639F
:10F1A00062000000417373657274696F6E202225DE
:10F1B0007322206661696C6564206174206C696EDD
:10F1C0006520256420696E2025730A002DE9F04F23
:10F1D00085B04FF00009E9480068401CE749086025
:10F1E000E7480078401CE649087000BF0025E54864
:10F1F0000468E3E200BF207D002808D100BFE2A33D
:10F2000040F2BE42ECA1F7A0F3F7F6FE00BF00BF4C
:10F2100000BF207D012808D100BFDBA340F2BF4220
:10F22000FAA1F0A0F3F7E8FE00BF00BF00BF207D09
:10F230000A2808D100BFD4A34FF49862FEA1E9A028
:10F24000F3F7DAFE00BF00BFA07FCD4909788842FE
:10F2500002D12546E468B1E2C9480078A0770026CB
:10F26000B046207D022806D194F84200062802DB31
:10F27000701CC6B2D1E094F842000C2802DB701C6E
:10F28000C6B2CAE094F8990000285DDD00BF206F87
:10F29000002808D000BFBCA340F2D442F2A1D1A004
:10F2A000F3F7AAFE00BF00BF00BFE06E002808D140
:10F2B00000BFB5A340F2D542F8A1CAA0F3F79CFE67
:10F2C00000BF00BF94F89A000C2802DB701CC6B285
:10F2D000A3E094F89900401EFE490F5C94F8980052
:10F2E000B84204DA94F89800401C84F8980094F826
:10F2F0009800B84227DB4FF0010AB4F8600030B93B
:10F30000204601F0B7FA70B14FF0000A0BE0B4F8F4
:10F310006010204600F0F4FA28B92046FCF7E0FE21
:10F3200008B94FF0000ABAF1000F0BD0002084F8A2
:10F33000980094F89900072804D294F89900401C8A
:10F3400084F8990000BF68E0B4F93000002809DBB8
:10F35000B4F9300047F6FF71884203DA208E401C72
:10F3600000B22086B4F93000B4F94010884254DB72
:10F370002046FFF777FC18B1206F70BBE06E60B3DA
:10F38000207D02281ED094F842200C2A02D294F844
:10F39000422000E00C221146B4F93E20B4F93C3082
:10F3A00002EBE302CC4B5B5C02FA03F047F6FF7220
:10F3B000904201DA024601E047F6FF7212B2A4F869
:10F3C000402000BF00202086B4F84800B4F8601048
:10F3D000884203DAB4F8480002E01EE0B4F86000A6
:10F3E000049004984010A4F84A00B4F84A00618ED2
:10F3F0004FF6FF7202EA4101884205DA608E11463B
:10F4000001EA4000A4F84A00608EA4F848000020F9
:10F41000A4F86A002046FFF7C9FB207D06280BD11F
:10F42000A07E00F0100038B15449206A0968081A1B
:10F43000282801D9701CC6B2607A00F00800D0B349
:10F44000207D042802D0207D072834D1A349D4F898
:10F45000940008444FF4FA71B0FBF1F0474A216A76
:10F460001268511A884206D2701CC6B208F1010017
:10F4700000F0FF081FE094F89B1042F29F4211FB3E
:10F4800002F1D4F8940000EBC1004FF4FA71B0FB24
:10F49000F1F03A4A216A1268511A88420BD220468A
:10F4A000FCF7F0F88146B9F1000F04D194F89B0005
:10F4B000401C84F89B00606F68B13049206A09687D
:10F4C000081AB4F9401001EB4101B0EB410F02D32F
:10F4D0002046FBF703FC207D032807D12749206A3B
:10F4E0000968081A282801D9701CC6B2207D09288D
:10F4F00007D12249206A0968081AF02801D9701C2E
:10F50000C6B2002E37D0D4F890A02046FDF77EFC7E
:10F510008DB100BF1B480068844208D100BF1AA308
:10F5200040F26D526EA12FA0F3F766FD00BF00BF41
:10F53000E068E86011E000BF12480068A04208D00F
:10F5400000BF11A340F2715270A126A0F3F754FD41
:10F5500000BF00BF0B49E0680860B8F1000F0BD096
:10F56000208BE18A221DCDE900210290234620460E
:10F57000626A216DE0E0FBE0E0E00000280100208D
:10F580003E010020340100202E2E2F4D6964646C52
:10F590006577617265732F54686972645F50617238
:10F5A00074792F4C7749502F7372632F636F726594
:10F5B0002F7463702E6300007463705F736C6F77D9
:10F5C000746D723A20616374697665207063622D90
:10F5D0003E737461746520213D20434C4F53454474
:10F5E0000A000000417373657274696F6E202225F2
:10F5F0007322206661696C6564206174206C696E99
:10F600006520256420696E2025730A007463705F8D
:10F61000736C6F77746D723A2061637469766520DC
:10F620007063622D3E737461746520213D204C49E6
:10F630005354454E0A0000007463705F736C6F771B
:10F64000746D723A20616374697665207063622D0F
:10F650003E737461746520213D2054494D452D57FA
:10F660004149540A000000007463705F736C6F7747
:10F6700074696D723A20706572736973742074696D
:10F68000636B696E67207769746820696E2D666C9C
:10F690006967687420646174610000007463705F5E
:10F6A000736C6F7774696D723A20706572736973E9
:10F6B00074207469636B696E67207769746820656C
:10F6C0006D7074792073656E64206275666665720C
:10F6D00000000000D1290108C4290108B84C0A0023
:10F6E0007463705F736C6F77746D723A206D6964C8
:10F6F000646C652074637020213D207463705F61C9
:10F7000063746976655F7063627300007463705F31
:10F71000736C6F77746D723A2066697273742070BF
:10F720006362203D3D207463705F61637469766538
:10F730005F70636273000000FFF730FBD4F810B015
:10F74000207D03902746E4683846FBF781F90020C6
:10F750004849087000BFBAF1000F03D06FF00C01E8
:10F760005846D04700BF4348007800B13EE524E04A
:10F770002546E468287F401C2877287F697F8842D7
:10F780001BDB002028773B49087000BFD5F88C00B0
:10F7900030B12946D5F88C2028699047814601E090
:10F7A0004FF0000900BF3348007800B11EE5B9F101
:10F7B000000F02D12846FCF793FC00BF002C7FF419
:10F7C00019AD00252C4804684EE000BF207D0A28B2
:10F7D0000AD000BFAFF2502340F2A15227A1AFF2EE
:10F7E000FC10F3F709FC00BF00BF00262F49206A78
:10F7F0000968081AF02801D9701CC6B2002E31D051
:10F800002046FDF703FB9DB100BF1B480068844202
:10F810000AD100BFAFF2902340F2AF5224A1AFF261
:10F820003C20F3F7E9FB00BF00BFE068E86013E0AD
:10F8300000BF11480068A0420AD000BFAFF2B82351
:10F8400040F2B35224A1AFF26420F3F7D5FB00BF1E
:10F8500000BF0949E06808602746E4683846FBF7BE
:10F86000F7F801E02546E468002CAED105B0BDE80C
:10F87000F08F00003C010020380100207463705FAD
:10F88000736C6F77746D723A2054494D452D574112
:10F890004954207063622D3E7374617465203D3D50
:10F8A0002054494D452D574149540000280100205E
:10F8B0007463705F736C6F77746D723A206D6964F6
:10F8C000646C652074637020213D207463705F74E4
:10F8D000775F7063627300007463705F736C6F773F
:10F8E000746D723A20666972737420706362203D91
:10F8F0003D207463705F74775F7063627300000013
:10F900002DE9F04F85B005460E4600270024A3469A
:10F9100000BF002D08D100BF79A340F24B3285A172
:10F920008DA0F3F769FB00BF00BFEC6E24B94FF068
:10F93000FF3005B0BDE8F08F002E0CD100BF00BF36
:10F940006FA340F253328EA183A0F3F755FB00BFA3
:10F9500000BFB01FEDE72089B04201DC0020E8E7DE
:10F9600000BF688EB04208DA00BF65A340F25B3288
:10F970008CA179A0F3F740FB00BF00BF00BF208936
:10F98000002808DC00BF5EA34FF4577289A172A063
:10F99000F3F732FB00BF00BF94F80A8008F00100C3
:10F9A00008B1042000E0002008F0020109B10021A4
:10F9B00000E00021084408F0080109B1002100E03E
:10F9C0000021084408F0100109B1002100E00021E5
:10F9D000084404902089801B1FFA80FA0498504440
:10F9E00081B24FF420723620F8F782F98346BBF1DA
:10F9F000000F00D16EE0606800892189401A304410
:10FA000080B20290DBF80430049A9918606852467C
:10FA1000029BF8F763FD504500D05BE0E168888900
:10FA2000F6F7D3FB00F03F090020039009F008002F
:10FA300028B129F00809039840F00800039009F064
:10FA4000010028B129F00109039840F0010003905A
:10FA5000E1684868F6F7ACFB30440346CDE9008026
:10FA600059462846039AFAF7D7FC074607B931E00A
:10FA70006068F8F7BDFB35F8661F081A28806268D1
:10FA80001289A2EB0A0291B26068F8F723FF20897D
:10FA9000A0EB0A0020814846F6F797FBE1688989C8
:10FAA0000843E16888816068F8F7A2FB2988084468
:10FAB00028807868F8F79CFB2988084425F86609AF
:10FAC000206838602760386810B90020A5F8680001
:10FAD00000202EE700BF47B100BF09A34FF47672A4
:10FAE00038A11DA0F3F788FA00BF00BFBBF1000FDB
:10FAF00002D05846F8F792FD4FF0FF3019E70000AA
:10FB00002E2E2F4D6964646C6577617265732F5476
:10FB1000686972645F50617274792F4C7749502F15
:10FB20007372632F636F72652F7463705F6F757488
:10FB30002E6300007463705F73706C69745F756E20
:10FB400073656E745F7365673A20696E76616C6980
:10FB50006420706362000000417373657274696FA2
:10FB60006E2022257322206661696C6564206174B1
:10FB7000206C696E6520256420696E2025730A005B
:10FB800043616E27742073706C6974207365676DB0
:10FB9000656E7420696E746F206C656E6774682082
:10FBA0003000000073706C6974203C3D206D7373ED
:10FBB00000000000757365672D3E6C656E203E2069
:10FBC00030000000736567203D3D204E554C4C00D1
:10FBD00010B50948006868B90848006810B90848B5
:10FBE000006838B101200449086000220549FA2064
:10FBF000F9F758FE10BD0000740100203401002008
:10FC000038010020950D01083EB5044629480078CA
:10FC100000F0040000B13EBD00BF002C08D100BFC1
:10FC200025A340F2EE2231A138A0F3F7E5F900BF99
:10FC300000BF2048007800F0020018B33D49606A18
:10FC40000968081A26D4218D606A08443949096870
:10FC5000081A00281EDC3848006800883649096800
:10FC60004988364ACDE9002102903248006834497B
:10FC700009884218314B1B1D324801682046FFF7A6
:10FC80008DF8C8E70B48007800F0010010B12E484D
:10FC9000006820622A480088002808DD00BF608BC9
:10FCA00040F00200608300BF2046FCF719FA00BF55
:10FCB000B1E70000600100202E2E2F4D6964646CB6
:10FCC0006577617265732F54686972645F50617201
:10FCD00074792F4C7749502F7372632F636F72655D
:10FCE0002F7463705F696E2E630000007463705F31
:10FCF00074696D65776169745F696E7075743A20B7
:10FD0000696E76616C69642070636200417373652B
:10FD10007274696F6E2022257322206661696C659A
:10FD200064206174206C696E6520256420696E20F2
:10FD300025730A005401002044010020EC8F0020AC
:10FD40005E010020580100202801002010B5FAF7BC
:10FD500031FE06480078401CC0B20449087000F02B
:10FD6000010008B1FFF732FA10BD00003D0100208C
:10FD70000348007840F01000014908707047000007
:10FD80006101002070B5044600BF002C08D100BFFF
:10FD90001CA340F2A63227A12FA0F3F72DF900BF34
:10FDA00000BF218D606A4518608EE16AB0F5866FEC
:10FDB00002DD4FF4866000E0608E0844281A04D407
:10FDC000208D6085E06A281A70BDE16A606A401A79
:10FDD000002802DD0020608512E0616AE06A461AB0
:10FDE00000BFB6F5803F08D300BF06A340F2B6328D
:10FDF00023A119A0F3F700F900BF00BF668500BF7B
:10FE00000020E1E72E2E2F4D6964646C65776172E6
:10FE100065732F54686972645F50617274792F4CF6
:10FE20007749502F7372632F636F72652F746370FD
:10FE30002E6300007463705F7570646174655F7237
:10FE400063765F616E6E5F776E643A20696E76618D
:10FE50006C69642070636200417373657274696FCA
:10FE60006E2022257322206661696C6564206174AE
:10FE7000206C696E6520256420696E2025730A0058
:10FE80006E65775F7263765F616E6E5F776E64201A
:10FE90003C3D203078666666660000002DE9FF4F25
:10FEA00091B004468A4617464FF0000B002500200B
:10FEB00010900F900E9000260B900A9081460990AA
:10FEC00000BF002C0DD100BFE7A34FF4CF72F3A108
:10FED000F8A0F3F791F800BF6FF00F0015B0BDE880
:10FEE000F08F00BFB4F8621001EBD1725210638E34
:10FEF0009A4201DD628E04E0B4F8620000EBD07239
:10FF0000521092B20792079A0AB1079800E0608EE9
:10FF1000079000BFBAF1000F0BD100BFD2A340F28F
:10FF2000AD12EEA1E3A0F3F767F800BF6FF00F008A
:10FF3000D4E700BF3946204600F0C2FB089008987D
:10FF400008B10898CAE7B4F866000D9000200C903C
:10FF5000E06E00287ED0E56E00E02D68286800285D
:10FF6000FBD1A87A00F0010008B1042000E00020D5
:10FF7000A97A01F0020109B1002100E00021084442
:10FF8000A97A01F0080109B1002100E0002108442C
:10FF9000A97A01F0100109B1002100E00021084414
:10FFA000069000BF2989069801440798814208DD20
:10FFB00000BFADA34FF4F372D5A1BEA0F3F71CF8B8
:10FFC00000BF00BF2989069801440798401A1FFA0C
:10FFD00080F8B4F868000A90BDF82800002831DDE8
:10FFE00000BFBDF82800404508DD00BF9EA34FF4C8
:10FFF000FC72CDA1AFA0F2F7FFFF00BF00BF1095CC
:020000040801F1
:10000000BDF82800B84202DABDF8280000E0384602
:10001000404501DD404607E0BDF82800B84202DA5D
:10002000BDF8280000E03846814606EB090086B29C
:10003000BDF82800A0EB090080B20A90A8EB0900E7
:100040001FFA80F800BFBDF8280060B1BE420AD098
:1000500000BF00E079E084A34FF40072BAA195A03C
:10006000F2F7CAFF00BF00BFBE426DDAB8F1000F61
:100070006ADD2889002867DDB81B404501DD404660
:1000800000E0B81B80B205901095149800F00100B4
:10009000E8B1012114980AAB4246CDE90040029133
:1000A00000200599FCF7F6FDB0F1000B00D18CE2C1
:1000B0000AEB0601DBF80400059AF0F727F9584629
:1000C000F8F796F80D99084480B20D9038E068680A
:1000D000049002E0049800680490049800680028E6
:1000E000F8D10498007B00F0C000A0B904984168E2
:1000F0004089084450450ED100BF46B100BF5AA305
:1001000040F2312298A16BA0F2F776FF00BF00BF4A
:100110000598099013E0012200200599F7F7E8FD02
:10012000B0F1000B00D150E20AEB0600CBF804005E
:100130005846F8F75DF80D99084480B20D9000BF5D
:100140000598304486B200BF0DE000BFB4F86800E7
:1001500040B100BF44A340F24A228EA155A0F2F75D
:100160004BFF00BF00BF7EE1B81B80B206900C9928
:100170000798401A80B20590DDE90510884201DA3F
:10018000069800E005980490149800F001000028FB
:100190002FD00E9808B9012100E000211498CDE974
:1001A000004002910C9A0498104481B20AAB3620A8
:1001B000079AFCF76FFDB0F1000800D105E200BF1F
:1001C000B8F80A100498814208DA00BF26A340F26A
:1001D00066227CA137A0F2F70FFF00BF00BF0AEB39
:1001E0000601D8F804300C9A9818049AF0F78EF8A3
:1001F0002BE000BFBDF8280040B100BF1AA340F2B9
:10020000712280A12BA0F2F7F7FE00BF00BF0122F0
:1002100036200499F7F76CFD039000B9D5E10AEB9D
:100220000601039841604FF4207236200C99F7F7CD
:100230005FFDB0F1000803D10398F8F7EFF9C4E1CE
:1002400040460399F7F72CFF00BF4046F7F7D0FF71
:100250000D99084480B20D900D98092803D94046A5
:10026000F8F7DCF9B1E1D5E02E2E2F4D6964646C0E
:100270006577617265732F54686972645F5061724B
:1002800074792F4C7749502F7372632F636F7265A7
:100290002F7463705F6F75742E6300007463705FFA
:1002A00077726974653A20696E76616C6964207052
:1002B00063620000417373657274696F6E2022255A
:1002C0007322206661696C6564206174206C696EBC
:1002D0006520256420696E2025730A007463705FB1
:1002E00077726974653A20617267203D3D204E55F2
:1002F0004C4C202870726F6772616D6D657220764C
:10030000696F6C61746573204150492900000000D9
:100310006D73735F6C6F63616C20697320746F6FB2
:1003200020736D616C6C0000696E636F6E7369732E
:1003300074656E74206F76657273697A6520767362
:100340002E20737061636500696E636F6E736973ED
:1003500074656E74206F76657273697A6520767342
:100360002E206C656E0000007463705F7772697494
:10037000653A20524F4D2070627566732063616E3E
:100380006E6F74206265206F76657273697A65643A
:1003900000000000756E73656E745F6F7665727332
:1003A000697A65206D69736D617463682028706374
:1003B000622D3E756E73656E74206973204E554CC8
:1003C0004C2900007463705F77726974653A20632A
:1003D0006865636B20746861742066697273742049
:1003E000706275662063616E20686F6C642074684B
:1003F0006520636F6D706C657465207365676C65EF
:100400006E0000006F76657273697A65203D3D204D
:10041000300000000B980090E06D831900224146E7
:100420002046F9F7F9FF109000B9CEE00E9810B908
:1004300010980E9011E000BF0F9850B900BFAFF2B6
:10044000D81340F2AB2275A1AFF29810F2F7D4FDA9
:1004500000BF00BFDDE90F10086010980F900498EE
:10046000304486B200BFBE42FFF67EAEB9F1000F47
:1004700021DDD5F8048017E0B8F808004844A8F852
:100480000800D8F8000068B9B8F80A20D8F80410B5
:1004900088184A465146EFF739FFB8F80A00484431
:1004A000A8F80A00D8F80080B8F1000FE4D1288934
:1004B0004844288100BFBDF82800A4F86800BBF1BB
:1004C000000F17D000BF55B900BFAFF264234FF43F
:1004D000387257A1AFF22420F2F78EFD00BF00BFA3
:1004E00059466868F7F7DCFD2889BBF8081008440E
:1004F000288132E0099800282FDD00BF0DB168681F
:1005000050B900BFAFF2A02340F2E62256A1AFF2ED
:100510005C20F2F771FD00BF00BFD5F8048007E052
:10052000B8F8081009980844A8F80800D8F800801E
:10053000D8F800000028F3D1B8F80810099808444A
:10054000A8F80800B8F80A1009980844A8F80A00A2
:10055000298909980844288100BF15B90E98E066DA
:1005600001E00E98286054F85C0F38442060208920
:10057000C01B20810D98608160895C3C80B100BF08
:10058000206F60B9E06E50B900BFAFF2243340F283
:10059000123243A1AFF2E420F2F72EFD00BF00BFFC
:1005A000109880B11098C06868B1149800F00200EB
:1005B00048B90820F5F709FE1099C96889890843E8
:1005C0001099C9688881002088E400BF608B40F0E2
:1005D0008000608300BFBBF1000F02D05846F8F7DF
:1005E0001DF80E9810B10E98FEF7D3FCB4F8660013
:1005F00080B100BF206F60B9E06E50B900BFAFF2AC
:10060000983340F2273226A1AFF25830F2F7F4FCCB
:1006100000BF00BF4FF0FF3060E4000070726576ED
:100620005F73656720213D204E554C4C0000000053
:100630007463705F77726974653A2063616E6E6F80
:100640007420636F6E636174656E61746520776892
:10065000656E207063622D3E756E73656E742069E1
:100660007320656D707479007463705F777269745C
:10067000653A20657874656E73696F6E206F6620C9
:100680007265666572656E63652072657175697203
:100690006573207265666572656E636500000000B3
:1006A0007463705F77726974653A2076616C69640F
:1006B000207175657565206C656E67746800000053
:1006C00070B504460D4600BF002C08D100BF2EA314
:1006D00040F2331239A141A0F2F78EFC00BF00BFF7
:1006E000207D04280BD0207D072808D0207D0228FB
:1006F00005D0207D032802D06FF00A0070BD0DB92F
:100700000020FBE7B4F86400A84208DA00BF608B61
:1007100040F08000608300BF4FF0FF30EEE7B4F898
:100720006600092808D300BF608B40F0800060831A
:1007300000BF4FF0FF30E1E7B4F86600002810D0AA
:1007400000BF206F00280BD1E06E002808D100BF49
:100750000DA340F255122BA120A0F2F74DFC00BFD3
:100760000FE000BF206F10B9E06E002808D000BF76
:1007700005A34FF4AC7232A118A0F2F73DFC00BF04
:1007800000BF0020BAE700002E2E2F4D6964646C74
:100790006577617265732F54686972645F50617226
:1007A00074792F4C7749502F7372632F636F726582
:1007B0002F7463705F6F75742E6300007463705FD5
:1007C00077726974655F636865636B733A20696EFD
:1007D00076616C6964207063620000004173736528
:1007E0007274696F6E2022257322206661696C65C0
:1007F00064206174206C696E6520256420696E2018
:1008000025730A007463705F77726974653A2070AB
:1008100062756673206F6E207175657565203D3E4B
:10082000206174206C65617374206F6E6520717532
:10083000657565206E6F6E2D656D707479000000B2
:100840007463705F77726974653A206E6F207062AE
:10085000756673206F6E207175657565203D3E204D
:10086000626F74682071756575657320656D70744D
:10087000790000002DE9FC5F04464FF0000A00BF3C
:10088000002C08D100BF37A340F64F0242A14BA075
:10089000F2F7B2FB00BF00BFE56E15B90020BDE85E
:1008A000FC9F94F89A00FF2804DA94F89A00401C00
:1008B00084F89A00E9688889F5F787FC00F0010060
:1008C00018B1288908B9012000E000208146B9F15B
:1008D000000F01D1012000E000208346E868436852
:1008E0005A4651462046FBF7ADFD064616B94FF075
:1008F000FF30D4E77768B9F1000F09D01120F5F780
:1009000064FCB9894CF2FF0211400843B8810DE044
:10091000706814300090696809892A89891A8BB235
:10092000012268680099F7F7D9FD00BFE9684868B7
:10093000F5F73EFC00F10108206DB0EB080001D591
:10094000C4F850805346002231462046FBF7F8FE9B
:10095000231D224631462046FBF774FE0190019884
:100960009DE700002E2E2F4D6964646C65776172DF
:1009700065732F54686972645F50617274792F4C8B
:100980007749502F7372632F636F72652F74637092
:100990005F6F75742E6300007463705F7A65726FA9
:1009A0005F77696E646F775F70726F62653A206916
:1009B0006E76616C696420706362000041737365D8
:1009C0007274696F6E2022257322206661696C65DE
:1009D00064206174206C696E6520256420696E2036
:1009E00025730A0070B505460C4616460549204693
:1009F000FDF7E0FD04480460012004490870002070
:100A000070BD0000110A01088C01002000000020C8
:100A10002DE9F043CDB081460E4614461F46802195
:100A20002DA8EFF79AFC80210DA8EFF796FC002582
:100A3000A846002C74D021893046FDF773FE228928
:100A40002DA86168EFF762FC257A9DF8B400AA280A
:100A500004D1681E2DA9085C3C280DD04FF0070872
:100A600001222DA90DA8F2F7DFFB012342460DA9B3
:100A70003046FFF713FA61E0E81E81B20DF1B500D0
:100A800001F0BEFEA91E2DAA515C88420DD04FF088
:100A9000070802222DA90DA8F2F7C6FB0123424642
:100AA0000DA93046FFF7FAF948E09DF8B8200DF19E
:100AB000B9016846EFF72AFC9DF8B700022815D166
:100AC0002649C1F800D0084600684078C01D00F0F3
:100AD000FF082DAA0DA92148006800F0DBFA0123C8
:100AE00042460DA93046FFF7D9F927E09DF8B70037
:100AF00003280DD11A49C1F800D00846006800F05B
:100B000009FB01232A462DA93046FFF7C7F915E056
:100B10009DF8B700042804D10020124908700DE0A8
:100B200010E04FF0070803222DA90DA8F2F77CFB77
:100B3000012342460DA93046FFF7B0F92046F7F7EA
:100B40006DFD09E047B90020074908703046F9F704
:100B500091FA4DB0BDE8F0830020FAE79001002043
:100B600094010020010000200000002038B5044658
:100B70000D46F5F731FB174804601748056006215C
:100B80001648F8F723FE00280AD000BF00BF14A3C0
:100B900040F261221EA127A0F2F72EFA00BF00BF8B
:100BA0002E48F8F749FE00280AD000BF00BF0CA36A
:100BB00040F265222AA11FA0F2F71EFA00BF00BF73
:100BC00000204FF4806302462E4900902EA0F8F7D3
:100BD0004DFE38BDC4000020C8000020CC0000201D
:100BE0002E2E2F4D6964646C6577617265732F5486
:100BF000686972645F50617274792F4C7749502F25
:100C00007372632F6170692F74637069702E630053
:100C10006661696C656420746F20637265617465D8
:100C20002074637069705F746872656164206D62BE
:100C30006F780000417373657274696F6E202225AE
:100C40007322206661696C6564206174206C696E32
:100C50006520256420696E2025730A00D0000020DD
:100C60006661696C656420746F2063726561746588
:100C7000206C6F636B5F74637069705F636F726524
:100C800000000000CD0D010874637069705F746826
:100C900072656164000000002DE9F04105460E46D2
:100CA000174600BF1448F8F7B8FD38B900BF13A3C2
:100CB000FC221EA121A0F2F79FF900BF00BF08206F
:100CC000F5F7FAFF04461CB94FF0FF30BDE8F0819C
:100CD000002020706560A660E76021460648F8F7AE
:100CE0008DFD30B121460820F5F718FF4FF0FF3099
:100CF000ECE70020EAE70000CC0000202E2E2F4D6C
:100D00006964646C6577617265732F546869726495
:100D10005F50617274792F4C7749502F7372632F33
:100D20006170692F74637069702E6300496E76611B
:100D30006C6964206D626F78000000004173736518
:100D40007274696F6E2022257322206661696C655A
:100D500064206174206C696E6520256420696E20B2
:100D600025730A0070B505460C4694F8310000F072
:100D7000180028B1054A21462846FFF78DFF70BDAF
:100D8000034A21462846FFF787FFF8E7CD420008CF
:100D9000454F000810B50446FEF7D8FF0748006825
:100DA00010B90748006828B100220649FA20F8F770
:100DB00079FD02E000200449086010BD34010020E4
:100DC00038010020950D01087401002008B5114874
:100DD000F8F72AFD1048006820B1104800680E4955
:100DE0000968884715E069460D4800F0C1F8009889
:100DF00000280AD100BF00BF0AA3912215A11DA09F
:100E0000F2F7FAF800BF00BF03E0009800F046F8E0
:100E100000BFE8E7D0000020C4000020C800002088
:100E2000CC0000202E2E2F4D6964646C65776172B2
:100E300065732F54686972645F50617274792F4CC6
:100E40007749502F7372632F6170692F74637069D3
:100E5000702E630074637069705F7468726561649A
:100E60003A20696E76616C6964206D6573736167A1
:100E700065000000417373657274696F6E202225EE
:100E80007322206661696C6564206174206C696EF0
:100E90006520256420696E2025730A0010B504467C
:100EA000207820B101280ED0022818D113E0201D8F
:100EB00007C8904710B16068F7F7B0FB21460820DB
:100EC000F5F72CFE16E0D4E90110884721460720EB
:100ED000F5F724FE0EE0D4E9011088470AE000BFD0
:100EE00000BF05A3CF2210A117A0F2F785F800BF1D
:100EF00000BF00BF00BF10BD2E2E2F4D6964646C73
:100F00006577617265732F54686972645F506172AE
:100F100074792F4C7749502F7372632F6170692F4A
:100F200074637069702E630074637069705F7468B5
:100F3000726561643A20696E76616C6964206D65E2
:100F40007373616765000000417373657274696F44
:100F50006E2022257322206661696C6564206174AD
:100F6000206C696E6520256420696E2025730A0057
:100F70002DE9F04106460F4600BFF8F7AFFD0446E5
:100F8000601C60B91148F8F767FC0022394630460A
:100F9000F8F7A0FB0D48F8F747FCBDE8F08114B95D
:100FA000F8F7DEFBE9E70948F8F756FC2246394630
:100FB0003046F8F78FFB05460448F8F735FC681C07
:100FC00010B9F8F7CDFBD8E700BFE6E7D000002066
:100FD00070B505460E4600BF1348F8F71EFC40B931
:100FE00000BF12A340F25D121CA120A0F2F704F88A
:100FF00000BF00BF0720F5F75FFE044614B94FF0AD
:10100000FF3070BD012020706560A6602146064853
:10101000F8F7F4FB30B121460720F5F77FFD4FF0DC
:10102000FF30EEE70020ECE7CC0000202E2E2F4D05
:101030006964646C6577617265732F546869726462
:101040005F50617274792F4C7749502F7372632F00
:101050006170692F74637069702E6300496E7661E8
:101060006C6964206D626F780000000041737365E5
:101070007274696F6E2022257322206661696C6527
:1010800064206174206C696E6520256420696E207F
:1010900025730A002DE9F04707460C4690460025C7
:1010A00097F800907E78F01D00F0FF0AAA202070CB
:1010B0000020607098F80200A07098F80300E070BB
:1010C000267100BF08E005EB0901C8B2F3F7C4FAC6
:1010D000691D6054681CC5B2B542F4DBAAF1030077
:1010E00081B2601C01F08CFB711D60543C21B01D6D
:1010F0002154BDE8F087000070B504460D46012379
:101100002A46214602480068FEF7C8FE70BD00006E
:101110008C0100202DE9F041054600242E786F78DF
:1011200000BF10E0A81C005D012805D13119C8B22C
:101130000121F3F70BFB04E03119C8B20021F3F7EA
:1011400005FB601CC4B2BC42ECDBBDE8F08101468B
:101150000A69D1E901309860D1E90103586050680B
:10116000884201D188685060002008611068401EE4
:101170001060106870470000034B0360034B0B6066
:101180008023136070470000C00100201C02002073
:1011900000F1080141604FF0FF31816000F108016A
:1011A000C160016100210160704700210161704749
:1011B00010B502460B685C1C0CB9106907E002F11F
:1011C000080000E04068446824689C42FAD94468FA
:1011D0004C604C68A160886041600A611468641CBE
:1011E000146010BD42684A6093688B6093685960D0
:1011F0009160086103685B1C0360704700BF50206A
:1012000080F31188BFF34F8FBFF36F8F00BF0E487D
:101210000068401C0C49086008460068012812D18B
:101220000A480068C0B208B9012000E0002050B9A7
:1012300000BF502080F31188BFF34F8FBFF36F8F33
:1012400000BF00BFFEE77047B800002004ED00E0DB
:101250000D48006850B900BF502080F31188BFF3DB
:101260004F8FBFF36F8F00BF00BFFEE706480068D7
:10127000401E054908600846006820B9002080F338
:10128000118800BF00BF7047B800002070B5064647
:101290003546002E44D0083D2C4622496068096836
:1012A000084008B1012000E0002050B900BF5020E4
:1012B00080F31188BFF34F8FBFF36F8F00BF00BF64
:1012C000FEE7206808B9012000E0002050B900BF07
:1012D000502080F31188BFF34F8FBFF36F8F00BF93
:1012E00000BFFEE70F49606809680840C0B1206888
:1012F000B0B90C49606809688843606000F08EF9F5
:101300000949606809680844074908602046F7F7FA
:10131000A1FF06480068401C0449086001F0EEF98E
:1013200070BD0000B4000020A4000020B000002028
:1013300000204FF0E02108618861064800684FF402
:101340007A71B0FBF1F0401E4FF0E02148610720B8
:10135000086170475800002070B5EEF77DFF044625
:10136000102C16D304F1E02090F8F05315480078C3
:10137000854201DB012000E0002050B900BF502071
:1013800080F31188BFF34F8FBFF36F8F00BF00BF93
:10139000FEE70D48006800F4E0600C4909688842E7
:1013A00001D8012000E0002050B900BF502080F398
:1013B0001188BFF34F8FBFF36F8F00BF00BFFEE7F1
:1013C00070BD0000BC0000200CED00E0C00000205B
:1013D00070B504460025D4B11248006808B9012050
:1013E00000E0002050B900BF502080F31188BFF307
:1013F0004F8FBFF36F8F00BF00BFFEE700F00EF905
:1014000000212046F7F7D4FC01F078F905463DB9F4
:101410004FF0805004490860BFF34F8FBFF36F8FC8
:1014200070BD00009400002004ED00E0034909684D
:101430000160034909684160704700008400002092
:1014400070000020012001490860704780000020E2
:1014500070B504460D4654B900BF502080F3118882
:10146000BFF34F8FBFF36F8F00BF00BFFEE705488C
:10147000016818312046FFF79BFE01212846F7F747
:1014800097FC70BD5C0000202DE9F04706460F4632
:1014900034464FF00109002E60D0206D50B900BFD6
:1014A000502080F31188BFF34F8FBFF36F8F00BFC1
:1014B00000BFFEE7E06CB84201D23D4600E0E56CBB
:1014C000E06AA8424AD0206D012847D1244800682C
:1014D000844201D0012000E0002050B900BF50201C
:1014E00080F31188BFF34F8FBFF36F8F00BF00BF32
:1014F000FEE7D4F82C80E562A06900F0004010B946
:10150000C5F12000A06108EB8801164A02EB8101B9
:101510006069884201D1012000E00020F0B1201D67
:10152000FFF715FE40B994F82C10012088400E49B1
:10153000096881430C48016094F82C100120884010
:1015400009490968084308490860E16A01EB81011B
:10155000044A02EB8100211DFFF744FEBDE8F0873D
:101560005C000020F85000207400002010B586B008
:1015700000200590049003AA04A905A8FFF7FCFD2C
:101580000022DDE904101346CDE9002102901CA1E0
:101590001D48039A00F084FE1C4908600846006854
:1015A00008B1012400E00024012C15D100BF502017
:1015B00080F31188BFF34F8FBFF36F8F00BF4FF0E1
:1015C000FF301349086001201249086000201249C9
:1015D000086000F071F810E0601C08B1012000E024
:1015E000002050B900BF502080F31188BFF34F8F07
:1015F000BFF36F8F00BF00BFFEE706B010BD000055
:1016000049444C4500000000CD90000890000020A7
:101610008C00002078000020700000200248006844
:10162000401C014908607047940000201D48006874
:1016300018B101201C49086032E000201A490860F6
:101640001A480068B0FA80F0C0F11F0101EB810078
:10165000174A52F8200008B1012000E0002050B9DC
:1016600000BF502080F31188BFF34F8FBFF36F8FFF
:1016700000BF00BFFEE701EB81020D4B03EB8200D0
:1016800042685268426000F108024368934202D106
:101690004268526842604268D268064B1A6000BFD6
:1016A000704700009400002080000020740000209B
:1016B000F85000205C0000201CB5524800685249D8
:1016C000884201D0012000E0002050B900BF502026
:1016D00080F31188BFF34F8FBFF36F8F00BF00BF40
:1016E000FEE7484800684849491E884201D0012069
:1016F00000E0002050B900BF502080F31188BFF3F4
:101700004F8FBFF36F8F00BF00BFFEE73F49084612
:1017100000780190FF200A4610700846007800907B
:101720009DF8000000F0F0009DF80020904201D1EB
:10173000012000E0002050B900BF502080F3118844
:10174000BFF34F8FBFF36F8F00BF00BFFEE79DF861
:10175000000000F050002E4A107007202D4A106043
:1017600009E02C480068401E2A4A10609DF80000DD
:101770004006000E00909DF8000000F080008028D8
:10178000EFD024480068C0F10700042801D10120EF
:1017900000E0002050B900BF502080F31188BFF353
:1017A0004F8FBFF36F8F00BF00BFFEE7194800687F
:1017B0000002184A10601046008800F4E0601060D3
:1017C000124A019810700F482030006840F47000F1
:1017D0000C49203108600846006840F070400860FD
:1017E000FFF7A6FD00200C490860EEF7FDFC0B4852
:1017F000006840F0404009490860EEF7E1FC002035
:101800001CBD000000ED00E071C20F4100E400E0EB
:10181000BC000020C0000020B800002034EF00E031
:101820002DE9F0410446012600272246002101202F
:1018300000F01CF805462846F7F75CFC2846BDE892
:10184000F0812DE9F84304460D4601274FF00008CA
:101850002B46002211460120009400F034F8064681
:101860003046F7F747FC3046BDE8F8832DE9F843EA
:1018700005460E4617460DB1012000E0002050B984
:1018800000BF502080F31188BFF34F8FBFF36F8FDD
:1018900000BF00BFFEE705FB06F808F14800F7F7B8
:1018A000ABFD044664B1A14609F14809002084F863
:1018B00046003B464A46314628460094F7F729FC45
:1018C0002046BDE8F8832DE9F84380460E461746CA
:1018D0001D46DDF82090B8F1000F01D0012000E096
:1018E000002050B900BF502080F31188BFF34F8F04
:1018F000BFF36F8F00BF00BFFEE70DB1012000E016
:10190000002050B900BF502080F31188BFF34F8FE3
:10191000BFF36F8F00BF00BFFEE707B10EB101201C
:1019200000E0002050B900BF502080F31188BFF3C1
:101930004F8FBFF36F8F00BF00BFFEE707B90EB92F
:10194000012000E0002050B900BF502080F3118832
:10195000BFF34F8FBFF36F8F00BF00BFFEE748207C
:1019600000900098482801D1012000E0002050B9E3
:1019700000BF502080F31188BFF34F8FBFF36F8FEC
:1019800000BF00BFFEE700BF2C464CB1012084F829
:1019900046004B463A46314640460094F7F7B9FBBD
:1019A0002046BDE8F883000070B505460E462C467B
:1019B00054B900BF502080F31188BFF34F8FBFF39D
:1019C0006F8F00BF00BFFEE7FFF718FCD4E90F12CE
:1019D000206801FB0200A0600020A0632068606016
:1019E000E06B401E226C216800FB0211E160FF20C9
:1019F00084F8440084F845009EB9206908B90120A4
:101A000000E00020A8B904F1100000F02BFE80B126
:101A10004FF0805009490860BFF34F8FBFF36F8FBD
:101A200007E004F11000FFF7B3FB04F12400FFF717
:101A3000AFFBFFF70DFC012070BD000004ED00E0DE
:101A40002DE9FF4383B0064688461D464FF0000946
:101A5000344654B900BF502080F31188BFF34F8F34
:101A6000BFF36F8F00BF00BFFEE7B8F1000F01D1D9
:101A7000206C08B9012000E0002050B900BF5020C0
:101A800080F31188BFF34F8FBFF36F8F00BF00BF8C
:101A9000FEE7022D02D1E06B012801D1012000E018
:101AA000002050B900BF502080F31188BFF34F8F42
:101AB000BFF36F8F00BF00BFFEE700F04FFC08B917
:101AC000059808B9012000E0002050B900BF50205F
:101AD00080F31188BFF34F8FBFF36F8F00BF00BF3C
:101AE000FEE700BFFFF78AFBA06BE16B884201D3E2
:101AF000022D28D12A4641462046F7F738FA0746F4
:101B0000606A08B9012000E0002068B904F12400EF
:101B100000F0A8FD88B14FF0805032490860BFF353
:101B20004F8FBFF36F8F08E03FB14FF080502D49CA
:101B30000860BFF34F8FBFF36F8FFFF789FB012062
:101B400007B0BDE8F083059818B9FFF781FB0020C6
:101B5000F6E7B9F1000F04D101A8FFF767FC4FF0D9
:101B60000109FFF775FBFFF759FDFFF747FB94F9F4
:101B70004400401C10B9002084F8440094F945004A
:101B8000401C10B9002084F84500FFF761FB05A94F
:101B900001A800F00DFBF0B92046F7F79CFBA0B1BF
:101BA00004F110000599FFF753FC2046F7F7DCFB22
:101BB00000F0A4FD002895D14FF08050094908603D
:101BC000BFF34F8FBFF36F8F8CE72046F7F7CCFB47
:101BD00000F094FD86E72046F7F7C6FB00F08EFD87
:101BE0000020ADE704ED00E02DE9F84F07468A46F6
:101BF00090461E463C4654B900BF502080F31188E1
